:020000040000FA
:1000000000040020810A000015070000610A0000BA
:100010001F07000029070000330700000000000050
:10002000000000000000000000000000A50A000021
:100030003D070000000000004707000051070000D6
:100040005B070000650700006F07000079070000EC
:10005000830700008D07000097070000A10700003C
:10006000AB070000B5070000BF070000C90700008C
:10007000D3070000DD070000E7070000F1070000DC
:10008000FB070000050800000F0800001908000029
:10009000230800002D080000370800004108000078
:1000A0004B080000550800005F08000069080000C8
:1000B000730800007D080000870800009108000018
:1000C0009B080000A5080000AF080000B908000068
:1000D000C3080000CD080000D7080000E1080000B8
:1000E000EB080000F5080000FF0800000909000007
:1000F000130900001D090000270900003109000054
:100100003B0900001FB500F003F88DE80F001FBD8C
:1001100000F0ACBC40F6FC7108684FF01022401CA7
:1001200008D00868401C09D00868401C04D0086842
:1001300000F037BA9069F5E79069F9E7704770B554
:100140000B46010B184400F6FF70040B4FF0805073
:100150000022090303692403406943431D1B104621
:1001600000F048FA29462046BDE8704000F042BA47
:10017000F0B54FF6FF734FF4B4751A466E1E11E0DA
:10018000A94201D3344600E00C46091B30F8027B3B
:10019000641E3B441A44F9D19CB204EB134394B25D
:1001A00004EB12420029EBD198B200EB134002EBB2
:1001B000124140EA0140F0BDF34992B00446D1E952
:1001C0000001CDE91001FF224021684600F0F4FB58
:1001D00094E80F008DE80F00684610A902E004C8FB
:1001E00041F8042D8842FAD110216846FFF7C0FF7C
:1001F0001090AA208DF8440000F099F9FFF78AFFCB
:1002000040F6FC7420684FF01025401C0FD0206889
:1002100010226946803000F078F92068401C08D030
:100220002068082210A900F070F900F061F9A869AF
:10023000EEE7A869F5E74FF080500369406940F6A2
:10024000FC71434308684FF01022401C06D0086838
:1002500000F58050834203D2092070479069F7E788
:100260000868401C04D00868401C03D00020704778
:100270009069F9E70420704770B504460068C34DE3
:10028000072876D2DFE800F033041929631E250021
:10029000D4E9026564682946304600F062F92A46CE
:1002A0002146304600F031F9AA002146304600F0E0
:1002B00057FB002800D0032070BD00F009FC4FF46C
:1002C000805007E0201D00F040F90028F4D100F034
:1002D000FFFB60682860002070BD241D94E80700C3
:1002E000920000F03DFB0028F6D00E2070BDFFF715
:1002F000A2FF0028FAD1D4E901034FF0805100EBAE
:10030000830208694D69684382420ED840F6F8704E
:1003100005684FF010226D1C09D0056805EB8305B8
:100320000B6949694B439D4203D9092070BD55694A
:10033000F4E70168491C03D00068401C02D003E0C8
:100340005069FAE70F2070BD2046FFF735FFFFF731
:1003500072FF0028F7D1201D00F0F7F80028F2D135
:1003600060680028F0D100F0E2F8FFF7D3FE00F05B
:10037000BFF8072070BD10B50C46182802D0012028
:10038000086010BD2068FFF777FF206010BD41684E
:10039000054609B1012700E0002740F6F8742068FF
:1003A0004FF01026401C2BD02068AA68920000F065
:1003B000D7FA38B3A86881002068401C27D020688D
:1003C000FFF7BDFED7B12068401C22D026684FF051
:1003D0008050AC686D68016942695143A9420DD9EA
:1003E000016940694143A14208D92146304600F0E5
:1003F000B8F822462946304600F087F800F078F831
:100400007069D2E700F093F8FFF784FEF6E77069B1
:10041000D6E77669DBE740F6FC7420684FF01026DB
:10042000401C23D02068401C0CD02068401C1FD0EA
:100430002568206805F18005401C1BD027683879A5
:10044000AA2819D040F6F8700168491C42D001680A
:10045000491C45D00168491C3ED001680968491C07
:100460003ED00168491C39D000683EE0B069DAE747
:10047000B569DEE7B769E2E710212846FFF778FEA5
:100480003968814222D12068401C05D0D4F8001080
:1004900001F18002C03107E0B169F9E730B108CA63
:1004A00051F8040D984201D1012000E000208A4259
:1004B000F4D158B1286810B1042803D0FEE72846CB
:1004C000FFF765FF3149686808600EE0FFF722FE1C
:1004D00000F00EF87169BBE77169BFE7706904E06D
:1004E0004FF480500168491C01D000F0CBFAFEE7C0
:1004F000BFF34F8F26480168264A01F4E06111439B
:100500000160BFF34F8F00BFFDE72DE9F0411746B3
:100510000D460646002406E03046296800F054F8EF
:10052000641C2D1D361DBC42F6D3BDE8F08140F69B
:10053000FC700168491C04D0D0F800004FF48051D1
:10054000FDE54FF010208069F8E74FF080510A690F
:10055000496900684A43824201D810207047002050
:10056000704770B50C4605464FF4806608E0284693
:1005700000F017F8B44205D3A4F5806405F5805562
:10058000002CF4D170BD0000F40A0000000000202F
:100590000CED00E00400FA05144801680029FCD0C5
:1005A0007047134A0221116010490B68002BFCD0E0
:1005B0000F4B1B1D186008680028FCD0002010603D
:1005C00008680028FCD07047094B10B501221A605A
:1005D000064A1468002CFCD0016010680028FCD08A
:1005E0000020186010680028FCD010BD00E4014015
:1005F00004E5014070B50C46054600F073F810B9EB
:1006000000F07EF828B121462846BDE8704000F091
:1006100007B821462846BDE8704000F037B8000012
:100620007FB5002200920192029203920A0B000B06
:100630006946012302440AE0440900F01F0651F80C
:10064000245003FA06F6354341F82450401C8242F8
:10065000F2D80D490868009A10430860081D016827
:10066000019A1143016000F03DF800280AD00649C4
:1006700010310868029A10430860091D0868039A3F
:10068000104308607FBD00000006004030B50F4CED
:10069000002200BF04EB0213D3F800582DB9D3F8A1
:1006A000045815B9D3F808581DB1521C082AF1D3C3
:1006B00030BD082AFCD204EB0212C2F80008C3F8CD
:1006C00004180220C3F8080830BD000000E0014013
:1006D0004FF08050D0F83001082801D0002070473A
:1006E000012070474FF08050D0F83011062905D016
:1006F000D0F83001401C01D0002070470120704725
:100700004FF08050D0F830010A2801D00020704707
:100710000120704708208F490968095808471020B0
:100720008C4909680958084714208A4909680958FA
:100730000847182087490968095808473020854923
:100740000968095808473820824909680958084744
:100750003C20804909680958084740207D490968BC
:100760000958084744207B49096809580847482028
:1007700078490968095808474C207649096809589A
:10078000084750207349096809580847542071499F
:1007900009680958084758206E49096809580847E8
:1007A0005C206C4909680958084760206949096854
:1007B00009580847642067490968095808476820AC
:1007C00064490968095808476C2062490968095852
:1007D000084770205F4909680958084774205D4937
:1007E00009680958084778205A490968095808478C
:1007F0007C205849096809580847802055490968EC
:10080000095808478420534909680958084788202F
:1008100050490968095808478C204E490968095809
:10082000084790204B4909680958084794204949CE
:10083000096809580847982046490968095808472F
:100840009C204449096809580847A0204149096883
:1008500009580847A4203F49096809580847A820B3
:100860003C49096809580847AC203A4909680958C1
:100870000847B0203749096809580847B420354966
:10088000096809580847B8203249096809580847D3
:10089000BC203049096809580847C0202D4909681B
:1008A00009580847C4202B49096809580847C82037
:1008B0002849096809580847CC2026490968095879
:1008C0000847D0202349096809580847D4202149FE
:1008D000096809580847D8201E4909680958084777
:1008E000DC201C49096809580847E02019490968B3
:1008F00009580847E4201749096809580847E820BB
:100900001449096809580847EC2012490968095830
:100910000847F0200F49096809580847F4200D4995
:10092000096809580847F8200A490968095808471A
:10093000FC2008490968095808475FF48070054998
:10094000096809580847000003480449024A034B54
:100950007047000000000020000B0000000B0000AA
:1009600040EA010310B59B070FD1042A0DD310C82C
:1009700008C9121F9C42F8D020BA19BA884201D97E
:10098000012010BD4FF0FF3010BD1AB1D30703D0C6
:10099000521C07E0002010BD10F8013B11F8014B7C
:1009A0001B1B07D110F8013B11F8014B1B1B01D198
:1009B000921EF1D1184610BD02F0FF0343EA032254
:1009C00042EA024200F005B87047704770474FF0A6
:1009D00000020429C0F0128010F0030C00F01B800C
:1009E000CCF1040CBCF1020F18BF00F8012BA8BF1A
:1009F00020F8022BA1EB0C0100F00DB85FEAC17CDE
:100A000024BF00F8012B00F8012B48BF00F8012B90
:100A100070474FF0000200B51346944696462039C1
:100A200022BFA0E80C50A0E80C50B1F12001BFF4A7
:100A3000F7AF090728BFA0E80C5048BF0CC05DF80D
:100A400004EB890028BF40F8042B08BF704748BF5B
:100A500020F8022B11F0804F18BF00F8012B7047CF
:100A6000014B1B68DB6818470000002009480A4951
:100A70007047FFF7FBFFFFF745FB00BD20BFFDE719
:100A8000064B1847064A1060016881F308884068E1
:100A900000470000000B0000000B000017040000DE
:100AA000000000201EF0040F0CBFEFF30881EFF3ED
:100AB0000981886902380078182803D100E0000015
:100AC000074A1047074A12682C3212681047000084
:100AD00000B5054B1B68054A9B58984700BD0000B0
:100AE0007703000000000020F00A0000040000006E
:100AF000001000000000000000FFFFFF0090D00386
:10100000D80C00207589010069910000DB8801007F
:1010100069910000699100006991000000000000E2
:10102000000000000000000000000000018A010034
:1010300069910000000000006991000069910000C2
:10104000698A01006F8A01006991000069910000BE
:1010500069910000699100006991000069910000A8
:10106000758A010069910000699100007B8A010086
:1010700069910000818A0100878A01008D8A010040
:101080006991000069910000699100006991000078
:101090006991000069910000699100006991000068
:1010A00069910000938A0100699100006991000034
:1010B0006991000069910000699100006991000048
:1010C0006991000069910000699100006991000038
:1010D0006991000069910000699100006991000028
:1010E0006991000069910000699100006991000018
:1010F0006991000069910000699100006991000008
:10110000699100006991000000F002F817F021FCDD
:101110000AA090E8000C82448344AAF10107DA4552
:1011200001D117F016FCAFF2090EBAE80F0013F068
:10113000010F18BFFB1A43F0010318479C7D010003
:10114000BC7D01000A444FF0000C10F8013B13F085
:10115000070408BF10F8014B1D1108BF10F8015B10
:10116000641E05D010F8016B641E01F8016BF9D103
:1011700013F0080F1EBF10F8014BAD1C0C1B09D15A
:101180006D1E58BF01F801CBFAD505E014F8016BCC
:1011900001F8016B6D1EF9D59142D6D3704700005E
:1011A0000023002400250026103A28BF78C1FBD870
:1011B000520728BF30C148BF0B6070471FB500F011
:1011C00003F88DE80F001FBD17F0C0BB70B51B4CB6
:1011D00005460A202070A01C00F0D7F85920A080F6
:1011E00029462046BDE8704006F002BE06F00BBE60
:1011F00070B50C461249097829B1A0F160015E2949
:1012000008D3012013E0602804D0692802D043F2FB
:1012100001000CE020CC0B4E94E80E0006EB8000A1
:10122000A0F58050241FD0F8806E2846B04720607B
:1012300070BD0120704706207047000008000020A4
:101240001C000020BC8A01003249884201D20120E2
:1012500070470020704770B50446A0F500002E4E80
:10126000B0F1786F02D23444A4F5000429488442D6
:1012700001D2012500E0002500F043F848B125B96E
:10128000B44204D32548006808E0012070BD002066
:1012900070BD002DF9D1B442F9D321488442F6D271
:1012A000F3E710B50446A0F50000B0F1786F03D263
:1012B00019480444A4F5000400F023F84FF08041DD
:1012C00030B11648006804E08C4204D2012003E0EB
:1012D00013488442F8D2002080F0010010BD10B500
:1012E00020B1FFF7DEFF08B1012010BD002010BDC6
:1012F00010B520B1FFF7AFFF08B1012010BD0020ED
:1013000010BD084808490068884201D10120704793
:101310000020704700900100000000202000002005
:101320000800002050000020BEBAFECA10B50446D6
:101330000021012000F037F800210B2000F033F8E5
:101340000021082000F02FF80421192000F02BF8CC
:1013500004210D2000F027F804210E2000F023F8CE
:1013600004210F2000F01FF80421C84300F01BF8EF
:101370000621162000F017F80621152000F013F8BA
:101380002046FFF723FF002010BD4FF4937101802A
:101390007047FFF72BBF002070470B487047FFF7DF
:1013A00027BF704770474907090E002804DB00F18A
:1013B000E02080F80014704700F00F0000F1E020FA
:1013C00080F8141D7047000003F9004230B5FF4D4E
:1013D0000446062CA9780ED2DFE804F0030E0E0EA8
:1013E0000509FFDF08E0022906D0FFDF04E003293A
:1013F00002D0FFDF00E0FFDFAC7030BDF34810B576
:10140000407E4108F14800F11A0005D00CF023F9A4
:10141000BDE8104006F07EBB0CF004F9F8E730B5EB
:101420000446A1F120000D460A2847D2DFE800F06B
:1014300005070C19202532373C41FFDF3FE02078BB
:1014400020283CD1FFDF3AE0E0488078052836D0FC
:101450002078242833D0252831D023282FD0FFDF2F
:101460002DE0207822282AD0232828D8FFDF26E064
:101470002078222823D0FFDF21E0207822281ED0E8
:1014800024281CD026281AD0272818D0292816D07E
:10149000FFDF14E02078252811D0FFDF0FE020784F
:1014A00025280CD0FFDF0AE02078252807D0FFDFB1
:1014B00005E02078282802D0FFDF00E0FFDF25705C
:1014C00030BD1FB50022ADF800200C88ADF80240F9
:1014D0004B88ADF80430CA88ADF808208988ADF88B
:1014E00006100021ADF80A10ADF80C1080B14FF6CF
:1014F000FF700621844201D1ADF80210834201D170
:10150000ADF80410824203D14FF44860ADF80800F2
:1015100068460CF071F906F0FDFA04B010BD70B524
:1015200016460C460546FFF796FE50B90CB1B4427C
:1015300009D90C2070BD00BF55F82400FFF78BFEC1
:1015400008B1102070BD2046641EE4B2F4D270BD14
:101550002DE9F04105461F4690460E4600240068DE
:10156000FFF7C6FE30B9A98828680844401EFFF777
:10157000BFFE10B11020BDE8F08128680028A888BF
:1015800002D0B84202D850E00028F4D00920F2E797
:101590002968085DB8B1671CCA5D152A2ED03CDCED
:1015A000152A3AD2DFE802F03912222228282A2A04
:1015B0003131393939393939393939392200085D08
:1015C00030BB641CA4B2A242F9D833E00228DDD1BA
:1015D000A01C085C88F80000072801D2400701D44D
:1015E0000A20C8E7307840F0010015E0C143C90780
:1015F00007E0012807D010E00620BCE70107A1F1B1
:1016000080510029F5D01846B5E73078810701D51B
:101610000B20B0E740F0020030702868005D3844CD
:1016200084B2A888A04202D2B0E74FF4485382B2F5
:10163000A242ADD800209EE710B50278540809D028
:10164000012243F20223012C07D0022C0DD0032CDF
:1016500013D10FE00020087005E080790324B4EB7B
:10166000901F0AD10A70002010BD8079B2EB901F44
:1016700003D1F7E780798009F4D0184610BD08B58A
:1016800000208DF80000514890F8221049B190F8E0
:10169000230002280ED003280ED0FFDF9DF80000A3
:1016A00008BD4A486946193001F0AAF80028F5D06B
:1016B000FFDFF3E7032000E001208DF80000EDE7F5
:1016C00038B50C460546694601F09AF800280DD158
:1016D0009DF80010207861F34700207055F8010F45
:1016E000C4F80100A888A4F80500002038BD38B56A
:1016F0001378C0B1022816D035A46D462468009432
:101700004C7905EB9414247864F347031370032891
:101710000ED003F0FE0010700868C2F8010088883F
:10172000A2F8050038BD23F0FE0313700228EED1A5
:10173000D8B240F00100EEE702210DF0F3B938B560
:101740000C460978222901D2082038BDADF80000E6
:101750008DF8022068460BF0C1FF06F0DBF90500AA
:1017600003D121212046FFF75AFE284638BD1CB57B
:1017700000208DF80000CDF80100ADF805001348F9
:1017800090F82200022801D0012000E000208DF80E
:10179000070068460CF00CF8002800D0FFDF1CBDE5
:1017A0002DE9FF478CB00025BDF8346082461C4609
:1017B00090468DF81C50700703D56068FFF74BFD0D
:1017C00098B9024F97F8220004E00000940100202D
:1017D0000302FF014FF0010958B197F823000228D6
:1017E00007D16068FFF784FD18B1102010B0BDE884
:1017F000F087300702D5A089802815D8700704D457
:10180000B8F1000F01D0387E70B1E07DC0F3001058
:101810008DF81B00617D072041B1012906D0022906
:10182000E4D00429E2D117E00720DFE78DF8179014
:101830008DF819908DF81580606878B107A9FFF7C9
:10184000FBFE0028D2D1606850F8011FCDF80F10C0
:101850008088ADF8130005E00620C7E7CDF80F50EB
:10186000ADF81350E07B0028F6D1207C0028F3D19E
:10187000607C0028F0D1A07C0028EDD1E07CC0067F
:10188000EAD18DF800A0BDF83400ADF80200A068E0
:101890000190A0680290FBA0D0E90010CDE90A10E9
:1018A000E07C0AA901EB501000788DF80C00FFF7DE
:1018B000E6FE8DF80D009DF81C008DF80E008DF8E9
:1018C00018508DF816508DF81A5009A968460BF07B
:1018D000E2FF06F01FF989E7F0B58FB000248DF81C
:1018E00030408DF814408DF8344006468DF828407D
:1018F000019402940394049419B10FC901AD85E8D1
:101900000F00E24DA878052801D004280CD10198D9
:101910006968884200D120B90398E968884203D1F8
:1019200010B108200FB0F0BD1F273B460DAA05A936
:1019300003A8FFF70DFE0028F4D13B460AAA0CA924
:1019400001A8FFF705FE0028ECD19DF81400C007A0
:1019500001D00A20E6E7A88A410708D4A97D31B161
:101960009DF82810890702D043F20120DAE79DF89C
:101970002810C90709D0400707D4288818B144F2B5
:101980005061884201D90720CCE78DF818408DF8C6
:101990001960BDF80800ADF81A000198079006A874
:1019A0000BF084FF06F0B6F80028BBD18DF820407C
:1019B0008DF82160BDF81000ADF822000398099061
:1019C00008A80BF095FF06F0A5F80028AAD101ACF5
:1019D0002D1D94E80F0085E80F000020A2E72DE9F7
:1019E000FE43040000D1FFDF2078A84E20F00F0056
:1019F000801C20F0F0007030207060680178C91FF2
:101A0000112929D2DFE801F04BFD2809FDFD38ED51
:101A1000282864EDEC28EDEDEB0086883046FFF7D2
:101A20008BFE0546304609F05AFFB8B160688079F0
:101A300085F83E0021212846FFF7F1FC304603F0EF
:101A40001FFA304604F0DEFB3146012010F09CFE08
:101A5000A87F20F01000A877BDE8FE83207820F052
:101A6000F00020302070032020726680606880794A
:101A7000607206F03EFADDE785882846FFF75CFED7
:101A800000B9FFDF60688078012800D0FFDF606860
:101A9000817903B02846BDE8F04309F0FDBF868890
:101AA0003046FFF749FE050000D1FFDF06F021FABE
:101AB00060683146C08828816068008968816068F4
:101AC0004089A881012010F05FFE0020A875C3E7BF
:101AD000807828B10228BFD03C28BDD0FFDFBBE70B
:101AE00006F007FA6568A879AD1C00B9FFDFF77842
:101AF000B5F80290B046384605F0ACFF060000D1BC
:101B0000FFDF0022022148460DF003F8040000D157
:101B1000FFDF22212046FFF782FCA17F012060F336
:101B20000101A177298B2181698B6181A98BA18119
:101B300084F822708DF8080002AA032148460CF0B0
:101B4000E8FF00B9FFDFB088ADF80400B0788DF889
:101B5000060001AA052148460CF0DBFF00B9FFDFB3
:101B6000B088ADF80000F0788DF802006A460421D4
:101B700048460CF0CEFF00B9FFDF062105F1120048
:101B80000BF0D9F808B36879800700D5FFDF6979D1
:101B9000E07D61F34700E075D5F80600A061688933
:101BA000A083062105F10C000BF0C5F8D8B198F818
:101BB00019104A08617862F347016170D8F81A1069
:101BC000C4F80210B8F81E0016E0E07D20F0FE0018
:101BD000801CE075D5F81200A061E88AE0E715E006
:101BE00020E01BE00DE0607820F0FE00801C6070BB
:101BF000E868C4F80200288AE0800320FFF7E6FBCB
:101C00002AE72046BDE8FE4301F0C0BC06F071F9AA
:101C100016F8240F40F0040030701DE7BDE8FE43C5
:101C200006F067B9B178052908D00429E8D106F093
:101C300060F90220BDE8FE43FFF7C8BB80780028AA
:101C4000DED0F07800F0C3FD06F053F90320F1E791
:101C50002DE9F047054600780027000991460C461B
:101C60003E4601287AD0022879D0072810D00A28C9
:101C70002BD0FFDFA9F800600CB127806680002020
:101C8000B5E50000070605040302010094010020E9
:101C9000D5F804C0DFF8B4874FF0010A9CF80000C3
:101CA0004FF6FF7113287AD008DC07280ED00E28D3
:101CB0001FD0112826D0122806D186E015280BD077
:101CC000162859D017286CD02146FBE01227102681
:101CD000BCF804002146B8E01C270A26ECB3BCF887
:101CE0000200A0806868007920726868407960729C
:101CF000C0E71B27092684B3032020726868408848
:101D0000A080B7E79CF802003C28B3D010272C260F
:101D10000CF1020C0CB3BCF80200A080BCF8180057
:101D20006082BCF818002082BCF81A00A082BCF8BF
:101D30001C00E0829CF8050004F108020CF1060189
:101D4000FFF7D5FC9CF80400012893D184F80FA07C
:101D50000020207608F1040002E00AE06DE077E060
:101D600090E80E00D8F81000C4E90930C4E9071261
:101D700080E7A9F8006082E720271126002CF8D020
:101D8000A180686804F10A02807820726868807A0D
:101D900060726968C878091DFFF7A9FC6AE729E045
:101DA000FFE721270A26002CE3D0BCF80200A08020
:101DB00068680079207268684079607298F8241029
:101DC00021F0040188F8241054E722270B26002C68
:101DD000CFD0BCF80400A080686880782072686862
:101DE000807900F02AFD60726868C07900F025FDF6
:101DF000A0723FE726271C26002CBAD0A180686875
:101E0000C078607268688079A07208F1040090E878
:101E10000E00D8F81000C4E90530C4E90312686860
:101E200080783C2803D0432804D0FFDF22E784F8E1
:101E300008A01FE7022020721CE7287A022801D0A0
:101E4000FFDF17E712271026688800F0E3FC11E790
:101E5000287AB0B3012835D0022833D0032801D026
:101E6000FFDF07E711270926002C82D0B5F8028092
:101E70004046FFF761FC90F822A0A4F80480687A3D
:101E80002072042140460CF05FFE052140460CF014
:101E90005BFE002140460CF057FE012140460CF04D
:101EA00053FE032140460CF04FFE022140460CF049
:101EB0004BFE062140460CF047FE504600F087FCE2
:101EC000D8E6FFE72846BDE8F04701F095BC70B5BD
:101ED000012801D0FFDF70BD8DB22846FFF72CFC32
:101EE000040000D1FFDF20782128F4D005F0FEFFA8
:101EF00080B1017821F00F01891C21F0F00110312F
:101F000001700221017245800020A075BDE870407B
:101F100005F0EFBF21462846BDE8704013220EE4CD
:101F20002DE9F04116460C00804600D1FFDF3078E5
:101F300020F00F00801C20F0F0001030307020786E
:101F4000022802D0FFDFBDE8F0814046FFF7F4FB36
:101F5000050000D1FFDF61884FF6FF700027814246
:101F600002D1A288824203D0814201D1A08848B127
:101F700005F0BFFF2068B0606068F06020893082A3
:101F8000AF75E0E7A87D0128DDD178230022414626
:101F900010F050FB0220A875D5E738B520380C4664
:101FA000072838D2DFE800F004062A372F251A0068
:101FB000062038BD6068FFF792F9A0B961882088D3
:101FC0006A460BF002FE05F0A5FD0028F1D161681C
:101FD0000029EED0BDF800200A8038BD206820B16D
:101FE000FFF786F908B1102038BD20460BF0B8FE87
:101FF0000DE0A17820880BF019FE08E02068BDE80C
:10200000384001F02EBE618820880BF077FDBDE8D6
:10201000384005F07FBD072038BD70B505460C4639
:102020000846FFF73EF908B1102070BD202D07D0FB
:10203000212D0DD0222D0BD0252D09D0072070BDCC
:102040002088A11C0BF099FBBDE8704005F062BD33
:10205000062070BDFD481930704708B528220021C0
:10206000FA4809F004FA0120FFF7B0F9F749684689
:102070001A3105F0D1FEF5489DF80020417E62F34B
:10208000470121F001014176002180F822104FF430
:1020900061710184022180F82310FFF7AFF900B1CC
:1020A000FFDF00F0FBFB01F043FA08BD10B50C4662
:1020B00040220021204609F0DAF9A07F20F0030039
:1020C000A077202020700020A07584F8230010BD88
:1020D00070472DE9FC410746FFF7BDF810B110200D
:1020E000BDE8FC81D94E06F11901D6F8190000901F
:1020F000B6F81D50ADF80450F47F8DF80640384610
:10210000FFF7DEFA0028EBD1FFF778F90028E7D0D7
:10211000009946F8191FB580B471E1E710B504467F
:10212000FFF7BFF808B1102010BDC848C7492246C4
:10213000407E1A314008FFF7DAFA002010BD3EB5A4
:1021400004460D460846FFF7ACF808B110203EBD26
:1021500014B143F204003EBDBC488078052803D08A
:10216000042801D008203EBD694602A809F01CFFE2
:102170002A4669469DF80800FFF7B9FA00203EBDDF
:10218000FEB50D4604004FF0000712D00822FFF7FD
:10219000C6F9002812D1002609E000BF54F8260035
:1021A0006946FFF749FA002808D1761CF6B2AE421C
:1021B000F4D30BF08CF910B143F20320FEBDA34E13
:1021C0003776FCB100271AE054F8270002A9FFF780
:1021D00033FA00B1FFDF9DF808008DF8000054F8D5
:1021E000270050F8011FCDF801108088ADF80500D8
:1021F00068460BF091F900B1FFDF7F1CFFB2AF42E0
:10220000E2D335760020FEBD2DE9F0418AB01546B7
:10221000884604001DD00F4608222946FFF77FF9A3
:10222000002810D1002612E054F82600694610302C
:1022300000F0E6FA002806D13FB157F82600FFF774
:102240000AF810B110200AB07DE6761CF6B2AE4254
:10225000EAD3681EC6B217E0701CC7B212E000BF16
:1022600054F82600017C4A0854F827100B7CB2EB86
:10227000530F05D106221130113109F0A1F850B1E8
:102280007F1CFFB2AF42EBD3761EF6B2E4D24646D5
:1022900024B1012003E043F20520D4E700200BF035
:1022A0005AF910B90BF063F910B143F20420CAE7F0
:1022B00064B300270DF1170826E000BF54F827008B
:1022C0006946103000F09CFA00B1FFDF54F8270097
:1022D000102250F8111FCDF801108088ADF80500CC
:1022E00054F827100DF1070009F097F896B156F849
:1022F00027101022404609F090F868460BF0F1F8DC
:1023000000B1FFDF7F1CFFB2AF42D7D3FFF72FFA38
:10231000002098E7404601F098FCEEE730B585B024
:102320000446FEF798FF18B96068FEF7E1FF10B1A8
:10233000102005B030BD60884AF2B811884206D836
:102340002078424D28B1012806D0022804D0072069
:10235000EFE7FFF753F818E06078022804D003286D
:1023600002D043F20220E4E785F82300C1B2002046
:102370000090ADF8040002292CD0032927D0FFDFFC
:1023800068460BF068F905F0C5FB0028D1D16068FC
:1023900001F04EFC207858B101208DF800000DF1BD
:1023A000010001F052FC68460BF0A7FC00B1FFDF12
:1023B000207885F82200FFF7DAF9608860B1288478
:1023C00080B20BF0C0F800B1FFDF0020B1E78DF85C
:1023D0000500D5E74020FAE74FF46170EFE710B54C
:1023E0000446FEF75EFF20B9606838B1FEF777FF5C
:1023F00008B1102010BD606801F027FC134830F8C8
:10240000201F6180C178617080782070002010BD2D
:102410002DE9F843144689460646FEF742FFB8B94F
:102420004846FEF765FF98B92046FEF761FF78B988
:10243000064DA878012800D154B13178FF2909D080
:1024400061B143F20400BDE8F8830000940100206C
:102450001020F8E7012801D00420F4E7CCB30528C8
:1024600011D004280FD06946204600F0F1F9002869
:10247000E9D1217D49B1012909D0022909D00329D7
:1024800009D00720DFE70820DDE7024604E001224B
:1024900002E0022200E00322804623461746002085
:1024A0000099FFF77DF90028CDD1A0892880A07B75
:1024B000E875BDF80000A882AF75BDF800100907E7
:1024C00001D5A18931B1A1892980C00704D0032099
:1024D00003E006E08021F7E70220FEF777FF86F8A9
:1024E00000804946BDE8F8430020FFF7F5B92DE923
:1024F000FC41E94C06460D46A078022803D003288B
:1025000001D00820ECE516B143F20400E8E506200E
:102510000CF0BCFA10B9A078032849D00EF020FACC
:1025200007460FF089FC381A00F0FF0806200CF06F
:10253000A5FA074606200CF0A9FA391AA078042853
:1025400009D000221144A8EB010111F0FF0F04D0C3
:10255000032804D00DE00122F4E71320C0E528464B
:1025600005F078FA10B3407810B3284605F065FD01
:10257000E570FFF784F809F062FC01208DF8000097
:102580008DF801008DF802602088ADF80400E07D30
:102590008DF8060068460BF074FA05F0BBFA0028C7
:1025A000B0D1A078032805D0042010E0052097E5DD
:1025B000122095E5E07805F04DFA040000D1FFDF28
:1025C000607800B9FFDF6078401E60700520FEF77C
:1025D000FDFE002084E51CB510B143F204001CBDD3
:1025E000AD4CA078042803D0052801D008201CBDDC
:1025F00000208DF8000001218DF801108DF80200F7
:1026000068460BF03EFA05F085FA0028EFD1A07875
:10261000052805D05FF00200FEF7D8FE00201CBDA3
:10262000E07800F0D4F80320F6E72DE9FC4180467D
:102630000D4603260846FEF75BFE08B110204FE565
:102640004046FFF779F8040004D02078222804D20D
:10265000082045E543F2020042E5A07F00F00307B1
:102660003DB1012F0AD000202946FEF72AFF0600BF
:10267000E5D1012F04D0FFDF304631E50120F3E73B
:10268000A07D2946022801D011B107E0112027E5DD
:10269000684600F037FA0028D1D16946404609F073
:1026A000DBF90600E8D10120A075E5E770B50C461E
:1026B0000546FFF741F8010005D022462846BDE84F
:1026C0007040FFF73CB843F2020070BD10B501281E
:1026D00007D1714B9B78012B00D011B143F204005C
:1026E00010BD0AF062FFBDE8104005F013BA0123E7
:1026F00000F077B800231A46194600F072B870B59A
:10270000064615460C460846FEF7CBFD18B9284686
:10271000FEF7C7FD08B1102070BD2A46214630469D
:102720000BF03BFA05F0F6F90028F5D121787F2966
:10273000F2D1052070BD7CB505460C460846FEF773
:102740008AFD08B110207CBD2846FEF7F5FF20B1B8
:102750000078222804D208207CBD43F202007CBD10
:102760004D4890F82400400701D511207CBD217808
:10277000C80802D16078C20801D007207CBD890852
:1027800001D1800801D006207CBDADF80050207832
:102790008DF8020060788DF803000220ADF8040087
:1027A00068460AF035FE05F0B5F97CBD70B5054602
:1027B0000C460846FEF775FD08B1102070BD214695
:1027C00028460BF00BF8BDE8704005F0A3B910B532
:1027D00005F040F9040000D1FFDF6078401C607014
:1027E00010BD1CB5ADF800008DF802308DF8031057
:1027F0008DF8042068460BF09FF905F08BF91CBD9D
:102800000278520804D0012A02D043F20220704715
:10281000FEF712BF70B50C0006460DD0FEF78CFF18
:10282000050000D1FFDFA6802889208128896081EA
:102830006889A081A889E08170BD00B530B1012808
:1028400003D0022801D0FFDF002000BDFF2000BD23
:1028500000220A8092B222F060020A8000780628E4
:1028600017D2DFE800F0160306090C1142F0110040
:1028700007E042F01D0009E042F0150006E042F0DA
:10288000100040F0020001E042F01000088000203B
:10289000704707207047000094010020FD48002188
:1028A00001604160018170472DE9FF4F93B09B4665
:1028B000209F160004460DD01046FEF7CCFC18B140
:1028C000102017B0BDE8F08F31460120FEF7F9FD6A
:1028D0000028F6D101258DF842504FF4C050ADF8D4
:1028E0004000002210A9284603F051FF0028E8D13B
:1028F0008DF84250A8464FF428500025ADF840000E
:102900001C2229466846079508F0B1FD9DF81C0079
:102910000DF11C0A20F00F00401C20F0F0001030D8
:102920008DF81C0020788DF81D0061789DF81E0040
:102930000DF1400961F3420040F001008DF81E00E6
:102940009DF8000008AA40F002008DF800002089E0
:10295000ADF83000ADF832506089ADF83400CDF8F4
:102960002CA060680E900AA9CDF82890684603F064
:102970001CFD0028A5D16068FEF7B1FC40B160687D
:10298000FEF7B6FC20B9607800F00300022801D001
:10299000012000E00020BF4C08AA0AA92072BDF85F
:1029A000200020808DF8428042F60120ADF84000E2
:1029B0009DF81E0020F00600801C20F001008DF81C
:1029C0001E000220ADF83000ADF8340014A80E90BF
:1029D000684603F0EAFC002889D1BDF82000608039
:1029E00036B1211D304600F059F90028C2D109E066
:1029F000BBF1000F05D008F0B5FAE8BB08F0B2FA59
:102A0000D0BBA58017B1012F43D04AE08DF842809A
:102A100042F6A620ADF8400046461C22002168463A
:102A2000079508F024FD9DF81C00ADF8346020F0F7
:102A30000F00401C20F0F00010308DF81C009DF8B5
:102A40001D0020F0FF008DF81D009DF81E0020F0F5
:102A5000060040F00100801C8DF81E009DF800006B
:102A60008DF8446040F002008DF80000CDE90A9A2C
:102A7000ADF8306011A800E011E00E9008AA0AA994
:102A8000684603F092FC0028A6D1BDF82000E08043
:102A900008E008F067FA10B908F064FA08B10320FA
:102AA0000FE7E58000200CE73EB50446794D08208D
:102AB000ADF80000A88828B12046FEF7CCFB18B17D
:102AC00010203EBD06203EBD21460120FEF7F9FC48
:102AD0000028F8D12088ADF804006088ADF8060021
:102AE000A088ADF80800E088ADF80A00A88801AB1E
:102AF0006A46002104F036F8BDF800100829E2D03B
:102B000003203EBD7FB5634D0446A88868B1002010
:102B100002900820ADF80800CDF80CD02046FEF752
:102B20009AFB20B1102004B070BD0620FBE7A988F5
:102B300002AA4FF6FF7004F058FA0028F3D1BDF84E
:102B40000810082901D00320EDE7BDF8001021800E
:102B5000BDF802106180BDF80410A180BDF8061018
:102B6000E180E0E701B582B00220ADF800004948FD
:102B700002AB6A464088002103F0F4FFBDF8001064
:102B8000022900D003200EBD1CB5002100910221B6
:102B9000ADF800100190FEF784FB08B110201CBDB9
:102BA0003C486A4641884FF6FF7004F01EFABDF8B3
:102BB00000100229F3D003201CBDFEB5354C06469B
:102BC0001546207A0F46C00705D00846FEF743FB9E
:102BD00018B11020FEBD0F20FEBDF82D01D90C202C
:102BE000FEBD3046FEF737FB18BB208801A903F075
:102BF000C6F80028F4D130788DF80500208801A9A6
:102C000003F08FFF0028EBD100909DF800009DF8A5
:102C1000051040F002008DF80000090703D040F0D5
:102C200008008DF800002088694603F017FF00288F
:102C3000D6D1ADF8085020883B4602AA002103F007
:102C400091FFBDF80810A942CAD00320FEBD7CB593
:102C500005460020009001900888ADF800000C4661
:102C600028460195FEF73BFB18B92046FEF719FBF5
:102C700008B110207CBD15B1BDF8000060B1054859
:102C80006A4601884FF6FF7004F0AFF9BDF80010F6
:102C900021807CBDBC0100200C20FAE730B5044641
:102CA00093B000200D4601460090142201A808F0C0
:102CB000DEFB1C22002108A808F0D9FB9DF80000CB
:102CC000CDF808D020F00F00401C20F0F0001030AC
:102CD0008DF800009DF8010006AA20F0FF008DF895
:102CE00001009DF8200001A940F002008DF82000AD
:102CF00001208DF8460042F60420ADF8440011A8EA
:102D000001902088ADF83C006088ADF83E00A088B6
:102D1000ADF84000E088ADF842009DF8020020F0D8
:102D20000600801C20F001008DF802000820ADF89C
:102D30000C00ADF810000FA8059008A803F035FBB3
:102D4000002803D1BDF818002880002013B030BD42
:102D50004FF0E0214FF40040C1F88001BFF34F8FE6
:102D6000BFF36F8F00F021B810B5044600F01DF8D6
:102D7000002C09D0124A124812491432124B012C6D
:102D800003D0022C07D0FFDF10BD022404601160C5
:102D90004FF0407004E00324046011604FF4000021
:102DA000186010BD00B5FFDF00BD054800210160BF
:102DB000016005494FF06070091D08607047000010
:102DC00000F500403C02002004F501400EF0E2BC9A
:102DD0000449002008604FF0E0210220C1F8800281
:102DE00070470000FC1F0040334901200860704715
:102DF00070B50D2000F041F8304C0020C4F80001FF
:102E00000125C4F804530D2000F048F825604FF068
:102E1000E0216014C1F8000170BD10B50D2000F074
:102E20002CF82648012141600021C0F80011BDE8BE
:102E300010400D2000F032B8204910B5D1F8000143
:102E4000012801D0FFDF10BD1B48001D00680022D3
:102E5000C0B2C1F80021BDE810400FF0D8B910B5DC
:102E6000164800BFD0F800110029FBD0FFF7E4FF9F
:102E7000BDE810400D2000F011B800280DDB00F077
:102E80001F02012191404009800000F1E020C0F8BC
:102E90008011BFF34F8FBFF36F8F7047002809DB9E
:102EA00000F01F02012191404009800000F1E02064
:102EB000C0F880127047000004D5004000D00040E8
:102EC0004FF0E0214FF00070C1F8800101F5C071B2
:102ED000BFF34F8FBFF36F8FC1F80001354B8022D6
:102EE00083F8002441F8800C704700B502460420A6
:102EF000314903E001EBC0031B792BB1401EC0B286
:102F0000F8D2FFDFFF2000BD41F8302001EBC00107
:102F100000224A718A7101220A7100BD264A0021ED
:102F200002EBC0000171704710B50446042800D3BD
:102F3000FFDF214800EBC4042079012800D0FFDF27
:102F40006079A179401CC0B2814200D060714FF01D
:102F5000E0214FF00070C1F8000210BD70B50425EB
:102F6000154E164C16E0217806EBC1000279012AB5
:102F700008D1427983799A4204D04279827156F815
:102F8000310080472078401CC0B22070042801D353
:102F9000002020706D1EEDB2E5D270BD054810B561
:102FA00090F800044009042800D0FFDFBDE810407D
:102FB000D4E7000019E000E08C0400204C00002061
:102FC0000348044A0168914201D100210160704721
:102FD00050000020BEBAFECA70B50C46054606F089
:102FE00021FC21462846BDE8704007F002BD70472D
:102FF00070477047100110013A0200001A020000E9
:103000002CFFFFFFDBE5B151009001002601FFFF1F
:103010007000000078DB6A007A2E9AC67DB66CFAE2
:10302000F35721CCC310D5E51471FB3C10B5044611
:10303000FEF711F908B1102010BD2078C0F302107E
:10304000042807D86078072804D3A178102901D86C
:10305000814201D2072010BDE078410706D42179D2
:103060004A0703D4000701D4080701D5062010BD84
:10307000002010BD70B514460D46064604F036FF1C
:1030800080B10178182221F00F01891C21F0F00194
:10309000A03100F8081B214608F0BFF9BDE87040D8
:1030A00004F027BF29463046BDE870401322FEF7E2
:1030B00046BB2DE9F047064608A8904690E8300444
:1030C00089461F4614220021284608F0D0F9002125
:1030D000CAF80010B8F1000F03D0B9F1000F03D106
:1030E00014E03878C00711D02068FEF7DAF8C0BBCA
:1030F000B8F1000F07D12068123028602068143022
:1031000068602068A8602168CAF8001038788007D5
:1031100024D56068FEF7E3F818BBB9F1000F21D0A1
:10312000FEF798FF0168C6F868118188A6F86C114F
:10313000807986F86E0101F032FAF84FEF6062682C
:1031400062B196F8680106F2691140081032FEF784
:10315000CEFA10223946606808F05FF90020BDE819
:10316000F08706E0606820B1E8606068C6F8640136
:10317000F4E71020F3E730B5054608780C4620F058
:103180000F00401C20F0F001103121700020607011
:1031900095F8230030B104280FD0052811D0062857
:1031A00014D0FFDF20780121B1EB101F04D295F875
:1031B000200000F01F00607030BD21F0F0002030D2
:1031C00002E021F0F00030302070EBE721F0F00059
:1031D0004030F9E7F0B591B0022715460C46064697
:1031E0003A46ADF80870082103AB08F019FA0490CC
:1031F000002810D004208DF804008DF80170E03410
:10320000099605948DF818500AA968460DF083F9BF
:1032100000B1FFDF012011B0F0BD2DE9F84F0646E7
:10322000808A0C4680B28246FEF786FA0546BB4F7E
:103230003078203F4FF002094FF000080F287CD271
:10324000DFE800F07BA39D082C5B6A7CBADAFD976F
:1032500048979700012150460BF064FC040000D110
:10326000FFDF97F85C00C00701D0386E0BE0032148
:1032700004F11D000EF0A9FFD4F81D00A849B0FB11
:10328000F1F201FB1200C4F81D0070686067B068BD
:10329000A0672878252872D0FFDF70E00121504612
:1032A0000BF040FC060000D1FFDF3078810702D52B
:1032B0002978252904D040F001003070BDE8F88F4E
:1032C00084F80090307F207106F11D002D36C4E98E
:1032D0000206F3E7012150460BF024FC050000D163
:1032E000FFDF2878C10604D5072020703D356560D2
:1032F000E4E740F008002870E0E7E87F000700D529
:10330000FFDF307CB28800F0010301B05046BDE819
:10331000F04F082108F01DBB05B9FFDF716821B12E
:10332000102205F1240008F078F828212846FEF73D
:1033300076F8307A85F82000C0E7F7E001215046A2
:103340000BF0F0FB050000D1FFDF022105F1850045
:103350000EF03BFF0420207005F5B4706060B5F8F6
:10336000850020826D4810387C356561C4E90270A3
:10337000A4E7012150460BF0D5FB00B9FFDF324630
:1033800029465046BDE8F84F74E605B9FFDF2878B6
:10339000212893D93079012803D1E87F40F0080033
:1033A000E877324629465046FFF764FE2846BDE8D6
:1033B000F84F2321FEF733B83279A28004F10803D5
:1033C0000821504608F02CF9E06010B1052020706B
:1033D00074E74546012150460BF0A4FB040000D1E0
:1033E000FFDF04F1620102231022081F0BF03FFAF5
:1033F00005703179417061E7012150460BF092FB75
:10340000040000D1FFDF94F8840000F003000128DD
:1034100059D1E87F10F0010003D194F8A010C9073A
:103420002AD0D4F8602132B394F88330117C63F34E
:1034300087011174AA7FD30963F3410100E071E0B1
:10344000D4F860211174D4F8602160F30001117484
:1034500090B1D4F86001102205F12401883407F0FE
:10346000DCFF207E40F001002076207820F0010073
:1034700004F8880919E0C0B994F88810C90714D075
:10348000D4F85C218AB194F88330117C63F387010E
:103490001174AA7FD309D4F85C2163F3410111743C
:1034A000D4F85C2160F30001117494F8880080075F
:1034B00009D594F87C00D4F86421400804F17D011A
:1034C0001032FEF714F98DF8009094F884006A46E3
:1034D00000F003008DF8010094F888108DF80210B8
:1034E00094F8A0008DF803002946504601F040F8FA
:1034F0002878252805D0212807D0FFDF2878222822
:1035000003D922212846FDF78AFF012150460BF0FE
:103510001BFB00283FF4DDAEFFDFCFE6E801002013
:1035200040420F00716881F80180C7E6FFDFC5E601
:1035300070B5FE4C002584F85C5025660CF0B7FF92
:1035400004F11001204604F08DFC84F8305070BD69
:1035500070B50D46FEF7F0F8040000D1FFDF4FF420
:10356000B8720021284607F082FF2434012105F1BA
:10357000E0002C610CF09CFF002800D0FFDF70BD44
:103580000A46014602F1E0000CF0B3BF70B50546F3
:10359000406886B00178082906D00B2933D00C2961
:1035A0002FD0FFDF06B070BD46883046FEF7C4F866
:1035B000040000D1FFDF20782128F3D028281BD178
:1035C000686802210C3000F09DFFA8B168680821EE
:1035D000001D00F097FF78B104F1240130460AF095
:1035E00052FA04F097FA00B1FFDF06B02046BDE8BA
:1035F00070402921FDF713BF06B0BDE8704004F00C
:1036000078BC01218171686886883046FEF794F89D
:10361000040000D1FFDF20782128C3D068688179B9
:1036200009B1807808B1FFDFBCE704F062FCA07F3D
:10363000000622D5E07FC00705D094F8200000F0F6
:103640001F00102817D0052084F82300207829288F
:1036500015D02428A6D1314604200FF095F8222158
:103660002046FDF7DCFE012130460BF06DFA002804
:1036700098D0FFDF96E70620E6E70420E4E7012183
:1036800030460BF04FFA050000D1FFDF2521204620
:10369000FDF7C5FE03208DF80000694605F1E00046
:1036A0000CF01EFF0228BFD00028BDD0FFDF79E755
:1036B0002DE9F04788B09A46164688468146FEF7BF
:1036C0003BF805003AD02878222837D3232835D074
:1036D000E87F000732D40027012148460BF022FA88
:1036E000040005D10121002248460BF012FA0446DD
:1036F000694600F064FF009800B9FFDF00983CB114
:10370000E03404612878222804D0242802D005E07F
:10371000076103E025212846FDF781FE009801217D
:103720004170C0F824908680C0E9028A01A90CF09B
:10373000F2FE022802D0002800D0FFDF08B00EE51C
:1037400070B586B00546FDF7F7FF0078222814D93A
:10375000012128460BF0E6F904002CD1FFDF2AE016
:10376000B4F85E0004F1620630440178427829B171
:1037700021462846FFF72EFDB0B913E7ADF8042027
:103780000821284602AB07F04BFF03900028F4D035
:1037900005208DF80000694604F1E0000CF0A0FE61
:1037A000022801D000B1FFDF02231022314604F1CC
:1037B0005E000BF092F8B4F860000028D0D1F1E67A
:1037C00010B586B00446FDF7B7FF0078222811D95E
:1037D000012120460BF0A6F9040000D1FFDF0620EE
:1037E0008DF80000694604F1E0000CF079FE002835
:1037F00000D0FFDF06B010BD2DE9F84F0546007878
:103800000C460027010904F1080090463E46BA46DE
:10381000009002297ED0072902D00A2909D142E06E
:1038200068680178082905D00B292CD00C292AD0EA
:10383000FFDF72E114271C26002C6CD04088A0808A
:10384000FDF77AFF5FEA000900D1FFDF99F8170062
:1038500009F118014008009AFDF749FF686880895E
:10386000208268684168C4F812108068C4F81600A5
:10387000A07E20F0060040F00100A07699F81E001E
:1038800040F020014FE01A270A26002CD5D080886E
:10389000A080FDF751FF050000D1FFDF2846009909
:1038A000FFF769FC39E10CB1A88BA080287A4FF0B2
:1038B000010B0B287ED006DC01287CD0022808D022
:1038C000032804D137E00D2876D00E2875D0FFDF0D
:1038D00023E11E270926002CAFD0A088FDF72CFF7E
:1038E0005FEA000900D1FFDF287B00F00300012818
:1038F000207A1DD020F001002072297B890861F315
:1039000041002072297BC90861F382002072297B63
:10391000090901E0F7E0AEE061F3C300207299F815
:103920001E0040F0400189F81E10F6E0C80100209A
:1039300040F00100E0E713270D26002CA6D0A08858
:10394000FDF7FAFE81460121A0880BF0EBF8050097
:1039500000D1FFDF686F817801F003010129217A2E
:1039600050D021F00101217283789B0863F341015B
:1039700021728378DB0863F38201217283781B094B
:1039800063F3C3012172037863F306112172437854
:1039900063F3C711217284F809A0C178A17202797A
:1039A000E17A62F30001E1720279520862F34101A7
:1039B000E17203E029E067E04EE05FE002799208FF
:1039C00062F38201E1720279D20862F3C301E1720B
:1039D0004279217B62F3000121734279520862F33C
:1039E000410121734279920862F382012173407987
:1039F000C00860F3C301217399F8000023282AD975
:103A0000262139E041F00101ADE71827102694B3D3
:103A1000A088FDF791FE00900121A0880BF082F8AC
:103A20005FEA000900D1FFDFE868A06099F80000B4
:103A300040F0040189F8001099F80100800708D5CA
:103A400084F80CB000980078232866D927210098C4
:103A500052E084F80CA060E015270F265CB1A08826
:103A6000FDF76AFE81460622E868009907F05DFDD1
:103A700084F80EB085E042E048463DE0162709266E
:103A8000ECB3287B207248E0287B19270E26B4B3BC
:103A9000C4F808A0A4F80CA0012807D0022808D078
:103AA00003280CD004280AD0FFDF15E084F808B002
:103AB00001E002202072607A20F003000BE0697BB5
:103AC000042801F00F0141F080012172F3D1607AE6
:103AD00020F00300401C6072A088FDF72DFE054613
:103AE0000078212819D0232800D0FFDF0121A088E9
:103AF0000BF02AF822212846FDF791FC0DE0FFE7A4
:103B0000A8F800600EE00CB16888A080287A10B395
:103B1000012809D002283AD0FFDFA8F800600CB1D4
:103B200027806680002007E415270F26002CE7D0A9
:103B3000A088FDF701FE0121A0880AF0F3FF05002F
:103B400000D1FFDFD5F81D000622009907F0EDFC3B
:103B500084F80EA0E1E717270926002CD0D0A08812
:103B6000FDF7EAFD81460121A0880AF0DBFF050090
:103B700000D1FFDF6878800701D5022000E0012036
:103B8000207299F800002328C7D9272174E7192744
:103B90000E26002CB4D0A088FDF7CEFD5FEA000908
:103BA00000D1FFDFC4F808A0A4F80CA084F808A096
:103BB000A07A40F00300A07299F81E10C90961F3C1
:103BC0008200A07299F81F2099F81E1012EAD11FE6
:103BD00005D099F8201001F01F01102925D020F000
:103BE0000800A07299F81F10607A61F3C300607238
:103BF000697A01F0030101298FD140F0040060725D
:103C0000E87A217B60F300012173AA7A607B62F37A
:103C100000006073EA7A520862F341012173A97AC5
:103C2000490861F34100607377E740F00800D8E786
:103C300010B5FE4C30B10146102204F1200007F00F
:103C4000ECFB012084F8300010BD10B5044600F0F4
:103C5000A6FCF64920461022BDE81040203107F0AE
:103C6000DCBB70B5F14D06004FF0000412D0FDF73B
:103C7000F2FA08B110240BE00621304607F03CFCB4
:103C8000411C04D02866012085F85C0000E0072470
:103C9000204670BD0020F7E7007810F00F0204D036
:103CA000012A05D0022A0CD110E0000909D10AE04E
:103CB0000009012807D0022805D0032803D00428D2
:103CC00001D0072070470870002070470620704719
:103CD00005282AD2DFE800F003070F171F00087835
:103CE00020F0FF001EE0087820F00F00401C20F0BC
:103CF000F000103016E0087820F00F00401C20F093
:103D0000F00020300EE0087820F00F00401C20F07A
:103D1000F000303006E0087820F00F00401C20F062
:103D2000F0004030087000207047072070472DE9F0
:103D3000F043804687B00D464FF000090846FDF776
:103D4000D7FAA8B94046FDF7F7FC060003D0307853
:103D500022280BD104E043F2020007B0BDE8F08353
:103D600035B1B07FC10601D4000703D50820F4E7C0
:103D70001020F2E7F07F000701D50D20EDE70027C6
:103D8000012140460AF0CEFE040006D101210022A6
:103D900040460AF0BEFE040005D0694600F00FFC64
:103DA000009818B901E00420D7E7FFDF009802214E
:103DB000E0344170C0F82480446107810121017121
:103DC000297801F00102017E62F3010101762A786F
:103DD000520862F3820101762A78920862F3C301E5
:103DE00001762A78D20862F3041101762421304644
:103DF000FDF715FB01A900980CF08DFB022801D0FE
:103E000000B1FFDF4846A8E72DE9FF4F8DB09A4685
:103E100090460E464FF000090D98FDF78DFC050009
:103E200006D02878262806D0082011B0BDE8F08FEB
:103E300043F20200F9E726B94046FFF7F7F80028F9
:103E4000F3D101210D980AF06DFE040000D1FFDFCF
:103E5000852E27D007DCEEB1812E1DD0822E1DD0FD
:103E6000832E08D11CE0862E1ED0882E1ED0892ECF
:103E70001ED08A2E1ED00F2020710F281CD004F0D7
:103E800035F8D8B101208DF81000201D059020795B
:103E9000B0B125E10020EFE70120EDE70220EBE7DC
:103EA0000320E9E70520E7E70620E5E70820E3E748
:103EB0000920E1E70A20DFE70720B6E71120B4E791
:103EC00098F80000D4E91D764208A87F002162F32B
:103ED000C710A87798F800008208E87F62F3000016
:103EE000E87798F80000C209607862F341006070DA
:103EF00098F800000209207862F34710207098F8C3
:103F00000000C208607862F30000607098F8010059
:103F1000607198F8000000F00102B07862F30100CF
:103F2000B070AA7FD20962F38200B070EA7F62F3B8
:103F3000C300B070627862F30410B0702278C0F3EE
:103F4000C000520932706278C2F34002727098F871
:103F50000220F27071713171B978C1F3C00108406B
:103F60005FEA000B2FD05046FDF775F980BBDAF8F9
:103F70000C00FDF770F958BBDAF81C00FDF76BF97F
:103F800030BBDAF80C00A060DAF81C00E060607862
:103F90007A7842EA500100BF61F341006070B9785D
:103FA000C0B200EA111161F30000607000202077B8
:103FB00005F117006061681CA061B07800F0030093
:103FC000012806D044E060787A7802EA5001E3E7FD
:103FD00019E0B87800F00300012839D1321D711DB5
:103FE000404600F09BFA3179387901408DF828106D
:103FF00070797A7910408DF82C00014328D0504612
:10400000FDF729F908B110200FE70AF1100004F5B7
:10401000AE7304F18C028DE80D0000210AAB5A4604
:104020002046FFF746F80028EED101E0C801002045
:1040300004F5B07204F1A403CDF800A0CDE901327B
:1040400001210BAB5A462046FFF733F80028DBD19D
:104050006078800722D4B078B978C0F38000C1F3CB
:10406000800108431AD03178FE4A387832F811209E
:104070004300DA4002F00309B9F1030F01D14FF018
:104080000209BBF1000F09D0012901D0042905D193
:10409000012801D0042801D14FF00409A87F40F085
:1040A0008000A877E87F6BF30000E87760788007EE
:1040B00006D50320A071BBF1000F11D100202CE028
:1040C0000220B9F1020F1AD0B9F1010F19D0B9F1DC
:1040D000040F2AD00020A071A87F20F08000A877CC
:1040E00025212846FDF79BF904A904F1E0000CF016
:1040F000F7F910B1022800D0FFDF002095E6A0718B
:10410000DCE7A0710D22002104F1200007F0AFF9D7
:10411000207840F00200207001208DF80C0003AAE6
:1041200029460D9800F024FADAE70120A071D7E7BC
:104130002DE9F04387B09046894604460025FDF7F7
:10414000FBFA070004D03878272804D0082004E6BA
:1041500043F2020001E6012120460AF0E3FC0400DC
:1041600000D1FFDFA6795FEA090005D0012821D040
:10417000B9F1020F26D110E0B8F1000F22D1012EC3
:1041800005D0022E05D0032E05D0FFDF2EE00C2532
:104190002CE001252AE0022528E04046FDF75BF8E7
:1041A000B0B9032E0ED11022414604F11D0007F0D4
:1041B00034F91BE0012E02D0022E03D104E0B8F145
:1041C000000F13D00720C8E54046FDF744F808B1BA
:1041D0001020C2E51022002104F11D0007F047F96C
:1041E0000621404607F088F9C4F81D0020782521F3
:1041F00040F0020020703846FDF711F92078C10721
:1042000013D020F00100207002208DF8000004F18E
:104210001D0002908DF804506946C3300CF060F91F
:10422000022803D010B1FFDF00E02577002094E5DD
:1042300030B587B00D460446FDF77EFA60B1012126
:1042400020460AF06FFC04000CD02846FDF703F866
:1042500028B1102007B030BD43F20200FAE7207801
:10426000400701D40820F5E7294604F13D0020224B
:10427000054607F0D2F8207840F0100020700107C2
:104280000FD520F00800207007208DF80000694647
:1042900004F1E00001950CF023F9022801D000B1EF
:1042A000FFDF0020D6E770B50D460646FDF744FA5D
:1042B00018B10078272817D102E043F2020070BD40
:1042C000012130460AF02EFC040000D1FFDFA07966
:1042D000022809D16078C00706D02A462146304618
:1042E000FEF778FF10B10FE0082070BDB4F8600051
:1042F0000E280BD204F1620102231022081F0AF0DB
:10430000B6FA012101704570002070BD112070BD0A
:1043100070B5064614460D460846FCF79CFF18B9D2
:104320002046FCF7BEFF08B1102070BDA6F57F4007
:10433000FF380ED03046FDF7FFF938B141782246FC
:104340004B08811C1846FDF7D2F907E043F2020042
:1043500070BD2046FDF7E2FE0028F9D11021E01DD6
:104360000DF033FFE21D294604F1170000F037F984
:10437000002070BD2DE9F04104468AB015460E4676
:1043800000270846FCF7B4FF18B92846FCF7B0FF31
:1043900018B110200AB0BDE8F0812046FDF7CCF935
:1043A0005FEA000804D098F80000272810D102E046
:1043B00043F20200EEE7012120460AF0B3FB0400BD
:1043C00000D1FFDF2078400702D56078800701D454
:1043D0000820DFE7D4E91D01497801B18DB14078AB
:1043E00000B176B1ADB1EA1D06A8E16800F0F7F8BA
:1043F000102206A905F1170006F0E2FF18B1042704
:1044000007E00720C6E71022E91D04F12D0007F0A0
:1044100004F82EB11022F11D04F11D0006F0FDFF7D
:104420002078252140F0020020704046FCF7F7FF7D
:104430002078C10718D020F00100207002208DF8EC
:10444000000004F11D000290103003908DF80470FC
:104450006946B3300CF044F8022806D028B1FFDFDB
:1044600003E00000F42F00002777002092E770B5EA
:104470000D4606460BB1072070BDFDF75DF904003F
:1044800007D02078222802D3A07F800604D40820F9
:1044900070BD43F2020070BDADB12946304609F04F
:1044A000F2FA03F037FB297C4A08A17F62F3C711B7
:1044B000A177297CE27F61F30002E277297C8908F9
:1044C00084F8201004E0304609F000FB03F022FBE2
:1044D000A17F21F02001A17770BD70B50D46FDF7D9
:1044E0002BF9040005D02846FCF7DBFE20B1102094
:1044F00070BD43F2020070BD29462046FEF73BFE28
:10450000002070BD05E000BF10F8012B0AB10020AB
:104510007047491E89B2F7D20120704710B5C478A0
:104520000B7864F300030B70C478640864F34103F0
:104530000B70C478A40864F382030B70C478E40899
:1045400064F3C3030B700379117863F300011170F6
:1045500003795B0863F34101117003799B0863F3EE
:10456000820111700079C00860F3C301117010BDA1
:1045700070B51546064603F0B9FC040000D1FFDF14
:10458000207820F00F00801C20F0F00020302070F8
:1045900066802868A060BDE8704003F0AABC10B532
:1045A000134C94F83000002808D104F12001A1F147
:1045B00010000BF0D7FF012084F8300010BD10B1BF
:1045C00090F8B9202AB10A4890F8350018B10020B7
:1045D00003E0B83001E0064834300860704708B5A1
:1045E0000023009313460A460AF099FC08BD000018
:1045F000C8010020F0B5007B059F1E4614460D46FD
:10460000012800D0FFDF0C2030803A203880002CB9
:1046100008D0287A032806D0287B012800D0FFDFA5
:1046200017206081F0BDA889FBE72DE9F0470D4612
:1046300086B095F80C900E991446B9F1010F0BD085
:104640001022007B2E8A9046052807D0062839D0F4
:10465000FFDF06B0BDE8F0870222F2E7E8890C220E
:1046600000EB400002EB4000188033200880002C53
:10467000EFD0E8896081002720E00096688808F183
:10468000020301AA696900F097FF06EB0800801C8D
:1046900007EB470186B204EB4102BDF804009081AC
:1046A000F848007808B1012300E000230DF106016D
:1046B00040460E320BF0BFFF7F1CBFB26089B8428C
:1046C000DBD8C6E734200880E889B9F1010F11D0A2
:1046D000122148430E301880002CBAD0E88960813E
:1046E0004846B9F1010F00D00220207300270DF1D8
:1046F000040A1FE00621ECE70096688808F102032F
:1047000001AA696900F058FF06EB0800801C86B218
:10471000B9F1010F12D007EBC70004EB4000BDF860
:104720000410C18110220AF10201103006F075FE5A
:104730007F1CBFB26089B842DED88AE707EB470129
:1047400004EB4102BDF80400D0810AF102014046A9
:1047500010320BF092FFEBE72DE9F0470E4688B0E0
:1047600090F80CC096F80C80378AF5890C20DFF899
:104770001493109902F10C04BCF1030F08D0BCF1A2
:10478000040F3DD0BCF1070F75D0FFDF08B061E723
:1047900005EB850C00EB4C00188031200880002AC6
:1047A000F4D0A8F1060000F0FF0A558124E016229B
:1047B000002101A806F05BFE00977088434601AA1D
:1047C000716900F0F9FEBDF804002080BDF8060014
:1047D000E080BDF80800208199F8000008B10123AD
:1047E00000E00023A21C0DF10A0150460BF023FF4C
:1047F00007EB080087B20A346D1EADB2D7D2C5E709
:1048000005EB850C00EB4C00188032200880002A54
:10481000BCD0A8F1050000F0FF0A558137E00097F1
:104820007088434601AA716900F0C6FE9DF8060033
:10483000BDF80410E1802179420860F3000162F3C1
:104840004101820862F38201C20862F3C3010209D6
:1048500062F30411420962F34511820962F3861181
:104860002171C0096071BDF80700208199F800002E
:1048700010B1012301E00EE0002322460DF10901F1
:1048800050460BF0D8FE07EB080087B20A346D1EC5
:10489000ADB2C4D27AE7A8F1020084B205FB08FCED
:1048A0000CF10E00188035200880002AA7D0558111
:1048B000948100971FFA8CF370880E32716900F0B2
:1048C0007BFE63E72DE9F84F1E460A9D0C468146A4
:1048D0002AB1607A00F58070D080E089108199F863
:1048E0000C000C274FF000084FF00E0A0D2872D272
:1048F000DFE800F09D070E1B272F374554697272C1
:104900007200214648460095FFF774FEBDE8F88F17
:10491000207B9146082802D0032800D0FFDF378093
:10492000302009E0A9F80A80F0E7207B91460428AE
:1049300000D0FFDF378031202880B9F1000FF1D19E
:10494000E4E7207B9146042800D0FFDF3780322047
:10495000F2E7207B9146022800D0FFDF378033202A
:10496000EAE7207B1746022800D0FFDF3420A6F8B4
:1049700000A02880002FC9D0A7F80A80C6E7207BB6
:104980001746042800D0FFDF3520A6F800A02880B5
:10499000002FBBD04046A7F80A8012E0207B1746C4
:1049A000052802D0062800D0FFDF102030803620F6
:1049B0002880002FAAD0E0897881A7F80E80B9F866
:1049C0000E00B881A2E7207B9146072800D0FFDFC8
:1049D00037803720B0E72AE04FF0120018804FF000
:1049E00038001700288091D0E0897881A7F80E80E0
:1049F000A7F8108099F80C000A2805D00B2809D0D8
:104A00000C280DD0FFDF81E7207B0A2800D0FFDFD4
:104A100001200AE0207B0B2800D0FFDF042004E007
:104A2000207B0C2800D0FFDF052038736EE7FFDF06
:104A30006CE770B50C460546FCF77EFE20B10078A9
:104A4000222804D2082070BD43F2020070BD052167
:104A500028460AF067F8206008B1002070BD0320E6
:104A600070BD30B44880087820F00F00C01C20F0E2
:104A7000F000903001F8080B1DCA81E81D0030BC21
:104A800003F037BA100000202DE9FF4784B000275B
:104A900082460297079890468946123004F0B3FB8D
:104AA000401D20F00306079828B907A95046FFF7D4
:104AB000C0FF002854D1B9F1000F05D00798017B41
:104AC00019BB052504681BE098F80000092803D0ED
:104AD0000D2812D0FFDF46E0079903254868B0B3E0
:104AE000497B42887143914239D98AB2B3B2011DE0
:104AF00009F0A9FE0446078002E0079C042508345B
:104B00000CB1208810B1032D29D02CE00798012189
:104B1000123004F0AAFBADF80C00024602AB2946A5
:104B2000504606F07DFD070001D1A01C02900798B9
:104B30003A461230C8F80400A8F802A003A940467B
:104B4000029B04F09FFBD8B10A2817D200E006E0D0
:104B5000DFE800F007091414100B0D1414121320D1
:104B600014E6002012E6112010E608200EE643F2BB
:104B700003000BE6072009E60D2007E6032005E603
:104B8000BDF80C002346CDE900702A46504607992F
:104B900000F022FD57B9032D08D10798B3B2417B2D
:104BA000406871438AB2011D09F061FEB9F1000F3E
:104BB000D7D0079981F80C90D3E72DE9FE4F9146A5
:104BC0001A881C468A468046FAB102AB494606F06E
:104BD00027FD050019D04046A61C27880AF0E5F8F5
:104BE0003246072629463B46009609F012FD2088EA
:104BF0002346CDE900504A465146404600F0ECFCC1
:104C0000002020800120BDE8FE8F0020FBE710B5CA
:104C100086B01C46AAB104238DF800301388ADF885
:104C200008305288ADF80A208A788DF80E2009885D
:104C3000ADF80C1000236A462146FFF725FF06B0A9
:104C400010BD1020FBE770B50D46052109F06AFF85
:104C5000040000D1FFDF294604F11200BDE87040D6
:104C600004F0ECBA2DE9F8430D468046002603F027
:104C70003DF904462878102878D2DFE800F0773B29
:104C800034533131123131310831313131312879F8
:104C9000001FC0B2022801D0102810D114BBFFDFC2
:104CA00035E004B9FFDF0521404609F03BFF007BFA
:104CB000032806D004280BD0072828D0FFDF0726BA
:104CC00055E02879801FC0B2022820D050B1F6E705
:104CD0002879401FC0B2022819D0102817D0EEE75B
:104CE00004B9FFDF13E004B9FFDF287901280ED1F2
:104CF000172137E00521404609F014FF070000D1D5
:104D0000FFDF07F11201404604F075FA2CB12A4684
:104D100021464046FFF7A5FE29E013214046FDF756
:104D2000C5FC24E004B9FFDF0521404609F0FAFE86
:104D3000060000D1FFDF694606F1120004F065FAB3
:104D4000060000D0FFDFA988172901D2172200E052
:104D50000A46BDF80000824202D9014602E005E0A1
:104D60001729C5D3404600F047FCD0E7FFDF3046A7
:104D7000BDE8F883401D20F0030219B102FB01F0E9
:104D8000001D00E000201044704713B5009858B192
:104D90000024684609F001FD002C04D1F749009A6F
:104DA0004A6000220A701CBD01240020F2E72DE9B0
:104DB000F0470C46154624220021204606F057FBFA
:104DC00005B9FFDFA87860732888DFF8B0A3401D1D
:104DD00020F00301AF788946DAF8040009F0FBFC03
:104DE000060000D1FFDF4FF000082660A6F8008023
:104DF00077B109FB07F1091D0AD0DAF8040009F0C0
:104E0000EAFC060000D1FFDF6660C6F8008001E022
:104E1000C4F80480298804F11200BDE8F04704F0CA
:104E2000DBB92DE9F047804601F112000D468146BD
:104E300004F0E9F9401DD14F20F003026E7B1446C7
:104E40002968786809F0F2FC3EB104FB06F2121DF5
:104E500003D06968786809F0E9FC052009F00EFEC6
:104E60000446052009F012FE201A012802D17868B4
:104E700009F0A6FC49464046BDE8F04704F0C2B937
:104E800070B50546052109F04DFE040000D1FFDF95
:104E900004F112012846BDE8704004F0ACB92DE9D8
:104EA000F04F91B04FF0000BADF828B0ADF804B062
:104EB00047880C46054692460521384609F032FEE1
:104EC000060000D1FFDF24B1A780A4F806B0A4F843
:104ED00008B0297809220B20B2EB111F73D12A7A6E
:104EE00004F1100138274FF00C084FF0120902911D
:104EF000102A69D2DFE802F068F2F1F08008D38965
:104F00008EA03DDCF3EEB7B7307B022800D0FFDF88
:104F1000A88908EBC001ADF804103021ADF82810C5
:104F2000002C25D06081B5F80E8000271DE004EB31
:104F3000C709317C89F80E10F189A9F80C10CDF859
:104F400000806888042305AA296900F035FBBDF8B4
:104F50001410A9F8101008F10400BDF816107F1CF9
:104F60001FFA80F8A9F81210BFB26089B842DED8E3
:104F70000CE1307B022800D0FFDFE98908EBC1009B
:104F8000ADF804003020ADF8280095F80C90002C06
:104F9000A9F10400C0B20F90EAD06181B5F8108089
:104FA000002725E0CDF8008068884B4603AA696990
:104FB00000F002FB08EB09001FFA80F86F48007848
:104FC00018B1012302E0DDE0DAE0002304EBC702C0
:104FD000009204A90C320F980BF02DFB009ABDF83B
:104FE0000C007F1C1082009ABDF80E00BFB25082E8
:104FF0006089B842D6D8C9E00AA8009001AB224621
:1050000029463046FFF711FBC0E0307B082805D069
:10501000FFDF03E0307B082800D0FFDFE889103095
:10502000ADF804003620ADF82800002C3FD0A98947
:105030006181F189A18127E0307B092800D0FFDF61
:10504000A88901460C30ADF804003720ADF82800DF
:10505000002C2CD06181E8890090AB89688804F12C
:105060000C02296955E0E8893921103080B2ADF889
:105070000400ADF82810002C72D0A9896181287A2B
:105080000E280AD002212173E989E181288A009043
:10509000EB8968886969029A3BE00121F3E70AA875
:1050A000009001AB224629463046FFF755FB6DE0E4
:1050B000307B0A2800D0FFDFADF80490ADF82870EF
:1050C0004CB3A9896181A4F810B0A4F80EB00120F6
:1050D00020735BE020E002E030E038E041E0307B2C
:1050E0000B2800D0FFDF288AADF828701230ADF809
:1050F000040084B104212173A9896181E989E181D6
:10510000298A2182688A00902B8A688804F1120219
:10511000696900F051FA39E0307B0C2800D0FFDFDC
:10512000ADF80490ADF828703CB305212173A4F8C4
:105130000AB0A4F80EB0A4F810B027E00AA80090B6
:1051400001AB224629463046FFF754FA1EE00AA872
:10515000009001AB224629463046FFF7B3FB15E02D
:1051600034E03B21ADF80400ADF8281074B3012001
:10517000E080A4F808B084F80AB007E0100000202E
:10518000FFDF03E0297A012917D0FFDFBDF8040013
:10519000AAF800006CB1BDF828002080BDF804001A
:1051A0006080BDF82800392803D03C2801D086F85B
:1051B0000CB011B00020BDE8F08F3C21ADF8040028
:1051C000ADF8281014B1697AA172DFE7AAF80000DF
:1051D000EFE72DE9F84356880F468046154605212E
:1051E000304609F09FFC040000D1FFDF1234009428
:1051F0003B46414630466A6804F078F9B8E570B538
:105200000D46052109F08EFC040000D1FFDF294680
:1052100004F11200BDE8704004F002B870B50D460C
:10522000052109F07FFC040000D1FFDF294604F1CD
:105230001200BDE8704004F020B870B505460521A5
:1052400009F070FC040000D1FFDF04F108032146DF
:105250002846BDE870400422AFE470B5054605213C
:1052600009F060FC040000D1FFDF214628462368D6
:10527000BDE870400522A0E470B50646052109F09E
:1052800051FC040000D1FFDF04F1120003F0BBFF6A
:10529000401D20F0030511E0011D00880322431882
:1052A00021463046FFF789FC00280BD0607BABB26B
:1052B000684382B26068011D09F00FFB6068418895
:1052C0000029E9D170BD70B50E46054602F00EFE0C
:1052D000040000D1FFDF0120207266726580207813
:1052E00020F00F00C01C20F0F00030302070BDE82E
:1052F000704002F0FEBD602801D00720704708789A
:10530000C54900F001000870002070472DE9F04306
:105310008BB00D461446814606A9FFF78AFB00288C
:1053200014D14FF6FF7601274FF420588CB103209B
:105330008DF800001020ADF8100007A8059007AA0E
:10534000204604A90BF09BF978B107200BB0BDE80B
:10535000F0830820ADF808508DF80E708DF800002D
:10536000ADF80A60ADF80C800CE00698A1780174E5
:105370002188C1818DF80E70ADF80850ADF80C8011
:10538000ADF80A606A4602214846069BFFF77CFB9F
:10539000DCE708B501228DF8022042F60202ADF8E2
:1053A00000200A4603236946FFF731FC08BD08B513
:1053B00001228DF8022042F60302ADF800200A46D1
:1053C00004236946FFF723FC08BD00B587B079B117
:1053D00002228DF800200A88ADF808204988ADF82F
:1053E0000A1000236A460521FFF74EFB07B000BDF7
:1053F0001020FBE709B1072309E40720704770B5C7
:1054000088B00D461446064606A9FFF712FB002891
:105410000ED17CB10620ADF808508DF80000ADF833
:105420000A40069B6A460821DC813046FFF72CFBC8
:1054300008B070BD05208DF80000ADF80850F0E709
:1054400000B587B059B107238DF80030ADF80820BA
:10545000039100236A460921FFF716FBC6E71020D7
:10546000C4E770B588B00C460646002506A9FFF7CC
:10547000E0FA0028DCD106980121123003F0F5FE95
:105480009CB12178062921D2DFE801F0200505161C
:105490000318801E80B2C01EE28880B20AB1A368E1
:1054A0001BB1824203D90C20C2E71020C0E70429B7
:1054B00004D0A08850B901E00620B9E7012913D033
:1054C000022905D004291CD005292AD00720AFE7DE
:1054D00009208DF800006088ADF80800E088ADF87C
:1054E0000A00A068039023E00A208DF8000060887D
:1054F000ADF80800E088ADF80A00A0680A2503901E
:1055000016E00B208DF800006088ADF80800A08838
:10551000ADF80A00E088ADF80C00A0680B250490F7
:1055200006E00C208DF8000060788DF808000C254E
:105530006A4629463046069BFFF7A6FA78E700B58B
:1055400087B00D228DF80020ADF8081000236A46C0
:105550001946FFF799FA49E700B587B071B1022201
:105560008DF800200A88ADF808204988ADF80A10A7
:1055700000236A460621FFF787FA37E7102035E750
:1055800070B586B0064601200D46ADF808108DF8BE
:105590000000014600236A463046FFF775FA040012
:1055A00008D12946304601F0F7FA0021304601F0D3
:1055B00011FB204606B070BDF8B51C4615460E46D8
:1055C000069F09F0E0FB2346FF1DBCB231462A4688
:1055D000009408F0EAFFF8BD30B41146DDE902425C
:1055E0003CB1032903D0002330BC06F0B2B901233B
:1055F000FAE71A8030BC704770B50C460546FFF7D5
:1056000022FB2146284601F0D6FA2846BDE8704024
:10561000012101F0DFBA00001000002018B18178EC
:10562000012938D101E010207047018842F60112AB
:10563000881A914231D018DC42F60102A1EB020037
:1056400091422AD00CDC41B3B1F5C05F25D06FF494
:10565000C050081821D0A0F57060FF381BD11CE0A5
:1056600001281AD002280AD117E0B0F5807F14D0A3
:1056700008DC012811D002280FD003280DD0FF2804
:1056800009D10AE0B0F5817F07D0A0F5807003381A
:1056900003D0012801D0002070470F2070470A284E
:1056A0001FD008DC0A2818D2DFE800F0191B1F1FE2
:1056B000171F231D1F21102815D008DC0B2812D01E
:1056C0000C2810D00D2816D00F2806D10DE0112877
:1056D0000BD084280BD087280FD0032070470020E0
:1056E000704705207047072070470F20704704203F
:1056F0007047062070470C20704743F20200704745
:1057000038B50C46050041D06946FEF7C5FA0028B9
:1057100019D19DF80010607861F30200607069464D
:10572000681CFEF7B9FA00280DD19DF800106078CA
:1057300061F3C5006070A978C1F34101012903D06C
:10574000022905D0072038BD217821F0200102E090
:10575000217841F020012170410704D0A978C908BF
:1057600061F386106070607810F0380F07D0A97868
:10577000090961F3C710607010F0380F02D160782A
:10578000400603D5207840F040002070002038BD4E
:1057900070B504460020088015466068FFF7B0FF2A
:1057A000002816D12089A189884211D860688078A4
:1057B000C0070AD0B1F5007F0AD840F20120B1FB42
:1057C000F0F200FB1210288007E0B1F5FF7F01D94D
:1057D0000C2070BD01F201212980002070BD10B5A0
:1057E0000478137864F3000313700478640864F396
:1057F000410313700478A40864F3820313700478DF
:10580000E40864F3C30313700478240964F30413F5
:1058100013700478640964F34513137000788009E9
:1058200060F38613137031B10878C10701D1800786
:1058300001D5012000E0002060F3C713137010BDF4
:105840004278530702D002F0070306E012F0380F47
:1058500002D0C2F3C20300E001234A7863F30202DC
:105860004A70407810F0380F02D0C0F3C20005E053
:10587000430702D000F0070000E0012060F3C502FA
:105880004A7070472DE9F04F95B00D00824613D055
:1058900012220021284605F0EAFD4FF6FF7B05AAFB
:1058A0000121584605F0ABFB0024264637464FF44D
:1058B00020586FF4205972E0102015B0BDE8F08F29
:1058C0009DF81E0001280AD1BDF81C1041450BD0DF
:1058D00011EB09000AD001280CD002280CD0042CAE
:1058E0000ED0052C0FD10DE0012400E00224BDF8FC
:1058F0001A6008E0032406E00424BDF81A7002E0F0
:10590000052400E00624BDF81A10514547D12C7437
:10591000BEB34FF0000810AA4FF0070ACDE902828B
:10592000CDE900A80DF13C091023CDF810904246B6
:105930003146584605F033FC08BBBDF83C002A460A
:10594000C0B210A90AF099FEC8B9AE81CFB1CDE9B5
:1059500000A80DF1080C0AAE40468CE84102132362
:1059600000223946584605F01AFC40B9BDF83C0003
:10597000F11CC01EC0B22A1D0AF07FFE10B1032028
:105980009BE70AE0BDF82900E881062C05D19DF8C7
:105990001E00A872BDF81C00288100208DE705A814
:1059A00005F039FB00288BD0FFF779FE85E72DE95C
:1059B000F0471C46DDE90978DDF8209015460E0019
:1059C000824600D1FFDF0CB1208818B1D5B111207B
:1059D000BDE8F087022D01D0012100E0002106F191
:1059E000140004F0D5F9A8F8000002463B46294609
:1059F000504605F015FEC9F8000008B9A41C3C602B
:105A00000020E5E71320E3E7F0B41446DDE9045293
:105A10008DB1002314B1022C09D101E0012306E06D
:105A20000D7CEE0703D025F0010501230D742146FE
:105A3000F0BC05F08EBF1A80F0BC70472DE9FE4F18
:105A400091461A881C468A468046FAB102AB4946FE
:105A500005F0E6FD050019D04046A61C278809F090
:105A6000A4F93246072629463B46009608F0D1FDA8
:105A700020882346CDE900504A4651464046FFF76C
:105A8000C3FF002020800120BDE8FE8F0020FBE73F
:105A90002DE9F04786B082460EA8904690E8B00007
:105AA000894604AA05A903A88DE807001E462A46D0
:105AB00021465046FFF77BFF039901B10121397060
:105AC000002818D1FA4904F1140204AB08600398C5
:105AD00005998DE8070042464946504604F00BFD03
:105AE000A8B1092811D2DFE800F005080510100A56
:105AF0000C0C0E00002006B06AE71120FBE707201F
:105B0000F9E70820F7E70D20F5E70320F3E7BDF8F4
:105B100010100398CDE9000133462A46214650462D
:105B2000FFF772FFE6E72DE9F04389B01646DDE99D
:105B300010870D4681461C461422002103A805F05B
:105B400096FC012002218DF810108DF80C008DF8C4
:105B50001170ADF8146064B1A278D20709D08DF845
:105B60001600E088ADF81A00A088ADF81800A0680B
:105B7000079008A80095CDE90110424603A94846C0
:105B80006B68FFF785FF09B0BDE8F083F0B58BB017
:105B900000240646069407940727089405A809944C
:105BA000019400970294CDE903400D46102322464C
:105BB000304605F0F4FA78B90AA806A901940097CE
:105BC0000294CDE90310BDF8143000222946304676
:105BD00005F083F8002801D0FFF761FD0BB0F0BDA0
:105BE00004F014BF2DE9FC410C468046002602F06B
:105BF0007DF9054620780D287ED2DFE800F0BC074D
:105C000013B325BD49496383AF959B00A84800683D
:105C100020B1417841F010014170ADE0404602F002
:105C200095F9A9E00421404608F07CFF070000D167
:105C3000FFDF07F11401404604F03FF8A5BB132134
:105C40004046FCF733FD97E00421404608F06AFF28
:105C5000070000D1FFDFE088ADF800000020B88128
:105C60009DF80000010704D5C00602D5A088B881C0
:105C700005E09DF8010040067ED5A088F88105B9B1
:105C8000FFDF22462946404601F0ACFC022673E0C5
:105C9000E188ADF800109DF8011009060FD507281E
:105CA00003D006280AD00AE024E00421404608F088
:105CB00039FF060000D1FFDFA088F0810226CDB9B0
:105CC000FFDF17E00421404608F02CFF070000D159
:105CD000FFDF07F1140004F0D0FE90F0010F02D1B5
:105CE000E079000648D5387C022640F0020038747E
:105CF00005B9FFDF224600E03DE02946404601F0BD
:105D000071FC39E00421404608F00CFF017C002DB5
:105D100001F00206C1F340016171017C21F0020132
:105D20000174E7D1FFDFE5E702260121404602F0DA
:105D30003FF921E00421404608F0F4FE0546606882
:105D400000902089ADF8040001226946404602F027
:105D500050F9287C20F0020028740DE0002DC9D1F4
:105D6000FFDFC7E7022600214046FFF757FA002D64
:105D7000C0D1FFDFBEE7FFDF3046BDE8FC813EB5A6
:105D80000C0009D001466B4601AA002005F08CFAF0
:105D900020B1FFF784FC3EBD10203EBD00202080D6
:105DA000A0709DF8050002A900F00700FDF790FF24
:105DB00050B99DF8080020709DF8050002A9C0F3B5
:105DC000C200FDF785FF08B103203EBD9DF8080025
:105DD00060709DF80500C109A07861F30410A070FF
:105DE0009DF80510890961F3C300A0709DF80410A7
:105DF000890601D5022100E0012161F342009DF8EE
:105E0000001061F30000A07000203EBD70B5144684
:105E100006460D4651EA040005D075B10846FBF769
:105E20005EFA78B901E0072070BD2946304605F0DA
:105E3000A2FA10B1BDE8704031E454B12046FBF73E
:105E40004EFA08B1102070BD21463046BDE87040C2
:105E500095E7002070BD2DE9FC5F0C469046054695
:105E6000002701780822007A3E46B2EB111F7DD14F
:105E700004F10A0100910A31821E4FF0020A04F176
:105E8000080B0191092A72D2DFE802F0EDE005F576
:105E900028287BAACE006888042108F043FE06006B
:105EA00000D1FFDFB08928B152270726C3E00000E8
:105EB0002C02002051271026002C7DD06888A0805D
:105EC0000120A071A88900220099FFF79FFF0028F8
:105ED00073D1A8892081288AE081D1E0B5F8129099
:105EE000072824D1E87B000621D5512709F11400A9
:105EF00086B2002CE1D0A88900220099FFF786FF26
:105F000000285AD16888A08084F806A0A88920813A
:105F10000120A073288A2082A4F81290A88A0090F9
:105F200068884B46A969019A01F038FBA8E0502720
:105F300009F1120086B2002C3ED0A88900225946F1
:105F4000FFF764FF002838D16888A080A889E08026
:105F5000287A072813D002202073288AE081E87B62
:105F6000C0096073A4F81090A88A01E085E082E07F
:105F7000009068884B4604F11202A969D4E7012019
:105F8000EAE7B5F81290512709F1140086B2002C07
:105F900066D06888042108F0C5FD83466888A08023
:105FA000A88900220099FFF731FF00286ED184F8FC
:105FB00006A0A889208101E052E067E00420A073D8
:105FC000288A2082A4F81290A88A009068884B46FC
:105FD000A969019A01F0E2FAA989ABF80E104FE025
:105FE0006888FBF7A9FB07466888042108F09AFD3A
:105FF000064607B9FFDF06B9FFDF687BC00702D09E
:106000005127142601E0502712264CB36888A0803F
:10601000502F06D084F806A0287B594601F0CEFA0E
:106020002EE0287BA11DF9E7FE49A8894989814214
:1060300005D1542706269CB16888A08020E053270C
:106040000BE06888A080A889E08019E068880421B6
:1060500008F068FD00B9FFDF55270826002CF0D1B5
:10606000A8F8006011E056270726002CF8D06888B1
:10607000A080002013E0FFDF02E0012808D0FFDF4E
:10608000A8F800600CB1278066800020BDE8FC9F66
:1060900057270726002CE3D06888A080687AA07173
:1060A000EEE7401D20F0030009B14143091D01EB5B
:1060B0004000704713B5DB4A00201071009848B1CA
:1060C0000024684608F069FB002C02D1D64A0099EA
:1060D00011601CBD01240020F4E770B50D46144684
:1060E000064686B05C220021284605F0C0F904B9B6
:1060F000FFDFA0786874A2782188284601F089FA29
:106100000020A881E881228805F11401304603F0BF
:10611000B8FD6A460121304604F071FF1AE000BF65
:106120009DF80300000715D5BDF806103046FFF7AF
:106130002DFD9DF80300BDF8061040F010008DF80D
:106140000300BDF80300ADF81400FF233046059AA4
:1061500005F0D9F8684604F05EFF0028E0D006B0EC
:1061600070BD10B50C4601F1140003F0C2FD0146EC
:10617000627C2046BDE8104001F080BA30B504468C
:10618000A84891B04FF6FF75C18905AA284604F0CA
:1061900036FF30E09DF81E00A0422AD001282AD107
:1061A000BDF81C00B0F5205F03D042F60101884223
:1061B00021D1002002AB0AAA0CA9019083E80700B4
:1061C00007200090BDF81A1010230022284604F082
:1061D000E6FF38B9BDF828000BAAC0B20CA90AF036
:1061E0004CFA10B1032011B030BD9DF82E00A04232
:1061F00001D10020F7E705A804F00DFF0028C9D061
:106200000520F0E770B50546042108F08BFC04007A
:1062100000D1FFDF04F114010C46284603F04DFDC8
:1062200021462846BDE8704003F04EBD70B58AB0E7
:106230000C460646FBF780FA050014D02878222881
:1062400027D30CB1A08890B101208DF80C00032059
:106250008DF8100000208DF8110054B1A088ADF821
:106260001800206807E043F202000AB070BD092060
:10627000FBE7ADF8180005900421304608F052FC09
:10628000040000D1FFDF04F1140003F048FD000713
:1062900001D40820E9E701F029FE60B108A8022135
:1062A0000094CDE9011095F8232003A930466368D6
:1062B000FFF7EEFBD9E71120D7E72DE9F04FB2F851
:1062C00002A0834689B0154689465046FBF734FA4A
:1062D00007460421504608F025FC00260446059692
:1062E0004FF002080696ADF81C6007B9FFDF04B94D
:1062F000FFDF4146504605F05AFC50B907AA06A9EF
:1063000005A88DE807004246214650466368FFF71E
:106310004EFB444807AB0660DDE9051204F11400AA
:10632000CDF80090CDE90320CDE9013197F8232085
:10633000594650466B6803F03BFD06000AD0022E1A
:1063400004D0032E14D0042E00D0FFDF09B0304655
:10635000BDE8F08FBDF81C000028F7D00599CDE905
:1063600000104246214650466368FFF74DFBEDE7BB
:10637000687840F008006870E8E710B50C46FFF751
:10638000BFF900280BD1607800F00701012905D181
:1063900010F0380F02D02078810601D5072010BDFB
:1063A00040F0C8002070002010BD2DE9F04F99B0DA
:1063B00004464FF000081B48ADF81C80ADF8208063
:1063C000ADF82480A0F80880ADF81480ADF81880EE
:1063D000ADF82880ADF82C80007916460D4647466A
:1063E000012808D0022806D0032804D0042802D0AF
:1063F000082019B0ACE72046FAF72DFFF0BB28467D
:10640000FAF729FFD0BB6068FAF772FFB0BB60688B
:1064100068B160892189884202D8B1F5007F05D929
:106420000C20E6E72C0200201800002080460EAA6F
:1064300006A92846FFF7ACF90028DAD16868807809
:10644000C0F34100022808D19DF8190010F0380F60
:1064500003D02869FAF743FF80B905A92069FFF73F
:106460004FF90028C5D1206950B1607880079DF8A8
:10647000150000F0380002D5F0B301E011E0D8BB00
:106480009DF8140080060ED59DF8150010F0380F09
:1064900003D06068FAF723FF18B96068FAF728FF9D
:1064A00008B11020A5E70BA906A8FFF7C9F99DF8C8
:1064B0002D000BA920F00700401C8DF82D0060690D
:1064C000FFF75BFF002894D10AA9A069FFF718F92C
:1064D00000288ED19DF8280080062BD4A06940B1F9
:1064E0009DF8290000F00701012923D110F0380F91
:1064F00020D0E06828B100E01CE00078D0B11C2872
:1065000018D20FAA611C2046FFF769F9012138460D
:1065100061F30F2082468DF85210B94642F603000F
:106520000F46ADF850000DF13F0218A928680AF097
:10653000A6F808B107205CE79DF8600015A9CDF822
:106540000090C01CCDE9019100F0FF0B00230BF27D
:106550000122514614A804F07DFCE8BBBDF85400AC
:106560000C90FB482A8929690092CDE901106B89BA
:10657000BDF838202868069904F06CFC010077D13A
:1065800020784FF0020AC10601D4800616D58DF896
:10659000527042F60210ADF85000CDF80C9008A9E8
:1065A00003AACDF800A0CDE90121002340F2032287
:1065B00014A80B9904F04EFC010059D1E4484D4653
:1065C00008380089ADF83D000FA8CDE90290CDF85C
:1065D0000490CDF8109000E00CE04FF007095B4606
:1065E0000022CDF80090BDF854104FF6FF7004F073
:1065F00074FB10B1FFF753F8FBE69DF83C00000672
:1066000024D52946012060F30F218DF852704FF4F4
:1066100024500395ADF8500062789DF80C000023DB
:1066200062F300008DF80C006278CDF800A05208EB
:1066300062F341008DF80C0003AACDE9012540F278
:10664000032214A804F006FC010011D1606880B395
:106650002069A0B905A906A8FFF7F2F860788007BD
:1066600007D49DF8150020F038008DF8150006E0DD
:1066700077E09DF8140040F040008DF814008DF88C
:10668000527042F60110ADF85000208940F201210D
:10669000B0FBF1F201FB1202606809ABCDF800809B
:1066A000CDE90103002314A8059904F0D3FB0100F0
:1066B00057D12078C00728D00395A06950B90AA9FE
:1066C00006A8FFF7BDF89DF8290020F00700401C40
:1066D0008DF829009DF8280007A940F040008DF8AA
:1066E00028008DF8527042F60310ADF8500003AA4E
:1066F000CDF800A0CDE90121002340F2032214A827
:106700000A9904F0A7FB01002BD1E06868B3294681
:10671000012060F30F218DF8527042F60410ADF89D
:106720005000E068002302788DF8582040788DF8FA
:106730005900E06816AA4088ADF85A00E068007970
:106740008DF85C00E068C088ADF85D00CDF8009081
:10675000CDE901254FF4027214A804F07BFB01007F
:1067600003D00C9800F0B6FF43E6794803210838BF
:10677000017156B100893080BDF824007080BDF8E9
:106780002000B080BDF81C00F080002031E670B51C
:1067900001258AB016460B46012802D0022816D1E0
:1067A00004E08DF80E504FF4205003E08DF80E50A9
:1067B00042F60100ADF80C005BB10024601C60F3F0
:1067C0000F2404AA08A9184609F059FF18B1072098
:1067D0004BE5102049E504A99DF820205C48CDE94F
:1067E0000021801E02900023214603A802F201220C
:1067F00004F030FB10B1FEF752FF36E5544808387C
:106800000EB1C1883180057100202EE5F0B593B03E
:10681000044601268DF83E6041F601000F46ADF8B2
:106820003C0011AA0FA93046FFF7B1FF002837D16D
:106830002000474C4FF00005A4F1080432D01C2280
:10684000002102A804F013FE9DF808008DF83E60B8
:1068500040F020008DF8080042F60520ADF83C001D
:1068600004200797ADF82C00ADF8300039480A90A5
:106870000EA80D900E950FA80990ADF82E506A46FF
:1068800009A902A8FFF791FD002809D1BDF8000071
:106890006081BDF80400A081401CE08125710020CA
:1068A00013B0F0BD6581A581BDF84400F4E72DE982
:1068B000F74F2749A0B00024083917940A79A14658
:1068C000012A04D0022A02D0082023B040E5CA8859
:1068D000824201D00620F8E721988A46824201D1FF
:1068E0000720F2E70120214660F30F21ADF84800B0
:1068F0004FF6FF788DF86E000691ADF84A8042F6AB
:10690000020B8DF872401CA9ADF86CB0ADF8704068
:106910001391ADF8508012A804F0ACFB00252E4670
:106920002F460DAB072212A9404604F0A6FB98B1F2
:106930000A2861D1B5B3AEB3ADF86450ADF8666066
:106940009DF85E008DF8144019AC012868D06FE006
:1069500034020020308C01009DF83A001FB301285A
:1069600059D1BDF8381059451FD118A809A901946B
:106970000294CDE9031007200090BDF836101023D3
:106980000022404604F00BFCB0BBBDF860000428B8
:1069900001D006284AD1BDF82410219881423AD16D
:1069A0000F2092E73AE0012835D1BDF83800B0F564
:1069B000205F03D042F6010188422CD1BAF80600CC
:1069C000BDF83610884201D1012700E0002705B14B
:1069D0009EB1219881421ED118A809AA019402945F
:1069E000CDE90320072000900D46102300224046E9
:1069F00004F0D5FB00B902E02DE04E460BE0BDF8F7
:106A00006000022801D0102810D1C0B217AA09A92D
:106A100009F033FE50B9BDF8369082E7052054E7FF
:106A200005A917A8221D09F02AFE08B103204CE78A
:106A30009DF814000023001DC2B28DF81420229886
:106A40000092CDE901401BA8069904F003FA10B9A1
:106A500002228AF80420FEF722FE36E710B50B4624
:106A6000401E88B084B205AA00211846FEF7B7FE82
:106A700000200DF1080C06AA05A901908CE807007A
:106A8000072000900123002221464FF6FF7004F0FA
:106A900024F90446BDF81800012800D0FFDF204685
:106AA000FEF7FDFD08B010BDF0B5FF4F044687B0FE
:106AB00038790E46032804D0042802D0082007B0F5
:106AC000F0BD04AA03A92046FEF762FE0500F6D138
:106AD00060688078C0F3410002280AD19DF80D005B
:106AE00010F0380F05D02069FAF7F9FB08B1102033
:106AF000E5E7208905AA21698DE807006389BDF8CB
:106B000010202068039904F0A5F910B1FEF7C7FD25
:106B1000D5E716B1BDF8140030800420387128463E
:106B2000CDE7F8B50C0006460BD001464FF6FF75D1
:106B300000236A46284604F0B7FB20B1FEF7AFFDFC
:106B4000F8BD1020F8BD69462046FEF7D9FD0028A3
:106B5000F8D1A078314600F001032846009A04F0ED
:106B6000D2FBEBE730B587B0144600220DF1080CDC
:106B700005AD01928CE82C00072200920A460146DE
:106B800023884FF6FF7004F0A8F8BDF81410218098
:106B9000FEF785FD07B030BD70B50D46042107F046
:106BA000C1FF040000D1FFDF294604F11400BDE855
:106BB000704003F0ADB870B50D46042107F0B2FF88
:106BC000040000D1FFDF294604F11400BDE8704045
:106BD00003F0C1B870B50D46042107F0A3FF04000F
:106BE00000D1FFDF294604F11400BDE8704003F036
:106BF000D9B870B50546042107F094FF040000D110
:106C0000FFDF214628462368BDE870400122FEF7D9
:106C100015BF70B50646042107F084FF040000D1BB
:106C2000FFDF04F1140003F064F8401D20F00305B9
:106C300011E0011D00880022431821463046FEF76E
:106C4000FDFE00280BD0607CABB2684382B2A06826
:106C5000011D07F042FEA06841880029E9D170BDFE
:106C600070B50546042107F05DFF040000D1FFDF89
:106C7000214628466368BDE870400222FEF7DEBE6A
:106C800070B50E46054601F031F9040000D1FFDF72
:106C90000120207266726580207820F00F00001DB0
:106CA00020F0F00040302070BDE8704001F021B9C4
:106CB00010B50446012900D0FFDF2046BDE8104092
:106CC0000121FEF7ABBA2DE9F04F97B04FF0000A63
:106CD0000C008346ADF814A0D04619D0E06830B15E
:106CE000A068A8B10188ADF81410A0F800A058461B
:106CF000FAF722FD070043F2020961D03878222812
:106D00005CD30421584607F00DFF050005D103E0D0
:106D1000102017B0BDE8F08FFFDF05F1140002F07E
:106D2000E8FF401D20F00306A078012803D00228C8
:106D300001D00720EDE7218807AA584604F05FF943
:106D400030BB07A804F067F910BB07A804F063F98B
:106D500048B99DF82600012805D1BDF82400A0F50A
:106D60002451023902D04FF45050D2E7E068B0B15C
:106D7000CDE902A00720009005AACDF804A0049256
:106D8000A2882188BDF81430584603F0A6FF10B140
:106D9000FEF785FCBDE7A168BDF8140008809DF8EA
:106DA0001F00C00602D543F20140B2E70B9838B18C
:106DB000A1780078012905D080071AD40820A8E717
:106DC0004846A6E7C007F9D002208DF83C00A86825
:106DD0004FF00009A0B1697C4288714391420FD9FC
:106DE0008AB2B3B2011D07F02EFD8046A0F800A0C4
:106DF00006E003208DF83C00D5F800804FF0010933
:106E00009DF8200010F0380F00D1FFDF9DF8200022
:106E10002649C0F3C200084497F8231010F8010C6B
:106E2000884201D90F2074E72088ADF8400014A9EA
:106E30000095CDE90191434607220FA95846FEF778
:106E400027FE002891D19DF8500050B9A078012864
:106E500007D1687CB3B2704382B2A868011D07F005
:106E600006FD002055E770B5064615460C46084657
:106E7000FEF7D4FB002805D12A4621463046BDE85E
:106E8000704084E470BD12E570B51E4614460D00D6
:106E90000ED06CB1616859B160B10349C9888142B3
:106EA00008D0072070BD00002C020020338C0100A8
:106EB0001020F7E72068FEF7B1FB0028F2D1324638
:106EC00021462846BDE87040FFF76FBA70B51546F9
:106ED0000C0006D038B1FE490989814203D0072051
:106EE000E0E71020DEE72068FEF798FB0028D9D104
:106EF00029462046BDE87040D6E570B5064686B006
:106F00000D4614461046FAF7CCF9D0BB6068FAF784
:106F1000EFF9B0BBA6F57F40FF3803D03046FAF753
:106F20000BFC80B128466946FEF7ACFC00280CD16A
:106F30009DF810100F2008293DD2DFE801F0080667
:106F40000606060A0A0843F2020006B0AAE7032072
:106F5000FBE79DF80210012908D1BDF80010B1F53A
:106F6000C05FF2D06FF4C052D142EED09DF806104F
:106F700001290DD1BDF80410A1F52851062907D229
:106F800000E029E0DFE801F0030304030303DCE78A
:106F90009DF80A1001290FD1BDF80810B1F5245F42
:106FA000D3D0A1F60211B1F50051CED00129CCD039
:106FB000022901D1C9E7FFDF606878B9002305AA7B
:106FC0002946304604F070F910B1FEF768FBBCE7C3
:106FD0009DF81400800601D41020B6E7618822468F
:106FE00028466368FFF7BEFDAFE72DE9F043814611
:106FF00087B0884614461046FAF753F918B11020A6
:1070000007B0BDE8F083002306AA4146484604F0D5
:107010004BF910B1FEF743FBF2E79DF81800C006EC
:1070200002D543F20140EBE70025072705A80195AB
:1070300000970295CDE9035062884FF6FF734146F1
:10704000484604F0ACF8060013D16068FAF729F955
:1070500060B960680195CDE90250009704952388D6
:1070600062884146484604F09AF80646BDF8140086
:1070700020803046CEE739B1954B0A889B899A42E9
:1070800002D843F2030070471DE610B586B0904C5D
:107090000423ADF81430638943B1A4898C4201D232
:1070A000914205D943F2030006B010BD0620FBE76C
:1070B000ADF81010002100910191ADF800300221CF
:1070C0008DF8021005A9029104A90391ADF81220D0
:1070D0006946FFF7F8FDE7E72DE9FC4781460D46D5
:1070E0000846FAF7B8F888BB4846FAF725FB5FEA86
:1070F00000080AD098F80000222829D30421484625
:1071000007F010FD070005D103E043F20200BDE8DF
:10711000FC87FFDF07F1140002F001FE0646287825
:10712000012803D0022804D00720F0E7B0070FD5CC
:1071300002E016F01C0F0BD0A8792C1DC00709D057
:10714000E08838B1A068FAF786F818B11020DEE7B9
:107150000820DCE721882A780720B1F5847F35D024
:107160001EDC40F20315A1F20313A94226D00EDC67
:10717000B1F5807FCBD003DCF9B1012926D1C6E778
:10718000A1F58073013BC2D0012B1FD113E0012B6D
:10719000BDD0022B1AD0032BB9D0042B16D112E08C
:1071A000A1F20912082A11D2DFE802F00B04041040
:1071B00010101004ABE7022AA9D007E0012AA6D0DC
:1071C00004E0320700E0F206002AA0DACDB200F0B7
:1071D0008DFE50B198F82300CDE90005FA892346C9
:1071E00039464846FEF79FFC91E711208FE72DE9CD
:1071F000F04F8BB01F4615460C4683460026FAF723
:107200009BFA28B10078222805D208200BB081E52E
:1072100043F20200FAE7B80801D00720F6E7032F8F
:1072200000D100274FF6FF79CCB1022D71D3204653
:10723000FAF75EF830B904EB0508A8F10100FAF797
:1072400057F808B11020E1E7AD1E38F8028CAAB259
:107250002146484604F07BF940455AD1ADB21C495D
:10726000B80702D58889401C00E001201FFA80F889
:10727000F80701D08F8900E04F4605AA41465846DD
:1072800003F0BDFE4FF0070A4FF00009FCB12046A5
:1072900008E0408810283CD8361D304486B2AE4203
:1072A00037D2A01902884245F3D352E09DF8170067
:1072B00002074ED57CB304EB0608361DB8F8023041
:1072C000B6B2102B25D89A19AA4222D802E040E083
:1072D0002C020020B8F8002091421AD1C0061BD51C
:1072E000CDE900A90DF1080C0AAAA11948468CE8BD
:1072F0000700B8F800100022584603F0EEFC10B169
:10730000FEF7CDF982E7B8F80200BDF828108842F0
:1073100002D00B207AE704E0B8F80200304486B2CD
:1073200006E0C00604D55846FEF730FC00288AD196
:107330009DF81700BDF81A1020F010008DF8170006
:10734000BDF81700ADF80000FF235846009A03F07F
:10735000DAFF05A803F05FFE18B9BDF81A10B942AC
:10736000A4D90421584607F0DDFB040000D1FFDF5B
:10737000A2895AB1CDE900A94D46002321465846BD
:10738000FEF7D1FB0028BDD1A5813FE700203DE7F6
:107390002DE9FF4F8BB01E4617000D464FF000043D
:1073A00012D0B00802D007200FB0B3E4032E00D1F2
:1073B00000265DB10846F9F792FF28B93888691EA2
:1073C0000844F9F78CFF08B11020EDE7C74AB00771
:1073D00001D5D18900E00121F0074FF6FF7802D0F6
:1073E000D089401E00E0404686B206AA0B9803F002
:1073F00006FE4FF000094FF0070B0DF1140A38E0BC
:107400009DF81B00000734D5CDF80490CDF800B0EE
:10741000CDF80890CDE9039A434600220B9803F07B
:10742000BEFE60BB05B3BDF814103A88214428198C
:10743000091D8A4230D3BDF81E2020F8022BBDF86A
:10744000142020F8022BCDE900B9CDE90290CDF847
:1074500010A0BDF81E10BDF8143000220B9803F0E8
:107460009EFE08B103209FE7BDF814002044001DD4
:1074700084B206A803F0CFFD20B10A2806D0FEF79B
:107480000EF991E7BDF81E10B142B9D934B17DB102
:107490003888A11C884203D20C2085E7052083E7A9
:1074A00022462946404604F052F801462819018038
:1074B000A41C3C80002077E710B50446F9F7F1FEE4
:1074C00008B1102010BD8948C0892080002010BD5F
:1074D000F0B58BB00D4606461422002103A803F038
:1074E000C6FF01208DF80C008DF8100000208DF8EB
:1074F0001100ADF814503046FAF71EF948B1007883
:10750000222812D30421304607F00CFB040005D1D9
:1075100003E043F202000BB0F0BDFFDF04F1140002
:10752000074602F0FCFB800601D40820F3E7207C2C
:10753000022140F00100207409A80094CDE9011057
:10754000072203A930466368FEF7A2FA20B1217C26
:1075500021F001012174DEE729463046FDF74FFE98
:1075600008A9384602F0CAFB00B1FFDFBDF8204091
:10757000172C01D2172000E02046A84201D92C4642
:1075800002E0172C00D2172421463046FFF713FBE8
:1075900021463046FDF757FB0020BCE7F8B51C46F6
:1075A00015460E46069F07F0EEFB2346FF1DBCB2B4
:1075B00031462A46009406F0F8FFF8BD70B50C4637
:1075C00005460E220021204603F051FF00202080B6
:1075D0002DB1012D01D0FFDF64E4062000E005207D
:1075E000A0715FE410B548800878134620F00F00C2
:1075F000001D20F0F00080300C460870142219465F
:1076000004F1080003F009FF00F073FC3748046040
:1076100010BD2DE9F047DFF8D890491D064621F04E
:10762000030117460C46D9F8000007F0D4F805000E
:1076300000D1FFDF4FF000083560A5F8008021463B
:10764000D9F8000007F0C7F8050000D1FFDF75602A
:10765000A5F800807FB104FB07F1091D0BD0D9F814
:10766000000007F0B8F8040000D1FFDFB460C4F8F0
:107670000080BDE8F087C6F80880FAE72DE9F04100
:107680001746491D21F00302194D064601681446AC
:10769000286807F0CBF822467168286807F0C6F81A
:1076A0003FB104FB07F2121D03D0B168286807F050
:1076B000BDF8042007F0E2F90446042007F0E6F9DB
:1076C000201A012804D12868BDE8F04107F078B8F5
:1076D000BDE8F08110B50C4603F060FC00B1FFDF9F
:1076E0002046BDE81040FDF7DABF00002C02002064
:1076F0001800002038B582880A800C46C188121D07
:1077000090B26A4606F0D4FABDF80000032800D310
:107710000320C1B2208800F093FF38BD38B58288BD
:107720000A800C46C188121D90B26A4606F0C0FA63
:10773000BDF80000022800D30220C1B2208800F06A
:107740007FFF401CC0B238BD2DE9FF5F8B46FD496D
:1077500082461446D1E90101CDE902010BF1030291
:1077600022F0030201A84421019207F016F8F64E18
:10777000002C02D1F549019A8A60019901440191D6
:10778000B57E05F1010504D1E8B208F0F9FE00B1BB
:10779000FFDF019800EB0510C01C20F003010191F0
:1077A00044B9727A00200870308C80B203F055FA28
:1077B00000B1FFDF0198316A08440190214601A819
:1077C00000F002FF80460198C01C20F003000190E9
:1077D000717A04B1002007F0CAF8019908440190B9
:1077E000214601A800F037FFD74800273D4690F812
:1077F00001900CE0284600F0CAFE06468178808899
:10780000FDF7B8FA71786D1C00FB0177EDB24D45BC
:10781000F0D10198C01C20F00300019004B10020B9
:107820003946FDF7B2FA0199002708440190C6488D
:107830003D4690F801900CE0284600F0A8FE064670
:10784000C1788088FEF72DFC71786D1C00FB0177F4
:10785000EDB24D45F0D10198C01C20F0030001901D
:1078600004B100203946FEF725FC01990844019037
:10787000B64800214278084604F013F8214601A8D2
:1078800000F064FE0198C01D20F007000190DAF8B6
:107890000010814204D3A0EB0B01B1F5803F04DB63
:1078A0004FF00408CAF8000004E0CAF80000B8F17C
:1078B000000F03D0404604B0BDE8F09F5CBBFAF770
:1078C000CCFBA14C207E0090607E012825D00023B7
:1078D00028B300229C4800210C30FAF7E5FF00B1E4
:1078E000FFDF9949E07E1C31FEF790FF00B1FFDF1A
:1078F00095484FF4F6720021383003F0B8FD9248F5
:107900000421383080F8E91180F8EA11062180F866
:10791000EB11032101710020CDE70123D8E702AA72
:10792000D8E770B5884C06463834207804EB40150B
:10793000E078083598B9A01990F8E80100280FD030
:10794000A0780F2800D3FFDF20220021284603F073
:107950008EFD687866F3020068700120E0702846AA
:1079600070BD2DE9F04105460C4600270078052141
:1079700090463E46B1EB101F00D0FFDF287A58B189
:1079800001280FD0FFDF00BFA8F800600CB12780EE
:1079900066800020BDE8F0810127092674B168885F
:1079A000A08008E00227142644B16888A0802869D6
:1079B000E060A88A2082287B2072E5E7A8F80060B2
:1079C000E7E730B5604C0120002120706170207223
:1079D00060726176217621730521A1821F21E182E7
:1079E00060735BA121610A21A176E0765548574D6D
:1079F000B0F80110A183C078A0774FF4B060206286
:107A00006868C11C21F00301814200D0FFDF686873
:107A1000606030BD30B54D4C1568636808339D42D9
:107A200002D20420136030BD474B5D785A6802EBE8
:107A3000C502107051700320D08017209080012063
:107A4000D07090705878401C587060680830606042
:107A5000002030BD70B506463B480024457807E05D
:107A6000204600F094FD0178B14204D0641CE4B2D9
:107A7000AC42F5D1002070BDF7B5064608780C463B
:107A8000F8B1FFF7E7FF0546202E06D0212E1AD0C9
:107A9000222E18D0232E14D110E000F083FD0DB15A
:107AA000697800E00021401A81B2A0780144FF29E2
:107AB00007D830B1A088022805D202E060881728D4
:107AC00001D20720FEBD65B9207802AA0121FFF787
:107AD000A1FF0028F6D12078FFF7BCFF050000D1F8
:107AE000FFDF202E08D0212E0ED0222E0FD0232EE5
:107AF00007D0FFDF0020FEBDA0786870A088E88076
:107B0000F8E76088A880F5E7A078A870F2E7A07889
:107B1000E870EFE71A283FD00DDC13283CD2DFE8ED
:107B200000F0253B2A3B3B31312D2F373B3B333B8C
:107B30003B3B3B390F00302802D00DDC1E282BD1F7
:107B400007207047388C0100680200201C000020CC
:107B50006E524635780000003A3809281CD2DFE81A
:107B600000F0151B0F1B1B1B1B1B07000020E8E769
:107B700043F20400E5E743F20200E2E70420E0E715
:107B80000D20DEE70F20DCE70820DAE71120D8E738
:107B90001320D6E70620D4E70320D2E710B50078FB
:107BA00000F0010006F07AF8BDE81040B2E710B529
:107BB000007800F0010006F076F8BDE81040A9E773
:107BC0000EB5017801F001018DF80010417801F047
:107BD00001018DF801100178C1F340018DF8021008
:107BE0004178C1F340018DF80310017889088DF8C0
:107BF0000410417889088DF8051081788DF80610F9
:107C0000C1788DF8071000798DF80800684605F0F6
:107C100033FDFFF77FFF0EBD2DE9FC5FDFF8F88332
:107C2000FE4C00261FE0012000F058FD0120FFF768
:107C300078FE054644214746D8F8080006F0CBFDFB
:107C4000686000B9FFDF686805F010FCA8B128463D
:107C5000F9F7C5FE284600F047FD20B944226968BF
:107C6000B86806F0E3FD94F9E9010428DBDA0220A4
:107C700006F004FF07460025ABE044226968D8F807
:107C8000080006F0D3FDF2E7B8F802104046491CA0
:107C900089B2A8F80210B94201D300214180022123
:107CA000B8F8020006F03EFF002867D0B8F80200DE
:107CB000694605F063FFFFF72DFF00B1FFDF9DF878
:107CC0000000019078B1B8F8020007F06EF85FEAA2
:107CD000000900D1FFDF484606F0FBFA18B1B8F8FA
:107CE000020003F052FFB8F8020007F04CF85FEA18
:107CF000000900D1FFDF484606F0E3FAF0BB03219C
:107D0000B8F8020006F00EFF5FEA000B4CD1FFDF6F
:107D10004AE000BFDBF80C0010B10078FF284DD01E
:107D2000022000F0DBFC0220FFF7FBFD8246484604
:107D300006F0D3FBCAF8040000B9FFDFDAF804004C
:107D400006F09BFC002100900170B8F8021050462C
:107D5000AAF8021003F044FE484606F090FC00B971
:107D6000FFDF019800B10126504600F0BDFC18B9B4
:107D70009AF80100000705D5009800E027E0CBF84D
:107D80000C0011E0DBF80C0038B10178491C11F04F
:107D9000FF01017008D1FFDF06E0002211464846CE
:107DA00000F0D2FB00B9FFDF94F9EA01022805DBFD
:107DB000B8F8020003F0EFFD0028ABD194F9E90117
:107DC000042804DB484606F0BEFC00B101266D1C09
:107DD000EDB2BD4204D294F9EA010228BFF654AFD5
:107DE000002E7FF41EAFBDE8FC5F032000F076BCE0
:107DF00010B5894CE06008682061AFF2E310FBF732
:107E000074F8607010BD85480021383801708248D0
:107E100001708349416094E670B505464FF080508B
:107E20000C46D0F8A410491C05D1D0F8A810C943BD
:107E30000904090C0BD050F8A01F01F001012970B2
:107E4000416821608068A080287830B970BD062123
:107E500020460AF0BAF901202870607940F0C0008D
:107E6000607170BD70B54FF080540D46D4F880102D
:107E7000491C0BD1D4F88410491C07D1D4F88810C0
:107E8000491C03D1D4F88C10491C0CD0D4F88010B4
:107E90000160D4F884104160D4F888108160D4F86F
:107EA0008C10C16002E010210AF08FF9D4F8900024
:107EB000401C0BD1D4F89400401C07D1D4F8980092
:107EC000401C03D1D4F89C00401C09D054F8900FFA
:107ED000286060686860A068A860E068E86070BDBD
:107EE0002846BDE8704010210AF06FB94B48007970
:107EF00017E570B5494CE07830B3207804EB4010BA
:107F0000407A00F00700204490F9E801002800DCE6
:107F1000FFDF2078002504EB4010407A00F00700D6
:107F2000011991F8E801401E81F8E8012078401C11
:107F3000C0B220700F2800D12570A078401CA0701E
:107F400009F0C2FFE57070BDFFDF70BD3EB50546AC
:107F5000032106F0E7FD0446284606F014FF054617
:107F600004B9FFDFE06818B10078FF2800D1FFDF17
:107F700001AA6946284600F0E7FA60B9FFDF0AE087
:107F8000002202A9284600F0DFFA00B9FFDF9DF8C1
:107F9000080000B1FFDF9DF80000411E8DF80010C1
:107FA000EED2E0680199884201D10020E0603EBD38
:107FB00070B50546A0F57F400C46FF3800D1FFDFC5
:107FC000012C01D0FFDF70BDFFF790FF040000D14E
:107FD000FFDF207820F00F00401D20F0F00050302F
:107FE000207065800020207201202073BDE8704061
:107FF0007FE72DE9F04116460D460746FFF776FF6D
:10800000040000D1FFDF207820F00F00401D20F099
:10801000F0005030207005E01C000020A00200207D
:10802000680D002067800120207228682061A888E0
:10803000A0822673BDE8F0415BE77FB5FFF70AFD3C
:10804000040000D1FFDF02A92046FFF753FB0546DD
:1080500003A92046FFF762FB8DF800508DF8010060
:10806000BDF80800001DADF80200BDF80C00001DB1
:10807000ADF80400E088ADF80600684605F0F2FDB2
:10808000002800D0FFDF7FBD2DE9F05FF74F80466D
:10809000387808B108200FE44046F9F702F908B132
:1080A000102009E4F24D287808B9FFF78AFC6C7AB1
:1080B000464600F077FAA04207D2201AC1B23246F3
:1080C0000020FFF7A7FC0028E5D17968BB46C91C52
:1080D00021F0030179600027E5483E46B946BA46DB
:1080E0003C46457807E0204600F051FA4078641C91
:1080F0000644E4B27F1CAC42F5D10AEB870000EBEA
:10810000C600DB4E00EB89005C46717A012200EB71
:10811000C100DBF80410451829464046FFF714FB60
:10812000070012D00020FFF795FC05000BD005F1E9
:108130000B00616820F00300884200D0FFDF7078F8
:10814000401E707065603846A5E70022294640460B
:10815000FFF7FAFA00B1FFDFD8F8000060604FF6D1
:10816000FF70608001202070002094E72DE9F0412D
:108170000446BE4817460D46007808B1082009E4B9
:108180000846F9F768F808B1102003E4B84E3078D3
:1081900008B9FFF716FC601E1E2807D8012C23D152
:1081A0002878FE2820D8B0760020E8E7A4F1200047
:1081B0001F2805D8E0B23A462946BDE8F0415BE405
:1081C000A4F140001F2805D829462046BDE8F0410B
:1081D00000F0B2BAA4F1A0001F2805D82946204615
:1081E000BDE8F04100F0DDBA0720C8E72DE9F05FF7
:1081F00081460F460846F9F754F848B94846F9F75A
:108200006EF828B909F1030020F00301494501D0B7
:10821000102040E796484FF0000B3830817869B164
:108220004178804600EB411408343E883A460021EC
:10823000204600F067FA050004D027E0A7F800B058
:10824000052028E7B9F1000F24D03888B04201D9C1
:108250000C251FE0607800F00700824600F03EFA2F
:1082600008EB0A063A4696F8E8014946401C86F8AB
:10827000E801204600F046FA054696F8E801401E5F
:1082800086F8E801032000F029FA2DB10C2D01D069
:10829000A7F800B02846FEE6744F5046BAF1010F29
:1082A00025D002280DD0BAF1030F34D0FFDF98F8A3
:1082B00001104046491CC9B288F801100F2936D078
:1082C00037E0606828B16078000702D46088FFF763
:1082D0003DFE98F8EA014446012802D17878FAF781
:1082E00023FE94F9EA010428E1DBFFDFDFE76168A0
:1082F00019B14422B86806F099FA98F8E9014446A1
:10830000032802D17878FAF70FFE94F9E9010428DE
:10831000CDDBFFDFCBE76078C00602D56088FFF7D2
:1083200015FE98F9EB010628C1DBFFDFBFE780F8F7
:1083300001B08178491E88F8021096F8E801401CC7
:1083400086F8E801A6E770B50C460546F8F783FF06
:1083500018B92046F8F7A5FF08B1102070BD2846CF
:1083600008F045F9207008B1002070BD042070BDF0
:1083700070B5054608F054F9C4B22846F8F7AFFFC7
:1083800008B1102070BD35B128782C7018B1A0420A
:1083900001D0072070BD2046FDF7F0FE052805D16D
:1083A00008F041F9012801D0002070BD0F2070BDF8
:1083B00070B5044615460E460846F8F74CFF18B946
:1083C0002846F8F76EFF08B1102070BD022C03D0CC
:1083D000102C01D0092070BD2A463146204608F0F5
:1083E0004CF90028F7D0052070BD70B514460D4635
:1083F0000646F8F730FF38B92846F8F752FF18B9A3
:108400002046F8F76CFF08B1102070BD22462946BF
:10841000304608F034F90028F7D0072070BD3EB58B
:108420000446F8F73EFF08B110203EBD684605F04F
:10843000ABF8FFF76FFB0028F7D19DF8060020701E
:10844000BDF808006080BDF80A00A08000203EBD95
:1084500070B505460C460846F8F741FF20B95CB1F7
:108460002068F8F71EFF28B1102070BD1C00002006
:1084700068020020A08828B121462846BDE8704047
:10848000FDF7D4BE0920F0E770B504460D46084656
:10849000F8F7E1FE58BB601E1E280ED8032C01D948
:1084A0000720E2E704B9FFDFFC4800EB840050F846
:1084B000041C2846BDE870400847A4F120001F288E
:1084C00005D829462046BDE87040F9F766BDA4F1FD
:1084D00060001F2805D829462046BDE87040FCF7FB
:1084E0000ABFF02CDCD1A868F8F7B5FE08B110205F
:1084F000BBE7284605F012FCBDE87040FFF70ABB59
:1085000070B504460D460846F8F7CBFE30B9601E3C
:108510001E280FD82846F8F79EFE08B11020A4E7C1
:10852000012C03D0022C01D0032C01D106209CE7A2
:1085300007209AE7A4F120001F28F9D829462046F1
:10854000BDE87040F9F769BD05F08ABE08B500299D
:108550001CD102F0AEFFD24800224178C06804F07E
:10856000D9FECF481030C0788DF8000010B1012836
:1085700002D004E0012000E000208DF800006846F1
:1085800005F05DF8C548243805F087F908BD30B519
:10859000C44D04466878A04200D8FFDF686800EB4D
:1085A000C40030BD70B5BF4800252C46467807E0B2
:1085B0002046FFF7ECFF4078641C2844C5B2E4B2C3
:1085C000B442F5D1284650E72DE9F0410546B548BB
:1085D0004FF00008427A9600FF2E01D94FF01308A1
:1085E0002868C01C20F003022A6051EA080121D14A
:1085F000AC48F3B20521243009F0ECFF002408E078
:10860000052C0FD2DFE804F0050307070900A64890
:1086100004E0A64802E0A64800E0A64809F0FAFFF8
:10862000074600E0FFDFA74200D0FFDF641CE4B292
:10863000052CE5D3286800EB0610286040469EE52F
:10864000021D5143452900D245210844C01CB0FBFE
:10865000F2F0C0B270472DE9FC5F064691484FF03A
:1086600000088B464746444690F8019022E0204699
:10867000FFF78DFF050000D1FFDF687869463844B9
:10868000C7B22846FFF736F8824601A92846FFF709
:1086900045F80346BDF804005246001D81B2BDF8FE
:1086A0000000001D80B206F0BBFA6A78641C00FB73
:1086B0000288E4B24C45DAD13068C01C20F00300D7
:1086C0003060BBF1000F00D000204246394606F072
:1086D000B5FA316808443060BDE8FC9F7149383113
:1086E00008710020C87070476E493831CA782AB1C5
:1086F0000A7801EB42110831814201D00120704714
:10870000002070472DE9F04106460078154600F03C
:108710000F0400201080601E0F46052800D3FFDFE5
:108720005E482A46183800EB8400394650F8043C6D
:108730003046BDE8F04118472DE9F041594E0C464E
:10874000402806D041281AD0422822D0432826D1DA
:108750001AE020786578012801D913200FE5FF2D54
:1087600008D808F0FDF8074609F066FB381A401EE5
:10877000A84201DA122002E5208830810DE0BDE830
:10878000F041084600F03EB80878022807D8307655
:1087900003E00878022802D870760020EFE4072072
:1087A000EDE4F8B500243F4DA02805D0A12814D051
:1087B000A22806D00720F8BD087800F00100E8766E
:1087C0001EE00E4669463046FDF7D7FD0028F2D17F
:1087D0003088A883B078A87712E008680921F828C3
:1087E00001D3820701D00846F8BD6A7B02F003027C
:1087F000012A04D1EA8AD73293B28342F3D828629D
:108800002046F8BD38B50446407800F00300012842
:1088100003D002280BD0072038BD606858B1F8F7A4
:1088200067FDD0B96068F8F75AFD20B915E06068B7
:10883000F8F711FD88B969462046FBF72DFA0028A4
:10884000EAD1607800F00300022808D19DF800000A
:1088500028B16068F8F743FD08B1102038BD618980
:10886000F8290DD8208988420AD8607800F00302E0
:108870000C48012A06D1D731026A89B28A4201D254
:10888000092038BD94E80E0000F10C0585E80E00C3
:108890000AB900218182002038BD00005C8C0100F3
:1088A0001C00002068020020CF1E0000F1B800006C
:1088B000D92F00007303010070B50B2000F0B9F947
:1088C000082000F0B6F900210B2000F0D0F90021BB
:1088D000082000F0CCF9EE4C01256560A560002071
:1088E000C4F84001C4F84401C4F848010B2000F06A
:1088F000B1F9082000F0AEF90B2000F08DF92560E9
:1089000070BD10B50B2000F094F9082000F091F92B
:10891000DF48012141608160DE490A68002AFCD1FC
:108920000021C0F84011C0F84411C0F848110B20D4
:1089300000F090F9BDE81040082000F08BB910B5A8
:108940000B2000F087F9BDE81040082000F082B944
:1089500000B530B1012806D0022806D0FFDF002084
:1089600000BDCD4800BDCD4800BDCC48001D00BDB8
:1089700070B5CB494FF000400860CA4DC00BC5F838
:108980000803C94800240460C5F840410820C435E4
:1089900000F04FF9C5F83C41C448047070BD08B5FB
:1089A000BB4A002128B1012811D002281CD0FFDFCA
:1089B00008BD4FF48030C2F80803C2F84803B54838
:1089C0003C300160C2F84011BDE80840D0E74FF4E8
:1089D0000030C2F80803C2F84803AE4840300160D6
:1089E000C2F84411AD480CE04FF48020C2F80803EF
:1089F000C2F84803A74844300160C2F84811A748AC
:108A0000001D0068009008BD70B516460D4604466E
:108A1000022800D9FFDF00229D48012304F1100144
:108A20008B4000EB8401C1F8405526B1C1F84021CC
:108A3000C0F8043303E0C0F80833C1F84021C0F89F
:108A4000443370BD2DE9F0411D46144630B1012874
:108A500033D0022838D0FFDFBDE8F081891E002224
:108A600021F07F411046FFF7CFFF012D23D00020DA
:108A70008E4D8C4F012668703E618B4900203C3939
:108A800008600220091D0860874904203039086009
:108A900085483D34046008206C6000F0DBF8300449
:108AA000C7F80403082000F0B7F87D49F007091F54
:108AB00008602E70D0E70120DAE7012B02D00022F7
:108AC000012005E00122FBE7012B04D00022022057
:108AD000BDE8F04198E70122F9E76E480068704769
:108AE00070B56B4CD4F840010025012809D1D4F8A9
:108AF0000803C00305D54FF48030C4F80803C4F858
:108B00004051D4F8440101280CD1D4F80803800363
:108B100008D54FF40030C4F80803C4F844510120CC
:108B200008F0A4FDD4F8480101280ED1D4F80803B8
:108B300040030AD54FF48020C4F80803C4F8485114
:108B4000BDE87040022008F091BD70BD10B5574CD3
:108B5000207850B1FFF70CFF6078002807D0002084
:108B60006070BDE8104008F081BD0320F9E710BD3A
:108B70004FF0E0214FF40010C1F8000270471520BB
:108B800000F068B8474901200861082000F062B889
:108B900044494FF47C10C1F8080300204FEA00025A
:108BA00001EB8003C3F84025C3F84021401CC0B24C
:108BB0000628F5D37047410A43F609525143C0F3E2
:108BC000080010FB02F000F5807001EB50207047A8
:108BD00010B5430B48F2376463431B0C5C020C6016
:108BE000334C03FB0400334B4CF2F72443435B0D3F
:108BF00013FB04F404EB402000F580704012107069
:108C000008681844086010BD284840687047254926
:108C10000120C1F800027047002809DB00F01F02A4
:108C2000012191404009800000F1E020C0F80011CE
:108C3000704700280DDB00F01F0201219140400920
:108C4000800000F1E020C0F88011BFF34F8FBFF328
:108C50006F8F7047002809DB00F01F02012191404F
:108C60004009800000F1E020C0F8801270474907F9
:108C7000090E002804DB00F1E02080F800147047A2
:108C800000F00F0000F1E02080F8141D7047000094
:108C900000B0004004B500404081004044B10040B5
:108CA00008F5014000800040408500403000002071
:108CB000F7C2FFFF6F0C010010B5EFF3108000F05A
:108CC000010472B6F7484178491C41704078012888
:108CD00001D109F021F9002C00D162B610BD70B5A8
:108CE000F04CA07848B90125A570FFF7E5FF09F021
:108CF00024F920B1002009F0EEF8002070BD4FF0FB
:108D00008040E570C0F80453F7E770B5EFF31080CA
:108D100000F0010572B6E34C607800B9FFDF6078BF
:108D2000401E6070607808B909F0FAF8002D00D193
:108D300062B670BDDB4810B5817821B10021C170E9
:108D40008170FFF7E2FF002010BD10B5044609F066
:108D5000F4F8D4498978084000D001202060002030
:108D600010BD10B5FFF7A8FF09F0E7F802220123B4
:108D7000CC49540728B1CC48026023610320087213
:108D800002E00A72C4F804330020887110BD2DE996
:108D9000F84FDFF810934278817889F80420002694
:108DA00089F80510074689F806600078DFF8FCB2FC
:108DB000354620B1012811D0022811D0FFDF09F07B
:108DC000CEF84FF0804498B109F0D0F8B0420FD1FE
:108DD000304609F0CFF80028FAD042E00126EEE74D
:108DE000FFF76AFF58460168C907FCD00226E6E78C
:108DF0000120E060C4F80451AD490E600107D1F8CC
:108E00004412AB4AC1F3423124321160A8493431D3
:108E100008604FF0020AC4F804A3A060A5480168E6
:108E2000C94341F3001101F10108016841F010014B
:108E3000016001E00FF046FDD4F804010028F9D0EC
:108E4000304609F097F80028FAD0B8F1000F04D1A5
:108E50009848016821F010010160C4F808A3C4F823
:108E6000045199F805004E4680B1387870B909F080
:108E700064F8804609F06CFA6FF00042B8F1000F18
:108E800002D0C6E9032001E0C6E90302DBF80000D6
:108E9000C00701D009F04DF8387810B13572BDE83F
:108EA000F88F4FF01808C4F808830127A7614FF422
:108EB0002070ADF8000000BFBDF80000411EADF805
:108EC0000010F9D2C4F80C51C4F810517548C01DF7
:108ED00009F0DAF83570FFF744FF676174493079BB
:108EE00020310860C4F80483D9E770B5050000D1CB
:108EF000FFDF4FF080424FF0FF30C2F8080300213F
:108F0000C2F80011C2F80411C2F80C11C2F8101115
:108F1000644C617009F01DF810B10120A070607000
:108F200062480068C00701D009F003F82846BDE890
:108F300070402CE75B48007A002800D00120704781
:108F40002DE9FF5F4FF080444FF0000AD4F808018C
:108F5000D146574610B14FF0010801E04FF000082C
:108F600009F065F878B1D4F8240100B101208246F7
:108F7000D4F81C0100B101208146D4F8200108B1C9
:108F8000012700E00027D4F8000100B1012083464A
:108F9000D4F8040100B101200390D4F80C0100B111
:108FA00001200290D4F8100100B101203D4D019044
:108FB000287800260090B8F1000F04D0C4F80861AA
:108FC000012008F088FFBAF1000F04D0C4F8246132
:108FD000092008F080FFB9F1000F04D0C4F81C612B
:108FE0000A2008F078FF27B1C4F820610B2008F0B0
:108FF00072FF2C48C01D09F04FF800B1FFDFDFF809
:10900000A8800127BBF1000F10D0C4F80873E878DE
:1090100018B1EE70002008F05EFF287A022805D112
:10902000032028720221C8F800102761039808B1B4
:10903000C4F80461029850B1C4F80C61287A03287E
:1090400000D0FFDFC8F800602F72FFF75EFE0198C6
:1090500038B1C4F81061287A012801D100F054F821
:109060006761009838B12E70287A012801D1FFF786
:1090700078FEFFF74AFE04B00A48BDE8F05FC01D65
:1090800009F020B8074810B5C01D09F005F80549DA
:1090900090B1012008704FF0E021C1F80002BDE856
:1090A000104009E638000020340C00400C04004059
:1090B0001805004010ED00E0087A012801D1FFF703
:1090C00050FEBDE81040244808F0FCBF70B5224CAB
:1090D000E41FA07808B908F023FF01208507A861E4
:1090E000207A0026032809D1D5F80C0120B90020E8
:1090F00008F040FF0028F7D1C5F80C6126724FF048
:10910000FF30C5F8080370BD70B5134CE41F6079DB
:10911000F0B1012803D0A179401E814218DA08F08D
:109120000CFF054609F014F96179012902D9A179EA
:10913000491CA1710DB1216900E0E168411A0229C1
:1091400002DA11F1020F06DC0DB1206100E0E060EF
:10915000BDE8704005E670BD3F0000200E4A126871
:109160000C498A420AD118470B4A1268094B9A42A5
:1091700004D101B509F0C6F8BDE801400749096806
:109180000958084706480749054A064B704700003A
:1091900000000000BEBAFECA5000002004000020FB
:1091A000D80C0020D80C0020F8B51D46DDE9064794
:1091B0000E000AD005F0F9FD2346FF1DBCB2314672
:1091C0002A46009405F025FAF8BDD0192246194622
:1091D00002F023F92046F8BD70B50D460446102272
:1091E000002102F044F9258117206081A07B40F026
:1091F0000A00A07370BD4FF6FF720A80014602207C
:1092000009F0C2BA704700897047827BD30701D149
:10921000920703D48089088000207047052070479A
:10922000827B920700D58181704701460020098822
:1092300041F6FE52114200D00120704700B50346AE
:10924000807BC00701D0052000BD59811846FFF77B
:10925000ECFFC00703D0987B40F004009873987B24
:1092600040F001009873002000BD827B520700D5BA
:1092700009B14089704717207047827B61F3C302B0
:10928000827370472DE9FC5F0E46044601789646CE
:10929000012000FA01F14DF6FF5201EA020962686D
:1092A0004FF6FF7B1188594502D10920BDE8FC9F8C
:1092B000B9F1000F05D041F6FE55294201D0012039
:1092C000F4E741EA090111801D0014D000232B703E
:1092D00094F800C0052103221F464FF0020ABCF19A
:1092E0000E0F76D2DFE80CF0F909252F47646B7773
:1092F000479193B4D1D80420D8E7616820898B7B4B
:109300009B0767D517284AD30B89834247D389899E
:10931000172901D3814242D185F800A0A5F80100A8
:109320003280616888816068817B21F002018173ED
:10933000C6E0042028702089A5F801006089A5F8FE
:1093400003003180BCE0208A3188C01D1FFA80F8FC
:10935000414524D3062028702089A5F801006089A2
:10936000A5F80300A089A5F805000721208ACDE90A
:109370000001636941E00CF0FF00082810D00820CC
:1093800028702089A5F801006089A5F803003180C4
:109390006A1D694604F10C0007F071F910B15EE036
:1093A0001020EDE730889DF800100844308087E0F9
:1093B0000A2028702089A5F80100328044E00C20A2
:1093C00028702089A5F801006089A5F80300318084
:1093D0003AE082E064E02189338800EB41021FFA21
:1093E00082F843453BD3B8F1050F38D30E222A70DB
:1093F0000BEA4101CDE90010E36860882A46714616
:10940000FFF7D2FEA6F800805AE04020287060895D
:109410003188C01C1FFA80F8414520D32878714656
:1094200020F03F00123028702089A5F801006089E3
:10943000CDE9000260882A46E368FFF7B5FEA6F88A
:109440000080287840063BD461682089888037E016
:10945000A0893288401D1FFA80F8424501D20427B6
:109460003DE0162028702089A5F801006089A5F844
:109470000300A089CDE9000160882A46714623696E
:10948000FFF792FEA6F80080DEE718202870207A09
:109490006870A6F800A013E061680A88920401D4FD
:1094A00005271CE0C9882289914201D0062716E0D1
:1094B0001E21297030806068018821F400510180EC
:1094C000B9F1000F0BD0618878230022022009F047
:1094D000B1F861682078887006E0338003276068FF
:1094E000018821EA090101803846DFE62DE9FF4FB6
:1094F00085B01746129C0D001E461CD03078C1075F
:1095000003D000F03F00192801D9012100E000211B
:109510002046FFF7AAFEA8420DD32088A0F57F4180
:10952000FF3908D03078410601D4000605D508205F
:1095300009B0BDE8F08F0720FAE700208DF80000A1
:109540008DF8010030786B1E00F03F0C0121A81E41
:109550004FF0050A4FF002094FF0030B9AB2BCF12D
:10956000200F75D2DFE80CF08B10745E7468748C79
:10957000749C74B574BA74C874D474E1747474F15E
:1095800074EF74EE74ED748B052D78D18DF8009026
:10959000A0788DF804007088ADF8060030798DF859
:1095A0000100707800F03F000C2829D00ADCA0F1FF
:1095B0000200092863D2DFE800F0126215621A6225
:1095C0001D622000122824D004DC0E281BD0102895
:1095D000DBD11BE016281FD01828D6D11FE0207839
:1095E000800701E020784007002848DAEEE0207884
:1095F0000007F9E72078C006F6E720788006F3E751
:1096000020784006F0E720780006EDE72088C005C6
:10961000EAE720884005E7E720880005E4E720889E
:10962000C004E1E72078800729D5032D27D18DF8E4
:1096300000B0B6F8010081E0217849071FD5062D5A
:109640001DD381B27078012803D0022817D102E01F
:10965000C9E0022000E0102004228DF8002072787A
:109660008DF80420801CB1FBF0F2ADF8062092B218
:1096700042438A4203D10397ADF80890A6E079E00F
:109680002078000776D598B282088DF800A0ADF852
:109690000420B0EB820F6DD10297ADF8061095E073
:1096A0002178C90666D5022D64D381B206208DF8D3
:1096B0000000707802285DD3B1FBF0F28DF8040051
:1096C000ADF8062092B242438A4253D1ADF80890D9
:1096D0007BE0207880064DD5072003E02078400607
:1096E0007FD508208DF80000A088ADF80400ADF803
:1096F0000620ADF8081068E02078000671D5092032
:10970000ADF804208DF80000ADF8061002975DE07A
:109710002188C90565D5022D63D381B20A208DF851
:109720000000707804285CD3C6E72088400558D52F
:10973000012D56D10B208DF80000A088ADF8040053
:1097400044E021E026E016E0FFE72088000548D548
:10975000052D46D30C208DF80000A088ADF804003C
:10976000B6F803006D1FADF80850ADF80600ADF86F
:109770000AA02AE035E02088C00432D5012D30D17E
:109780000D208DF8000021E02088800429D4B6F84F
:109790000100E080A07B000723D5032D21D3307882
:1097A00000F03F001B2818D00F208DF80000208803
:1097B00040F40050A4F80000B6F80100ADF8040031
:1097C000ED1EADF80650ADF808B003976946059850
:1097D000FBF748FA050008D016E00E208DF80000CF
:1097E000EAE7072510E008250EE0307800F03F009A
:1097F0001B2809D01D2807D00220059908F0C4FFB6
:10980000208800F400502080A07B400708D5204627
:10981000FFF70BFDC00703D1A07B20F00400A0736D
:10982000284685E61FB5022806D101208DF80000E4
:1098300088B26946FBF716FA1FBD0000F8B51D4651
:10984000DDE906470E000AD005F0AFFA2346FF1DFA
:10985000BCB231462A46009404F0DBFEF8BDD019B4
:109860002246194601F0D9FD2046F8BD2DE9FF4FEB
:109870008DB09B46DDE91B57DDF87CA00C46082B1C
:1098800005D0E06901F0FEF850B11020D2E0288840
:10989000092140F0100028808AF80010022617E005
:1098A000E16901208871E2694FF420519180E169FA
:1098B0008872E06942F601010181E069002181734B
:1098C0002888112140F0200028808AF80010042602
:1098D00038780A900A2038704FF0020904F1180015
:1098E0004D460C9001F0C6FBB04681E0BBF1100F75
:1098F0000ED1022D0CD0A9EB0800801C80B20221F1
:10990000CDE9001005AB52461E990D98FFF796FF62
:10991000BDF816101A98814203D9F74800790F90C4
:1099200004E003D10A9808B138702FE04FF002012B
:10993000CDE900190DF1160352461E990D98FFF757
:109940007DFF1D980088401B801B83B2C6F1FF007D
:10995000984200D203461E990BA8D9B15FF00002CD
:10996000DDF878C0CDE9032009EB060189B2CDE925
:1099700001C10F980090BDF8161000220D9801F05B
:109980000EFC387070B1C0B2832807D0BDF8160045
:1099900020833AE00AEB09018A19E1E7022011B0BD
:1099A000BDE8F08FBDF82C00811901F0FF08022DF1
:1099B0000DD09AF80120424506D1BDF82010814211
:1099C00007D0B8F1FF0F04D09AF801801FE08AF8A1
:1099D0000180C94800680178052902D1BDF8161038
:1099E000818009EB08001FFA80F905EB080085B2B9
:1099F000DDE90C1005AB0F9A01F03FFB28B91D986B
:109A00000088411B4145BFF671AF022D13D0BBF159
:109A1000100F0CD1A9EB0800801C81B20220CDE907
:109A2000000105AB52461E990D98FFF707FF1D98E0
:109A30000580002038700020B1E72DE9F8439C46EE
:109A4000089E13460027B26B9AB3491F8CB2F18F60
:109A5000A1F57F45FF3D05D05518AD882944891DE6
:109A60008DB200E000252919B6F83C800831414547
:109A700020D82A44BCF8011022F8021BBCF80310BD
:109A800022F8021B984622F8024B914605F07BF91A
:109A90004FF00C0C41464A462346CDF800C004F076
:109AA00084FDF587B16B00202944A41D2144088062
:109AB00003E001E0092700E083273846BDE8F8838A
:109AC00010B50B88848F9C420CD9846BE0180488F5
:109AD00044B1848824F40044A41D23440B80106006
:109AE000002010BD0A2010BD2DE9F0478AB00025E6
:109AF000904689468246ADF8185007274BE00598F6
:109B000006888088000446D4A8F8006007A801955C
:109B100000970295CDE903504FF4007300223146BF
:109B2000504601F03CFB04003CD1BDF81800ADF8F4
:109B30002000059804888188B44216D10A0414D400
:109B400001950295039521F400410097049541F495
:109B5000804342882146504601F0BFF804000BD1F3
:109B60000598818841F40041818005AA08A94846EA
:109B7000FFF7A6FF0400DCD0009705980295019539
:109B8000039504950188BDF81C300022504601F071
:109B9000A4F80A2C06D105AA06A94846FFF790FFAB
:109BA0000400ACD0ADF8185004E00598818821F489
:109BB0000041818005AA06A94846FFF781FF0028D9
:109BC000F3D00A2C03D020460AB0BDE8F08700206D
:109BD000FAE710B50C46896B86B051B10C218DF8AF
:109BE0000010A18FADF80810A16B01916946FBF739
:109BF000F9FF00204FF6FF71A063E187A08706B050
:109C000010BD2DE9F0410D460746896B0020069EE8
:109C10001446002911D0012B0FD13246294638466F
:109C2000FFF762FF002808D1002C06D032462946F3
:109C30003846BDE8F04100F034BFBDE8F0812DE9C1
:109C4000FC411446DDE9087C0E46DDE90A15521D8B
:109C5000BCF800E092B2964502D20720BDE8FC8134
:109C6000ACF8002017222A70A5F80160A5F803308F
:109C70000522CDE900423B462A46FFF7DFFD0020E2
:109C8000ECE770B50C46154648220021204601F04D
:109C9000EEFB04F1080044F81C0F00204FF6FF71A2
:109CA000E06161842084A5841720E08494F82A0070
:109CB00040F00A0084F82A0070BD4FF6FF720A8057
:109CC0000146032008F060BD30B585B00C4605465E
:109CD000FFF77FFFA18E284629B101218DF80010E2
:109CE0006946FBF77FFF0020E0622063606305B0F8
:109CF00030BDB0F8400070475400002090F8462076
:109D0000920703D4408808800020F4E70620F2E799
:109D100090F846209207EED5A0F84410EBE70146F4
:109D2000002009880A0700D5012011F0F00F01D0AA
:109D300040F00200CA0501D540F004008A0501D5B3
:109D400040F008004A0501D540F010000905D2D5C1
:109D500040F02000CFE700B5034690F84600C0076A
:109D600001D0062000BDA3F842101846FFF7D7FF28
:109D700010F03E0F05D093F8460040F0040083F841
:109D8000460013F8460F40F001001870002000BD97
:109D900090F84620520700D511B1B0F84200AAE76A
:109DA0001720A8E710F8462F61F3C3020270A2E75C
:109DB0002DE9FF4F9BB00E00DDE92B34DDE929785A
:109DC000289D24D02878C10703D000F03F0019282F
:109DD00001D9012100E000212046FFF7D9FFB04260
:109DE00015D32878410600F03F010CD41E290CD071
:109DF000218811F47F6F0AD13A8842B1A1F57F42E0
:109E0000FF3A04D001E0122901D1000602D5042056
:109E10001FB0C5E5FA491D984FF0000A08718DF88A
:109E200018A08DF83CA00FAA0A60ADF81CA0ADF8F0
:109E300050A02978994601F03F02701F5B1C04F185
:109E4000180C4FF0060E4FF0040BCDF858C01F2A27
:109E50007ED2DFE802F07D7D107D267DAC7DF47D35
:109E6000F37DF27DF17DF47DF07D7D7DEF7DEE7DF6
:109E70007D7D7D7DED0094F84610B5F801008907E1
:109E800001D5032E02D08DF818B01EE34FF4006107
:109E9000ADF85010608003218DF83C10ADF8400003
:109EA000D4E2052EEFD1B5F801002083ADF81C00F7
:109EB000B5F80310618308B1884201D9012079E126
:109EC0000020A07220814FF6FF702084169801F0C8
:109ED000D1F8052089F800000220029083460AABE1
:109EE0001D9A16991B9801F0C8F890BB9DF82E009A
:109EF000012804D0022089F80100102003E001208D
:109F000089F8010002200590002203A90BA806F0A1
:109F1000B6FBE8BB9DF80C00059981423DD139881C
:109F2000801CA1EB0B01814237DB02990220CDE9B5
:109F300000010DF12A034A4641461B98FFF77EFCBB
:109F400002980BF1020B801C81B217AA029101E06A
:109F50009CE228E003A90BA806F091FB02999DF86A
:109F60000C00CDE9000117AB4A4641461B98FFF7AC
:109F700065FC9DF80C000AAB0BEB00011FFA81FB9E
:109F800002991D9A084480B2029016991B9800E02D
:109F900003E001F072F80028B6D0BBF1020F02D046
:109FA000A7F800B04FE20A208DF818004BE200211C
:109FB0000391072EFFF467AFB5F801002083ADF8D9
:109FC0001C00B5F80320628300283FF477AF90426D
:109FD0003FF674AF0120A072B5F805002081002083
:109FE000A073E06900F04EFD78B9E1690120887145
:109FF000E2694FF420519180E1698872E16942F68B
:10A0000001000881E06900218173F01F20841E98FF
:10A01000606207206084169801F02CF8072089F808
:10A0200000000120049002900020ADF82A0028E0F2
:10A0300019E29FE135E1E5E012E2A8E080E043E0CB
:10A040000298012814D0E0698079012803D1BDF875
:10A050002800ADF80E00049803ABCDE900B04A46E5
:10A0600041461B98FFF7EAFB0498001D80B204905C
:10A07000BDF82A00ADF80C00ADF80E00059880B2CE
:10A0800002900AAB1D9A16991B9800F0F6FF28B9AA
:10A0900002983988001D05908142D1D2029801288A
:10A0A00081D0E0698079012803D1BDF82800ADF89E
:10A0B0000E00049803ABCDE900B04A4641461B9818
:10A0C000FFF7BCFB0298BDE1072E02D0152E7FF4EE
:10A0D000DAAEB5F801102183ADF81C10B5F80320F5
:10A0E000628300293FF4EAAE91423FF6E7AE0121D8
:10A0F000A1724FF0000BA4F808B084F80EB0052E42
:10A1000007D0C0B2691DE26906F0B7FA00287FF4F3
:10A110004AAF4FF6FF70208401A906AA14A8CDF813
:10A1200000B081E885032878214600F03F031D9A9E
:10A130001B98FFF79BFB8246208BADF81C0082E149
:10A140000120032EC3D14021ADF85010B5F8011005
:10A150002183ADF81C100AAAB8F1000F00D000232B
:10A16000CDE9020304921D98CDF804800090388850
:10A170000022401E83B21B9801F011F88DF81800E0
:10A1800090BB0B2089F80000BDF8280035E04FF0A7
:10A19000010C052E9BD18020ADF85000B5F80110C0
:10A1A0002183B5F803002084ADF81C10B0F5007FC2
:10A1B00003D907208DF8180087E140F47C422284FF
:10A1C0000CA8B8F1000F00D00023CDE90330CDE991
:10A1D000018C1D9800903888401E83B21B9800F0B7
:10A1E000DEFF8DF8180018B18328A8D10220BFE047
:10A1F0000D2189F80010BDF83000401C22E100005C
:10A2000054000020032E04D248067FF53CAE002007
:10A2100018E1B5F80110ADF81C102878400602D5F9
:10A220008DF83CE002E007208DF83C004FF000087C
:10A230000320CDE902081E9BCDF810801D980193E4
:10A24000A6F1030B00901FFA8BF342461B9800F017
:10A2500044FD8DF818008DF83C80297849060DD50D
:10A260002088C00506D5208BBDF81C10884201D17E
:10A27000C4F8248040468DF81880E3E0832801D19B
:10A280004FF0020A4FF48070ADF85000BDF81C008A
:10A290002083A4F820B01E986062032060841321FC
:10A2A000CDE0052EFFF4EFADB5F80110ADF81C10B0
:10A2B000A28F6AB3A2F57F43FE3B29D008228DF816
:10A2C0003C2000BF4FF0000B0523CDE9023BDDF839
:10A2D00078C0CDF810B01D9A80B2CDF804C040F41B
:10A2E00000430092B5F803201B9800F0F6FC8DF8AF
:10A2F0003CB04FF400718DF81800ADF85010832871
:10A3000010D0F8B1A18FA1F57F40FE3807D0DCE076
:10A310000B228DF83C204FF6FE72A287D2E7A4F8FC
:10A320003CB0D2E000942B4631461E9A1B98FFF7B2
:10A3300084FB8DF8180008B183284BD1BDF81C00B0
:10A34000208353E700942B4631461E9A1B98FFF753
:10A3500074FB8DF81800E8BBE18FA06B0844831DE7
:10A360008DE888034388828801881B98FFF767FC83
:10A37000824668E095F80180022E70D15FEA0800FD
:10A3800002D0B8F1010F6AD109208DF83C0007A86E
:10A3900000908DF840804346002221461B98FFF72D
:10A3A00030FC8DF842004FF0000B8DF843B050B9EF
:10A3B000B8F1010F12D0B8F1000F04D1A18FA1F5AF
:10A3C0007F40FF380AD0A08F40B18DF83CB04FF4E9
:10A3D000806000E037E0ADF850000DE00FA91B9859
:10A3E000FBF700FC82468DF83CB04FF48060ADF87E
:10A3F0005000BAF1020F06D0FC480068C07928B1BD
:10A400008DF8180027E0A4F8188044E0BAF1000F96
:10A4100003D081208DF818003DE007A80090434646
:10A42000012221461B98FFF7ECFB8DF8180021460E
:10A430001B98FFF7CEFB9DF8180020B9192189F869
:10A440000010012038809DF83C0020B10FA91B9816
:10A45000FBF7C8FB8246BAF1000F33D01BE018E0CF
:10A460008DF818E031E02078000712D5012E10D1C8
:10A470000A208DF83C00E088ADF8400003201B99CD
:10A4800008F082F90820ADF85000C0E648067FF5D4
:10A49000FAAC4FF0040A2088BDF850100843208021
:10A4A000BDF8500080050BD5A18FA1F57F40FE3887
:10A4B00006D11E98E06228982063A6864FF0030A12
:10A4C0005046A5E49DF8180078B1012089F80000F5
:10A4D000297889F80110BDF81C10A9F802109DF820
:10A4E000181089F80410052038802088BDF8501015
:10A4F00088432080E4E72DE9FF4F8846087895B02F
:10A50000012181404FF20900249C0140ADF8201048
:10A510002088DDF88890A0F57F424FF0000AFF3ACE
:10A5200006D039B1000705D5012019B0BDE8F08F7C
:10A530000820FAE7239E4FF0000B0EA886F800B023
:10A5400018995D460988ADF83410A8498DF81CB0FB
:10A55000179A0A718DF838B0086098F80000012841
:10A560003BD0022809D003286FD1307820F03F007B
:10A570001D303070B8F80400E08098F80010032017
:10A58000022904D1317821F03F011B31317094F858
:10A590004610090759D505ABB9F1000F13D00021BA
:10A5A00002AA82E80B000720CDE90009BDF83400BB
:10A5B000B8F80410C01E83B20022159800F0EFFD19
:10A5C0000028D1D101E0F11CEAE7B8F80400A6F8B0
:10A5D0000100BDF81400C01C04E198F805108DF8C6
:10A5E0001C1098F80400012806D04FF4007A0228C5
:10A5F0002CD00328B8D16CE12188B8F8080011F4F8
:10A600000061ADF8201020D017281CD3B4F84010FA
:10A61000814218D3B4F84410172901D3814212D1D2
:10A62000317821F03F01C91C3170A6F801000321E7
:10A63000ADF83410A4F8440094F8460020F002006D
:10A6400084F8460065E105257EE177E1208808F180
:10A65000080700F4FE60ADF8200010F0F00F1BD0EA
:10A6600010F0C00F03D03888228B9042EBD199B9FB
:10A67000B878C00710D0B9680720CDE902B1CDF88D
:10A6800004B00090CDF810B0FB88BA8839881598CE
:10A6900000F023FB0028D6D12398BDF82010401CE1
:10A6A00080294ED006DC10290DD020290BD040295E
:10A6B00087D124E0B1F5807F6ED051457ED0B1F5D1
:10A6C000806F97D1DEE0C80601D5082000E0102099
:10A6D00082460DA907AA0520CDE902218DF8380090
:10A6E000ADF83CB0CDE9049608A93888CDE9000161
:10A6F0005346072221461598FFF7B8F8A8E09DF8C1
:10A700001C2001214FF00A0A002A9BD105ABB9F1A8
:10A71000000F00D00020CDE902100720CDE900098C
:10A72000BDF834000493401E83B2218B002215989B
:10A7300000F035FD8DF81C000B203070BDF81400C2
:10A7400020E09DF81C2001214FF00C0A002A22D1A4
:10A7500013ABB9F1000F00D00020CDE902100720A3
:10A76000CDE900090493BDF83400228C401E83B269
:10A77000218B159800F013FD8DF81C000D20307012
:10A78000BDF84C00401CADF8340005208DF83800B1
:10A79000208BADF83C00BCE03888218B88427FF4E8
:10A7A00052AF9DF81C004FF0120A00281CD1606ABD
:10A7B000A8B1B878C0073FF446AF00E018E0BA6827
:10A7C0000720CDE902B2CDF804B00090CDF810B06A
:10A7D000FB88BA88159800F080FA8DF81C001320C9
:10A7E00030700120ADF8340093E0000054000020E8
:10A7F0003988208B8142D2D19DF81C004FF0160A77
:10A800000028A06B08D0E0B34FF6FF7000215F4630
:10A81000ADF808B0019027E068B1B978C907BED19A
:10A82000E18F0DAB0844821D03968DE80C0243882E
:10A830008288018809E0B878C007BCD0BA680DAB3F
:10A8400003968DE80C02BB88FA881598FFF7F7F994
:10A8500005005ED0072D72D076E0019005AA02A90E
:10A860002046FFF72DF90146E28FBDF8080082422D
:10A8700001D00029F1D0E08FA16B08440780019836
:10A88000E08746E09DF81C004FF0180A40B1208B8D
:10A89000C8B13888208321461598FFF79AF938E027
:10A8A00004F118000090237E012221461598FFF73D
:10A8B000A8F98DF81C000028EDD119203070012076
:10A8C000ADF83400E7E7052521461598FFF781F933
:10A8D0003AE0208800F40070ADF8200050452DD1FA
:10A8E000A08FA0F57F41FE3901D006252CE0D8F8D5
:10A8F00008004FF0160A48B1A063B8F80C10A18701
:10A900004FF6FF71E187A0F800B002E04FF6FF704C
:10A91000A087BDF8200030F47F611AD07823002290
:10A920000320159907F086FE98F800002071208812
:10A93000BDF82010084320800EE000E007252088A5
:10A94000BDF8201088432080208810F47F6F1CD031
:10A950003AE02188814321809DF8380020B10EA97A
:10A960001598FBF73FF905469DF81C000028EBD031
:10A9700086F801A001203070208B70809DF81C00AB
:10A9800030710520ADF83400DEE7A18EE1B11898F2
:10A990000DAB0088ADF834002398CDE90304CDE970
:10A9A0000139206B0090E36A179A1598FFF700FAB7
:10A9B000054601208DF838000EA91598FBF712F90D
:10A9C00000B10546A4F834B094F8460040070AD513
:10A9D0002046FFF7A4F910F03E0F04D114F8460FFB
:10A9E00020F0040020701898BDF83410018028462B
:10A9F0009BE500B585B0032806D102208DF8000044
:10AA000088B26946FBF7EEF805B000BD10B5384CCA
:10AA10000B782268012B02D0022B2AD111E0137887
:10AA20000BB1052B01D10423137023688A889A8007
:10AA30002268CB88D38022680B8913814989518190
:10AA40000DE08B8893802268CB88D38022680B89A5
:10AA500013814B8953818B89938109691161216825
:10AA6000FBF7C0F8226800210228117003D00028EB
:10AA700000D0812010BD832010BD806B002800D045
:10AA8000012070478178012909D10088B0F5205F45
:10AA900003D042F60101884201D10020704707200F
:10AAA0007047F0B587B0002415460E460746ADF84E
:10AAB000184011E005980088288005980194811DB0
:10AAC000CDE90241072104940091838842880188DE
:10AAD000384600F002F930B905AA06A93046FEF75B
:10AAE000EFFF0028E6D00A2800D1002007B0F0BD13
:10AAF0005400002010B58B7883B102789A4205D1BA
:10AB00000B885BB102E08B79091D4BB18B789A42BF
:10AB1000F9D1B0F801300C88A342F4D1002010BD67
:10AB2000812010BD072826D012B1012A27D103E0C9
:10AB3000497801F0070102E04978C1F3C201052913
:10AB40001DD2DFE801F00318080C12000AB103203F
:10AB500070470220704704280DD250B10DE005283F
:10AB600009D2801E022808D303E0062803D0032858
:10AB700003D005207047002070470F2070478120C8
:10AB80007047C0B282060BD4000607D5FA48807A17
:10AB90004143C01D01EBD00080B2704708467047AA
:10ABA0000020704770B513880B800B781C0625D5E4
:10ABB000F14CA47A844204D843F0100008700020BD
:10ABC00070BD956800F0070605EBD0052D78F540BF
:10ABD00065F304130B701378D17803F0030341EA93
:10ABE000032140F20123B1FBF3F503FB1511926839
:10ABF000E41D00FB012000EBD40070BD906870BD27
:10AC000037B51446BDF804101180117841F00401E5
:10AC100011709DF804100A061ED5D74AA368C1F327
:10AC20000011927A824208D8FE2811D1D21DD20892
:10AC30004942184600F01BFC0AE003EBD00200F08A
:10AC40000703012510789D40A843994008431070E0
:10AC5000207820F0100020703EBD2DE9F04107461D
:10AC6000C81C0E4620F00300B04202D08620BDE88A
:10AC7000F081C14D002034462E60AF802881AA7239
:10AC8000E8801AE0E988491CE980810614D4E1785B
:10AC900000F0030041EA002040F20121B0FBF1F294
:10ACA00001FB12012068FFF76CFF2989084480B27C
:10ACB0002881381A3044A0600C3420784107E1D450
:10ACC0000020D4E7AC4801220189C08800EB400095
:10ACD00002EB8000084480B270472DE9FF4F89B035
:10ACE0001646DDE9168A0F46994623F44045084684
:10ACF00000F054FB040002D02078400703D4012068
:10AD00000DB0BDE8F08F099803F0D6FE02902078D0
:10AD1000000606D59848817A0298814201D887209A
:10AD2000EEE7224601A90298FFF73CFF8346002088
:10AD30008DF80C004046B8F1070F1AD001222146C9
:10AD4000FFF7F0FE0028DBD12078400611D5022065
:10AD50008DF80C00ADF81070BDF80400ADF81200CD
:10AD6000ADF814601898ADF81650CDF81CA0ADF8E9
:10AD700018005FEA094004D500252E46A8460127A1
:10AD80000CE02178E07801F0030140EA012040F274
:10AD90000121B0FBF1F2804601FB12875FEA4940D6
:10ADA00009D5B84507D1A178207901F0030140EA1F
:10ADB0000120B04201D3BE4201D90720A0E7A81963
:10ADC0001FFA80F9B94501D90D2099E79DF80C00CB
:10ADD00028B103A90998FAF703FF002890D1B845D4
:10ADE00007D1A0784FEA192161F30100A07084F81F
:10ADF00004901A9800B10580199850EA0A0027D0EB
:10AE0000199830B10BEB06002A46199900F005FBA2
:10AE10000EE00BEB06085746189E099803F0B3FFA7
:10AE20002B46F61DB5B239464246009503F0BDFBF0
:10AE3000224601A90298FFF7B5FE9DF804002246BC
:10AE400020F010008DF80400DDE90110FFF7D8FEB6
:10AE5000002055E72DE9FF4FDFF81C91824685B0B1
:10AE6000B9F80610D9F8000001EB410100EB8104AC
:10AE700040F20120B2FBF0F1174600FB1175DDE94D
:10AE8000138B4E4629460698FFF77BFE0346FFF7D5
:10AE900019FF1844B1880C30884202D9842009B0C7
:10AEA0002FE70698C6B2300603D5B00601D50620B6
:10AEB000F5E7B9F80620521C92B2A9F80620BBF1BA
:10AEC000000F01D0ABF80020B00602D5C4F808800E
:10AED0000AE0B9F808201A4492B2A9F80820D9F873
:10AEE0000000891A0844A0602246FE200699FFF758
:10AEF00087FEE77025712078390A61F301002A0A7C
:10AF0000A17840F0040062F30101A17020709AF86A
:10AF100002006071BAF80000E08000252573300659
:10AF200002D599F80A7000E00127B00601D54FF06C
:10AF300000084E4600244FF007090FE0CDE9025803
:10AF40000195CDF800900495F1882046129B089A4F
:10AF5000FFF7C3FE0028A2D1641CE4B2BC42EDD3CB
:10AF600000209CE700B5FFF7ADFE03490C308A884E
:10AF7000904203D9842000BDAC040020CA88086830
:10AF800002EB420300EB8300521C037823F004031E
:10AF90000370CA80002101730846ECE72DE9F047F1
:10AFA000804600F0FBF9070005D000264446F74D27
:10AFB00040F2012916E00120BDE8F087204600F0AC
:10AFC000EDF90278C17802F0030241EA0222B2FBF5
:10AFD000F9F309FB13210068FFF7D3FD3044641C2B
:10AFE00086B2A4B2E988601E8142E7DCA8F10100C4
:10AFF000E8802889801B288100203870DCE710B5A4
:10B00000144631B1491E218003F056FDA070002086
:10B0100010BD012010BD70B50446DC48C18803682E
:10B0200001E0401C20802088884207D200EB4002CB
:10B0300013EB820202D015786D07F2D580B28842F8
:10B0400016D2AAB15079A072D08820819178107957
:10B0500001F0030140EA0120A081A078E11CFFF784
:10B06000A1FD20612088401C2080E080002070BD70
:10B070000A2070BD0121018270472DE9FF4F85B084
:10B080004FF6FF798246A3F8009048681E460D46A9
:10B0900080788DF8060048680088ADF8040000202C
:10B0A0008DF80A00088A0C88A04200D304462C823E
:10B0B00051E03878400708D4641C288AA4B2401CA8
:10B0C000288208F10100C0B246E0288A401C28828C
:10B0D000781D6968FFF70EFDD8BB3188494501D15D
:10B0E000601E30803188A1EB080030806888A04263
:10B0F00038D3B878397900F0030041EA002801A973
:10B10000781DFFF7F7FC20BB298949452ED0002286
:10B1100039460798FFF706FDD8B92989414518D166
:10B12000E9680391B5F80AC0D7F808B05046CDF8E1
:10B1300000C003F028FEDDF800C05A460CF1070CF1
:10B140001FFA8CFC43460399CDF800C003F0F7F9D1
:10B1500060B1641CA4B200208046204600F01EF9B5
:10B160000700A6D1641E2C820A2098E674807879A4
:10B17000B071F888B0803978F87801F0030140EABE
:10B1800001207081A6F80C80504603F095FC3A46E9
:10B1900006F10801FFF706FD306100207FE62DE98A
:10B1A000FF4F87B081461C469246DDF860B0DDF85F
:10B1B0005480089800F0F2F8050002D02878400783
:10B1C00002D401200BB09CE5484603F075FC2978B9
:10B1D000090605D56D49897A814201D88720F1E7B2
:10B1E000CAF309062A4601A9FFF7DCFC07461498B2
:10B1F00007281CD000222946FFF794FC0028E1D143
:10B200002878400613D501208DF808000898ADF87D
:10B210000C00BDF80400ADF80E00ADF81060ADF8FC
:10B22000124002A94846FAF7DBFC0028CAD1297867
:10B23000E87801F0030140EA0121AA78287902F0B8
:10B24000030240EA0220564507D0B1F5007F04D939
:10B25000611E814201DD0B20B4E7864201D907203F
:10B26000B0E7801B85B2A54200D92546BBF1000F8F
:10B2700001D0ABF80050179818B1B9192A4600F060
:10B28000CCF8B8F1000F0DD03E4448464446169F16
:10B2900003F08BFD2146FF1DBCB232462B460094C5
:10B2A00003F0B7F900208DE72DE9F04107461D4670
:10B2B0001646084600F072F8040002D020784007D5
:10B2C00001D40120D3E4384603F0F6FB21780906C7
:10B2D00005D52E49897A814201D88720C7E42246C4
:10B2E0003146FFF75FFC65B12178E07801F003019A
:10B2F00040EA0120B0F5007F01D8012000E00020E5
:10B3000028700020B3E42DE9F04107461D4616469B
:10B31000084600F043F8040002D02078400701D42A
:10B320000120A4E4384603F0C7FB2178090605D5BF
:10B330001649897A814201D8872098E4224631460D
:10B34000FFF75EFCFF2D14D02178E07801F00302B6
:10B3500040EA022040F20122B0FBF2F302FB1300AC
:10B3600015B900F2012080B2E070000A60F301011B
:10B37000217000207BE410B50C4600F00FF810B1EE
:10B380000178490704D4012010BD0000AC0400205E
:10B39000C18821804079A0700020F5E70749CA885C
:10B3A000824209D340B1096800EB40006FF00B0204
:10B3B00002EB80000844704700207047AC04002076
:10B3C00070B504460D4621462B460AB9002070BDD3
:10B3D00001E0491C5B1C501E021E03D008781E7839
:10B3E000B042F6D008781E78801BF0E730B50C46E6
:10B3F00001462346051B954206D202E0521E9D5C83
:10B400008D54002AFAD107E004E01D780D70491C24
:10B410005B1C521E002AF8D130BDF0B50E46014625
:10B42000334680EA030404F00304B4B906E002B929
:10B43000F0BD13F8017B01F8017B521E01F00307F8
:10B44000002FF4D10C461D4602E080CD80C4121FAF
:10B45000042AFAD221462B4600BF04E013F8014B20
:10B4600001F8014B521E002AF8D100BFE0E7F0B509
:10B470000C460146E6B204E002B9F0BD01F8016BEA
:10B48000521E01F00307002FF6D10B46E5B245EA44
:10B49000052545EA054501E020C3121F042AFBD219
:10B4A000194602E001F8016B521E002AFAD100BFD2
:10B4B000E3E710B507F009FBF7F74AFC07F0B0F92E
:10B4C000BDE8104007F042BA202801D201207047A1
:10B4D0000020704701224FF0A043824011B1C3F811
:10B4E0000C257047C3F8082570474FF0A041012292
:10B4F0008240C1F81825704770B503460020024607
:10B500006FF02F050EE09C5CA4F130060A2E02D3EA
:10B510004FF0FF3070BD00EB800005EB4000521C87
:10B520002044D2B28A42EED370BD30B50A230BE07C
:10B53000B0FBF3F403FB1404B0FBF3F08D183034CC
:10B54000521E05F8014CD2B2002AF1D130BD30B5FF
:10B5500000234FF6FF7510E0040A44EA002084B28D
:10B56000C85C6040C0F30314604005EA0034444006
:10B57000E0B25B1C84EA40109BB29342ECD330BD36
:10B5800070B514460B880122A240134207D1134321
:10B590000B8001230922011D03F069F9047070BDBD
:10B5A0002DE9FF4F81B00878DDE90E7B9A46914680
:10B5B0000E4640072CD4019803F0F7FB040000D19D
:10B5C000FFDF07F1040820461FFA88F102F054FD5E
:10B5D000050000D1FFDF204629466A4602F09FFFA2
:10B5E0000098A0F80370A0F805A0284603F045F8DD
:10B5F000017869F306016BF3C711017020461FFA49
:10B6000088F102F07CFD00B9FFDF019801F030FE07
:10B6100006EB0900017E491C017605B0BDE8F08FFC
:10B620002DE9F84F0E469A4691460746032103F04E
:10B6300079FA0446808CDFF8AC85002518B198F8BB
:10B640000000B0421ED1384603F0AFFB070000D126
:10B65000FFDF09F10401384689B202F00DFD050053
:10B6600010D0384629466A4602F059FF009800215A
:10B670000A460180817001F06AFE0098C01DCAF878
:10B68000000021E098F80000B04216D104F1220732
:10B6900034F8301F012000FA06F911EA090F00D032
:10B6A000FFDF2088012340EA090020800922391D9C
:10B6B000384603F0F7F8067006E0324604F1300130
:10B6C00004F12200FFF75CFF092188F800102846EA
:10B6D000BDE8F88FFEB515460C46064602AB0C22B7
:10B6E0000621FFF79DFF002827D0029960781222DB
:10B6F0000A70801C487008224A80A070029829882D
:10B70000052381806988C180A9880181E9884181F8
:10B7100000250C20CDE90005062221463046FFF722
:10B720003FFF2946002266F31F41F023104606F032
:10B7300081FF6078801C60700120FEBD10B504465A
:10B74000032103F0EFF9014600F110022046BDE8A5
:10B750001040BFE72DE9FE438146507816468846E3
:10B7600040B1FFDF3168C8F804107168C8F80810EC
:10B77000BDE8FE83B778022417B1022F13D0FFDF94
:10B78000251D2A4602AB07214846FFF749FF00283E
:10B79000E8D002980121022F017031784170448075
:10B7A000878002D005E00624EAE7B188C180F188ED
:10B7B00001810024CDE90054052307224146484673
:10B7C000FFF7EEFE88F80440D2E710B504460321E7
:10B7D00003F0A8F90146021D2046BDE81040B9E774
:10B7E0002DE9F0410E46054686B0144650880321E7
:10B7F00003F098F900218DF80010042E17D36A7811
:10B80000002A14D02B7802274FF6FF78012B2AD07C
:10B81000122B01D0132B0DD00391049169788DF870
:10B820000C106388014603AA1846FFF793FF06B081
:10B83000BDE8F08183789342F9D102781307F6D5F9
:10B84000062EF4D122F008020270608860F31F41D6
:10B85000002006F099FF8DF80070ADF80280A888EE
:10B86000ADF8040017E0062EE1D383789342DED1D1
:10B8700002781307DBD522F008020270608860F3BB
:10B880001F41002006F080FF8DF80070A888ADF8F9
:10B890000200ADF80480608822466946F6F740FB56
:10B8A000C5E7D04A002009211170704770B50C46D9
:10B8B0001546342200212046FFF7D9FD0120607093
:10B8C0000922002104F11800FFF7D1FD05B9FFDFBF
:10B8D0002978207861F30100207070BD7047002145
:10B8E00010B560F31F41002006F04EFF002010BD90
:10B8F000FEB506460F0CFCF7F9FA050007D06F807D
:10B900000321384603F00EF9040008D106E003B025
:10B910003846BDE8F0401321F6F7C8BEFFDF0EB190
:10B92000FFDFFEBD20782A4620F0080020700220AC
:10B930008DF800004FF6FF70ADF80200ADF804007E
:10B9400069463846F6F7ECFAFEBD00B5FFDF002089
:10B9500000BD2DE9FC410C461E46174680460321DA
:10B9600003F0E0F80546092C0AD2DFE804F00505EB
:10B970000505050509090700042303E0062301E086
:10B98000FFDF0023CDE90076224629464046FFF737
:10B9900007FEBDE8FC8138B50546A0F57F40FF38BD
:10B9A0001CD0284603F0EFF9040000D1FFDF204649
:10B9B00002F093FD002810D001466A46204602F0AE
:10B9C000AEFD00980321B0F80540284603F0AAF820
:10B9D000052C03D1007908B1002038BD012038BD05
:10B9E000F8B50446408803F0CEF9050000D1FFDF2A
:10B9F0006A462846616800F0E5F801460098091F8C
:10BA00008BB230F8032F028042884280018899422D
:10BA10000CD1042A0BD0052A19D0062A06D1636856
:10BA200064880A46011D2046F7F742FEF8BD001D56
:10BA30000E460546014622463046F9F7CAFB08285D
:10BA4000F4D1224629463046FAF737FCF8BD2246A3
:10BA5000001DFFF7C5FEF8BD70B50D460646032173
:10BA600003F060F8040004D02078000704D511200A
:10BA700070BD43F2020070BD2A4621463046FFF7F2
:10BA800029FE18B92868206168686061207840F054
:10BA900008002070002070BD2DE9F04F0E4691B0D7
:10BAA0008046032103F03EF80446404603F07DF94A
:10BAB00007460020079008900990ADF830000A90E2
:10BAC00002900390049004B9FFDF0DF10809FFB95B
:10BAD000FFDF1DE038460BA9002202F0C1FB9DF8F4
:10BAE0002C0000F07F05092D00D3FFDF6019017ED7
:10BAF000491E01769DF82C00000609D52A460CA99E
:10BB000007A8FFF73DFD19F80510491C09F80510B5
:10BB1000761EF6B2DED204F13000324D04F1220B73
:10BB2000DFF8C4A004F12607069010E058460699F5
:10BB300000F04AF806462870092800D3FFDF5AF8BB
:10BB4000261040468847608CC05DB04202D0A08C71
:10BB50000028EBD109202870234D4E4624350EE0F5
:10BB60000CA907A800F030F80446375D55F824000A
:10BB700000B9FFDF55F82420394640469047BDF80C
:10BB80001E000028ECD111B048E510B5032102F0E9
:10BB9000C9FF040000D1FFDF0922002104F11800D1
:10BBA000FFF765FC207840F00400207010BD10B550
:10BBB0000C46032102F0B6FF2044007E002800D08E
:10BBC000012010BD02F0ABBC10B50C4601230922C8
:10BBD000011D02F082FE00782188012282409143FB
:10BBE000218010BD5C000020688C0100FE4A1378A3
:10BBF00082F88730A2F8880082F88610012082F847
:10BC0000840092F8600008B192F85C0082F88A0023
:10BC1000704710B50B46114658B11846FFF7E6FFBE
:10BC2000F2488068008803F0AEF8BDE8104002F0EA
:10BC300063BDBDE810404FF6FF70D7E770B5002632
:10BC400004464670E94D1120207029682022A01C6E
:10BC50006431FFF7E2FB0121A171286800F8626FEF
:10BC60008078002811D1E048B0F86620A0F88E2036
:10BC7000AA68537B80F8903080F88C10108803F00D
:10BC800082F8BDE8704002F046BD70BDD74910B5DE
:10BC9000096891F892300022012B0DD091F88C3078
:10BCA000012B18D091F86230012B1ED091F884300E
:10BCB000012B1DD0002010BD42701623037051F8D7
:10BCC000933FC0F802304B68C0F806300B7A83729D
:10BCD00001F8012C1BE0427005230370D1F88E306F
:10BCE000C0F8023081F88C2011E0FFF7A7FF0EE0CA
:10BCF00091F86230012BF8D042701323037051F891
:10BD0000863FC0F802308B88C38001F8022C0120E6
:10BD100010BDB648006890F8621011B1B0F8660026
:10BD200070474FF6FF70704770B5B04C206800B98F
:10BD3000FFDF2068417811B10C25284670BD002531
:10BD40009C222946FFF793FB2168FF2008707F2083
:10BD500081F8360013204884282081F861000120F2
:10BD600081F85800002081F85B0007F0C3FA06F064
:10BD70007FFDE2E770B59D4C0546206800B9FFDF06
:10BD80002168002048706560FFF7CEFF002800D0D2
:10BD9000FFDF70BD954909680978814201D1012012
:10BDA000704700207047914800B5016891F8240061
:10BDB000498CC0F38002C0F340031A4400F0010034
:10BDC0001044102908D012290DD013290BD01529A1
:10BDD00004D0FFDF002000BD854901E0844908311F
:10BDE00031F8100000BD82490839F9E77F4840F278
:10BDF00071210068806A484370477C48006890F869
:10BE00003500002800D00120704710B5764C207B0B
:10BE100000F049FD40B1207D04F115010BF032FA2C
:10BE2000082801D0012010BD207B30B1022804D0A9
:10BE30000120BDE8104007F0CABD0020F9E76A49BB
:10BE4000087370476949096881F83000704770B518
:10BE50000646654890F82D000BF0A2F9050018D0B1
:10BE6000102100F068FF002813D1604C01203246F9
:10BE70002168C87628461C3107F0B6FDD4E90010C9
:10BE80001C310BF02BFB6068BDE8704001210BF00A
:10BE900034BB70BD2DE9F041534C074694F82D009A
:10BEA0000BF0FBF9064694F82F0004F10E0528B1BB
:10BEB00026B194F82D000BF016F9A0B194F83000DB
:10BEC000002824D094F82E00002820D0607B29463A
:10BED00000F0FAFCA8B10BF088FA3A462946BDE812
:10BEE000F04107F081BD012060733A462946304693
:10BEF00007F07AFD94F82D102846BDE8F0410BF0CC
:10BF000063BA39462846BDE8F04107F0A2BDBDE856
:10BF1000F08170B5354C2168087BB0B1022814D08F
:10BF2000012048730E3107F03CFD2068007B00F0D3
:10BF3000BAFC216881F82F00082081F82D00487B89
:10BF40000E3100F0B8FC40B901E00020E9E72168BB
:10BF5000487B0E3100F0B8FC00B10120216881F867
:10BF60002E0091F82F0018B991F82200400706D54D
:10BF7000087D15310BF086F9216881F82D002068C5
:10BF80000025456004F043FF216888600020FFF72A
:10BF900081FF2068C57690F82200400703D5BDE8F0
:10BFA0007040002053E770BD104A1268137B037085
:10BFB000D2F80E000860508A8880704778B50A4928
:10BFC00004460A4D407B08732A6820781070608808
:10BFD000ADF8000080B200F00101C0F3400341EA77
:10BFE0004301C0F3800305E0B80400206000002096
:10BFF000C08C010041EA8301C0F3C00341EAC301E0
:10C00000C0F3001341EA0311C0F3401341EA4311A6
:10C01000C0F3801041EA80105084E07D012825D0D3
:10C02000022825D0FFDF286880F85A60217B80F83D
:10C030002410418C1D291DD061688162617D80F8CA
:10C040003510A17BC1B1022916D00121017554F828
:10C050000F1FC0F81510A188A0F81910217B012925
:10C0600000D0002180F83410002078BD0126DAE7E6
:10C070000226D8E70021E0E70021E7E7FA48006858
:10C0800090F82200C0F38000704700B5FFF7F6FF7C
:10C0900008B1002000BD1F2000BD00B5FFF7F5FF6F
:10C0A000002800D0012000BDEF4900220968CA65C0
:10C0B0004B8C1D2B02D081F86000704781F8602006
:10C0C0007047E94A0023126882F8593042F8481F45
:10C0D0009080012050747047E34A0023126882F870
:10C0E0005830A2F8540042F8501F012010727047D7
:10C0F000DD49096881F85B007047DB48006890F90A
:10C100005B007047D848006890F8220000F00100FA
:10C110007047D548006890F82200C0F3400070478F
:10C1200000207047D048006890F82200C0F3C0009B
:10C13000704701207047012070470120704770B59B
:10C1400000F0D6FBC84C2068C16D491CC16590F851
:10C150003300002530B107F0CDF806F089FB2068E8
:10C1600080F833502068457090F8371009B10220EC
:10C170001AE090F86010B1B1C06D814213D802206E
:10C1800008F0A0F8206890F82200C00704D0A0684A
:10C1900043220188012003E043224FF6FF71002073
:10C1A000BDE8704035E50020BDE8704008F08AB871
:10C1B00010B501280DD002280DD004280FD0FFDFC4
:10C1C000A948006890F85A10BDE81040252006F0F4
:10C1D000FABC252000E0262006F0D6FDF0E7272057
:10C1E000FAE702460020D30701D0CB0705D093071A
:10C1F00005D58B0703D402207047012070475207F2
:10C20000FCD54907FAD4042070472DE9F041964C3B
:10C2100086B0206800B9FFDF20684178E9BB01786B
:10C22000FF2942D0002580F83150A0F85650857083
:10C2300080F83750284606F0A7FF18228B49684639
:10C24000FFF7EBF8684606F093FF06F0C8FC20689D
:10C2500090F95B0006F088FD84481D3806F08AFDE1
:10C260008248203806F075FF606806F090FF20686D
:10C27000002190F82400FFF7B4FFFFF799FF206832
:10C2800080F82C5006F07AFF206890F85A100020B1
:10C2900006F034FE0F21052000E006E006F03BFD2D
:10C2A000206890F82E1051B902E00C2006B02EE65E
:10C2B00090F82F1019B990F8220040072BD504F000
:10C2C000A6FD804620684146806805F0A8FA684FC0
:10C2D000064690FBF7F007FB10604142404604F031
:10C2E0006AFA2168886096FBF7F04A681044486053
:10C2F0000AF0C4FF21684A6890420CD8C1E901588D
:10C300000120FFF7C7FD206890F82200400702D502
:10C310000120FFF79CFD2068417B0E3006F0EDFC0C
:10C32000206890F8581039B1B0F85410A0F84410B3
:10C33000016D016480F8585090F8591031B1B0F88F
:10C340004C108187816C816380F859500BF003F8A1
:10C35000032160680BF036F8216881F83300002073
:10C36000A4E74149886070472DE9F0413E4C0746FB
:10C37000002620683146C57E6068068000F0AFFA6E
:10C380002068408C132837D004DC102858D012289D
:10C3900004D153E0152838D01D2836D0FFDF00BF68
:10C3A00000F0B1FA2068418C1D2907D0152905D06D
:10C3B000B0F84420016C60680BF0A6F8206890F893
:10C3C0002C1090F82400FFF70CFF05463FB1FFF753
:10C3D000EFFE01224FF49671002006F032FE206835
:10C3E00090F82C10294380F82C1090F824208A43D0
:10C3F0004FF0010129D02DE0002160680BF042F8D8
:10C400000121606800F06BFACAE7012160680BF057
:10C4100039F80121606800F062FAD4E9001025B112
:10C420001C310BF05BF8012104E015310BF056F8DC
:10C430002068017D60680BF060F8B1E7062100E03C
:10C44000022160680BF01EF8AAE7428C1D2A11D069
:10C4500080F831104170418C132914D00DDC102963
:10C4600010D012290DD10EE060000020D08C010008
:10C4700040420F0080F82C60ECE7152903D01D29FD
:10C4800001D0FFDF43E590F85A20BDE8F0410121DB
:10C49000084606F06ABFFF4810B50068417841B908
:10C4A0000078FF2805D00021084600F03AFA002065
:10C4B00010BD00F01DFA0C2010BD2DE9F041F54D26
:10C4C0000446174628680E4690F8620000B1FFDF68
:10C4D0002968002F81F864704ED12088A1F8660089
:10C4E0006088A1F87C00A088A1F87E00E088A1F80F
:10C4F000800094F8510181F8820091F82F0020B15A
:10C50000487B0E3100F0E0F940B9296891F830001D
:10C5100060B1487B0E3100F0CEF938B12868D0F810
:10C520000E100167418AA0F8741003E028680767BD
:10C53000A0F874706968FF2E0878C0F380106076E8
:10C54000D1F80300C4F81A00B1F80710E18314D041
:10C55000296801F16A02C1F87600E08BA1F87A003F
:10C56000304669310AF0A3FE00B9FFDF286810F8F1
:10C57000691F41F002010170C9E42868C0F87670B3
:10C58000A0F87A70617E80F86910D4F81A1040F82B
:10C590006A1FE18B8180BAE470B5FFF7C3FDBD4C23
:10C5A000012538B13C22FF21A068FFF786FF2068F3
:10C5B00080F86250206890F82200C00704D0A0687C
:10C5C0003C220188012003E03C224FF6FF7100204D
:10C5D000FFF71FFB206880F8375070BDAD49096830
:10C5E00081F83200704770B5AA4C00252068417868
:10C5F000012905D0022901D0032933D0FFDF70BD06
:10C6000081780029FBD1418C102913D090F8330098
:10C6100020B106F01FF9402006F042FE206890F895
:10C620002210490710D490F83510012904D00329AD
:10C6300002D002E0002119E0102590F85A2045F0C0
:10C640000E01002006F091FE206890F8340008B139
:10C6500006F069FE0021962006F0C5FD2168022043
:10C66000487070BD81780029FBD18178BDE87040A9
:10C67000012000F056B962E510B5864C206890F8AC
:10C68000340008B100F060F9206890F8330018B168
:10C6900006F030FE06F0ECF807F015FF88B12068D0
:10C6A0004078022800D0FFDF0021012000F039F996
:10C6B00020684178002903D04078012800D0FFDFAE
:10C6C00010BDBDE810403AE510B50AF0DBFD0446A8
:10C6D0000AF08DFE38B120460AF062FD18B1102133
:10C6E00000F029FB08B1002010BD012010BD2DE98C
:10C6F000F047DFF8A0910E460746032809D0FFF760
:10C7000001FD0446D9F8000090F8320020B1012064
:10C7100003E0FFF7FEFC04460020804606F026FBFF
:10C720000546032F2BD0012734EA080453D0D9F84B
:10C7300000004C4690F8330068B10AF0F2FD30700A
:10C740000146FF2807D06068C01C0AF0C7FD30789A
:10C750000AF0F1FD054360680178C1F38012216899
:10C760000B7D9A4205D10622C01C1531FEF728FE2A
:10C7700038B100203178FF290BD0D8B903E0022767
:10C78000D2E70120F6E7206890F82D00884211D00A
:10C7900008E038B1616811F8030BC0F38010FFF7AF
:10C7A00093FF38B10020216891F82210490703D582
:10C7B000A0B910E00120F6E785B9374890F83500B8
:10C7C00008B1B84207D1616811F8030BC0F38010BB
:10C7D000FFF77AFF10B10020BDE8F0870120FBE7EA
:10C7E0002DE9F0412B4C07460025206840780228AF
:10C7F00000D0FFDF206890F8340008B100F0A4F802
:10C8000060680AF061FE06469FB106F080FA80B1CA
:10C8100060680AF099FE60B1062E0AD2DFE806F0E1
:10C8200009090903090600F0D2F801E000F09BF8BD
:10C8300000B90125206890F8330018B106F05AFDC0
:10C8400006F016F84DB107F03EFE20B100210120A0
:10C8500000F067F801E0FFF772FC206841780029DA
:10C8600006D04178012903D04078032800D0FFDFAB
:10C8700008E670B5074E05460C46306880780028FB
:10C8800010D106F054F903463068214690F85A203A
:10C89000284603E060000020B8040020BDE8704096
:10C8A00007F012BF70BD022803D0032801D000207A
:10C8B000704701207047012802D14879800901D0D2
:10C8C0000020704701207047012806D148790121D6
:10C8D000B1EB901F01D10120704700207047027812
:10C8E000202322F0200203EA41110A43027070471C
:10C8F00010B506F0C8FC06F0A6FC06F0F5FBBDE896
:10C90000104006F02CBC10B57A4C794960680AF0EA
:10C91000DFFD77480E38417B6068BDE810400AF0C3
:10C92000E3BD744A10B5126892F8313033B1508CBF
:10C930001D2800D1FFDFBDE8104000E4002902D12E
:10C94000BDE8104010E510BD10B56A4C20683630C7
:10C9500006F0F4FC18B921687F2081F83600BDE8A4
:10C96000104006F0D6BC38B5FF208DF80000012538
:10C9700069460520FFF7BBFE30B35E4C2068807827
:10C9800008BB6268A0681278417BC2F34012114074
:10C990004173012100F049F800229DF80010A068C1
:10C9A000FFF78BFD2068012100F8621F82788188E3
:10C9B0000120FFF72EF9216800204870FFF798FF4B
:10C9C000012007F07FFC00E00025284638BD38B57F
:10C9D000FF208DF80000012569460320FFF787FE40
:10C9E000444C002820681BD090F8341031B190F8E6
:10C9F000920018B99DF8000000F046F86068002128
:10CA0000018004210AF03EFDFFF77DFF2068828F40
:10CA1000816B60680AF088FD21680320487002E09D
:10CA2000807800B90025284638BD324B10B55A68C9
:10CA300052F80F4FC0F80E409488448294790475E0
:10CA4000D47944751489C48254894480948984803B
:10CA5000D489C48014698460147D0473547D04F007
:10CA60001F040476527D520980F8512180F8381055
:10CA700080F83910196891F8612080F83A2091F80F
:10CA80005B1080F83B1010BD70B51A4C0122216874
:10CA900081F892200A7881F89320FF280DD001F1C7
:10CAA000950294310AF003FC00B9FFDF206810F80A
:10CAB000941F41F0020101700CE060680278C2F33B
:10CAC000801281F89420D0F8032041F8952FB0F817
:10CAD00007008880256895F836009B357F2800D1AF
:10CAE000FFDF206810F8361F29707F21017070BDAC
:10CAF000C60400206000002010B50024C484448DCA
:10CB0000DB004C43B3FBF2F394FBF2F45B1C448573
:10CB10009BB203FB02F40385B4F5C84F01DD5B1E35
:10CB200003854FF4FA43B3FBF2F35B1CC385438CDC
:10CB300002EBC3035B1EB3FBF2F30384C38B4B43D3
:10CB4000B3FBF2F1C18310BD70B50546087B0E46FC
:10CB500000F01F0008730020687604463019007A40
:10CB600000F06FFA2919641C0875697EE4B2084464
:10CB70006876052CF2D3C0B2252800D9FFDF70BD3E
:10CB80000023C383428401EBC202521EB2FBF1F1C7
:10CB900001847047F0B56FF01F02010C02EA902586
:10CBA0001F24A1F5AA4054380DD0A1F5AA4055384C
:10CBB00009D0A1F52850AA3805D0A1F52A40AA38F5
:10CBC00001D0012000E00020002213465FF015078D
:10CBD00082EA0106F6431E43761C0ED005F00106DC
:10CBE000520842EAC63204F001065B086D08640888
:10CBF00043EAC6337F1EEBD2F0BD0020F0BD2DE925
:10CC0000F04101270446002500F1400651B10129F9
:10CC10004ED0022973D0032948D101463046BDE8E1
:10CC2000F04191E7782200213046FEF720FCB571F3
:10CC3000F57135737573F57335747571B576F57671
:10CC400086F83E70412086F83F00FE2086F873008B
:10CC500026883C2200212046FEF709FC24F8AE6B12
:10CC6000282004F8767C04F8757C04F8740C04F829
:10CC7000A17C4FF4486024F8AC0C6581A581E58166
:10CC8000258265822575E5752584A5776586A58647
:10CC900084F8D05084F8D15084F8A65084F8A95074
:10CCA00084F8C250C4F8BA50C4F8BE50BDE8F08150
:10CCB000A4F8CE5084F8C3506188FE480A46084460
:10CCC000B0FBF1F0A4F860004BF68030A4F86200ED
:10CCD000E3883046FFF710FF21463046FFF734FF68
:10CCE00005F0B2F920B1D4F80E00FFF753FF18B1E8
:10CCF00084F85051DAE702E084F85071D6E74188B1
:10CD0000B4F87C31B4F878213046BDE8F041F3E660
:10CD1000437E0BB1252B01D9122070472AB14B7BE2
:10CD20002BB1012B05D01F2070470020704700F069
:10CD3000F2B900F096B903E0425C0AB100207047F6
:10CD4000491EC9B2F8D20120704730B5134606E03B
:10CD5000CC18D51A14F8014C5B1E4455DBB2002BDD
:10CD6000F6D130BD70B50E468CB0144601461D4656
:10CD700010226846FFF7E9FF1022314604A8FFF7AA
:10CD8000E4FF68460AF0B4FD08A94FF010022846F7
:10CD90001CB1FFF7DAFF0CB070BDFEF73EFBFAE7FF
:10CDA00038B505460C46684606F0C8FA002820D07B
:10CDB0009DF900002072E17E617294F90A10002250
:10CDC000411A00D5494295F82D308B4210DCFF2BDB
:10CDD0000ED0E17A491CC9B2E17295F82E30994221
:10CDE00002D8A17A7F2903D1A0720020E07201222B
:10CDF000104638BD0C2813D00B2811D00D280FD0A9
:10CE00001C280DD01D280BD01E2809D01F2807D0A4
:10CE1000202805D0212803D0232801D000207047E6
:10CE20000120704710B5A2F10F030C293AD2DFE8B8
:10CE300001F006080D1215181C392437392772B372
:10CE400030E0072A30D0082A2ED02BE00C2A2BD035
:10CE50000B2A29D026E00D2A26D023E00C2B23D93B
:10CE600020E0103A0B2A1FD91CE0032B1CD990F8A4
:10CE70003600B8B11B2A17D914E0062A14D011E0E5
:10CE80001C2A11D01D2A0FD01E2A0DD01F2A0BD00C
:10CE9000202A09D0212A07D0232A05D002E003E066
:10CEA0000E2A01D0002010BD012010BD2DE9F04157
:10CEB0000C46054640F23677866805E003F0A7FF8A
:10CEC000394603F078FCA860284604F05BF9002896
:10CED000F4D08CB13046A96804F0A1FC00280BDD29
:10CEE0002044401EB0FBF4F707FB04F1304603F08A
:10CEF00062FCA8603846D9E60020D7E670B5044643
:10CF000090420BD2101B642800D2642025188D4259
:10CF100005D8042104F0B7FC08B1284670BD2046AE
:10CF200070BD11F00C0F19D04A074FF41671002A8A
:10CF300003DA00BF4FF0100201E04FF0400201DAC7
:10CF40004FF0960101F5BC71A0EB0103884202D9B4
:10CF500093FBF2F000E0002080B27047022904D079
:10CF60006FF00D0101EBD000F6E76FF00E0101EB61
:10CF70009000F1E70844184498300AB1042100E019
:10CF800000210844704701207047106848637047CB
:10CF9000C10701D001207047810701D502207047E9
:10CFA000400701D508207047002070472DE9F04167
:10CFB000054616468846012408460AF0B0FB074697
:10CFC00040460AF0AEFB0346FFF7E2FF0246384652
:10CFD000FFF7DEFF52EA000100D10024990700D1DB
:10CFE0000022B90700D1002095F83810914200D1F5
:10CFF0000022327095F83910814200D10020707003
:10D0000072B968B940460AF08EFBB5F84010401A74
:10D0100000B247F6FE71884201DC002800DC0024E3
:10D02000204643E610B540F6C4125410012903D03F
:10D03000022902D0FFDF02E008B1104610BD2046F1
:10D0400010BD552101EA5001401AC0B200F0330171
:10D05000332202EA9000084400EB101000F00F00A9
:10D060007047F0B50C7C8B7BCD7B5C404B7C0288A1
:10D070006B4044EA0324467E62400023D5B2120A84
:10D0800095FAA5F592FAA2F22D0E120E45EA0222A9
:10D0900002EB02125B1C2244DBB292B2032BEDD3F3
:10D0A00062402523B2FBF3F403FB1423837603F0E1
:10D0B000070701E0FFDB050001EBD3040125247A1B
:10D0C00005FA07F73C4201D0C3761AE05643320C0A
:10D0D000521CD2B2002403191B7D934213D30023A8
:10D0E0000E19367A05FA03F73E4201D0521ED2B22B
:10D0F00022B15B1CDBB2082BF4D306E003EBC401C6
:10D10000C1760020F0BDD21AD2B2641CE4B2052C64
:10D11000E1D31F20F0BDF0B5837E0C7E012504FB1A
:10D1200002322523B2FBF3F403FB142201EBD204F9
:10D13000827602F00703247A05FA03F31C4201D039
:10D14000C2761EE0437EB2FBF3F403FB1422521CB2
:10D15000D2B20023C418247D944214D30024CE18E4
:10D1600096F8086005FA04F73E4201D0521ED2B28A
:10D1700022B1641CE4B2082CF4D306E004EBC30132
:10D18000C1760020F0BD121BD2B25B1CDBB2052BB6
:10D19000E0D31F20F0BD00002DE9FC470C460646F9
:10D1A000694600F018FE002860D1FEF7B2FDB042DB
:10D1B0005CD02146304608F0A6FC28BB019D95F8BE
:10D1C000F400403518B9287F08B1012000E00020A4
:10D1D000814695F837004FF000084FF0010AA0B1E2
:10D1E00095F83800800710D584F8018084F800A0F5
:10D1F00084F80280A68095F83910A171698F218189
:10D20000A98F618185F837802DE0304601F0CDFD92
:10D21000070000D1FFDF384600F0FBFF40B184F883
:10D2200001800D212170A680E08084F802A01AE020
:10D23000304601F0A8FD070000D1FFDFB9F1000F73
:10D2400014D0384601F03DF880B1304606F024FB9A
:10D2500084F801800A21217084F80280A680697F09
:10D26000A17185F81C800120BDE8FC870020FBE748
:10D270001CB5694600F0AFFD00B1FFDF684600F065
:10D28000B7FDF84900208968A1F8BA001CBD2DE956
:10D29000FC4104460E46062001F0F0FB002507463F
:10D2A000A846064417E02088401C80B22080B04287
:10D2B00002D34046A4F8008080B2B84204D3B04202
:10D2C00002D20020BDE8FC81694600F084FD002800
:10D2D000F8D06D1CEDB2AE42E5D84FF6FF7020805D
:10D2E0001220EFE710B506F049FB09F006FFDE4813
:10D2F0004FF6FF7100224181818102700321817309
:10D30000C17381700423C3701B238380C380018198
:10D31000827410BD70B5D34C0D466060217006F06C
:10D32000B9FA00F071FDFFF7DDFF207809F0A8F9E8
:10D33000284607F03EF8CC482838FEF71BFD217838
:10D34000606808F096FCBDE8704009F0D6BE10B5E4
:10D3500001240AB1002010BD21B1012903D000240D
:10D36000204610BD02210AF01FF9F9E7887800B9BC
:10D370000320C97801B9032110701970002070478B
:10D3800030B587B004460088694600F024FD0028C7
:10D3900006D1A08830B1012804D0022802D0122082
:10D3A00007B030BD05AB04AA21466846FFF7DEFF93
:10D3B0000400F5D10199012081F87F01019991F8CC
:10D3C000AE11002539B9019991F87E1119B9019969
:10D3D00091F8651009B13A2415E00199039581F897
:10D3E0007E0101989DF8102080F88021019B9DF816
:10D3F000140083F881018DF80C208DF80D0003AA2C
:10D400000120FFF7C2FD019880F87F512046C7E751
:10D4100010B504460020A17801B90120E2780AB9CC
:10D4200040F0020000F004FD002803D12046BDE8D2
:10D430001040A5E710BD10B50446FEF727FC0028F4
:10D4400013D0207813280FD1A07868B1A0880621C6
:10D4500001F068FB40B1008806F01EFAA0880621A2
:10D4600001F072FB00B1FFDF012010BD2DE9F0419A
:10D47000060000D1FFDF7C4802210C308046FFF718
:10D4800006FF00B1FFDF784C0620A78901F0F6FA0D
:10D490000546A089A84203D13046FFF7CCFF20B94A
:10D4A000A0893146FFF778FE38B1304600F0D0FC55
:10D4B0000028EED10120BDE8F08102214046FFF7AF
:10D4C000E6FE10B9A089B842E3D10020F3E710B519
:10D4D00000F062FC08B10C2010BD09F049FE0020EC
:10D4E00010BD10B50446007818B1012801D01220F3
:10D4F00010BD00F05CFC20B109F0B0FE08B10C20BA
:10D5000010BD207800F032FCE21D04F11703611C0D
:10D51000BDE8104009F04EBE10B5044600F03CFCDA
:10D5200008B10C2010BD207818B1012801D01220BC
:10D5300010BD00F01BFC611C09F0F4FD08B10020D7
:10D5400010BD072010BD10B509F08CFE08B10020F9
:10D5500010BD302010BD10B5044600F028FC08B105
:10D560000C2010BD204609F075FE002010BD10B53E
:10D5700000F01DFC20B109F071FE08B10C2010BDB7
:10D5800009F05AFE002010BDFF2181704FF6FF7197
:10D590008180344949680A7882718A880281498881
:10D5A000418101214170002070471CB50024022AEE
:10D5B00019D015DC12F10C0F15D009DC12F1280F6F
:10D5C00011D012F1140F0ED012F1100F0FD10AE08A
:10D5D00012F1080F07D012F1040F04D03AB902E09B
:10D5E000D31E052B03D8012804D0032806D012240B
:10D5F00020461CBD1046FEF77BFDF9E708461446A1
:10D60000694600F0E8FB08B10224F1E7019880F8D0
:10D610003B400024ECE710B513460122FFF7A2FBC4
:10D62000002010BD10B5044600F0C1FB08B10C206D
:10D6300010BD2146002006F0A2F9002010BD10B553
:10D64000044607F066F820B1207806F0BEFE002000
:10D6500010BD0C2010BD10B5044600F0A8FB28B189
:10D660000C2010BD6C0000207C050020214601200C
:10D6700006F085F90020F4E738B504464FF6FF7050
:10D68000ADF80000A079E179884216D02079FDF745
:10D690001BFF90B16079FDF717FF70B10022A079F0
:10D6A00011460AF0D9FB40B90022E07911460AF090
:10D6B000D3FB10B9207A072801D9122038BD07F012
:10D6C00034F848B900216846FFF7E1FD20B1204653
:10D6D00005F050FA002038BD0C2038BD2DE9FC4182
:10D6E000817804461A2925D00EDC16292DD2DFE8D0
:10D6F00001F02C2C2C2C2C212C2C2C2C2C2C2C2CDC
:10D700002C2C2C2C2C2121212A291ED00BDCA1F120
:10D710001E010C2919D2DFE801F018181818181882
:10D7200018181818180D3A3904290ED2DFE801F03C
:10D730000D020D022088B0F5706F06D201276946F0
:10D7400000F049FB18B10220BCE51220BAE5019DAA
:10D7500068462E4605F5AA7506F2551600F02EFB12
:10D7600008B1287808B10C20ACE52F70A078307093
:10D77000684600F03DFB0020A4E51CB50C46694658
:10D7800000F029FB002118B12160217102201CBD8D
:10D790000198024610F1400080F840109368236021
:10D7A000137B237190F84030002BF5D100201CBD75
:10D7B00010B5044600F0FBFA20B109F04FFD08B1A6
:10D7C0000C204EE7207800F0D1FAE279611C09F0D4
:10D7D0001AFE08B1002044E7022042E71CB50C46BF
:10D7E000694600F0F8FA002805D10198B0F8400029
:10D7F000401C208000201CBDF0B544888188C28870
:10D80000038945898089A71F40F67B46B74215D218
:10D810008F1FB74212D28C4210D8B2F5FA7F0DD2C8
:10D82000A3F10A04361FB44208D2521C4A43B2EB99
:10D83000830F03DA854201D80020F0BD3020F0BD0F
:10D84000F8B515460E46044606F06FFF08B10C20E9
:10D85000F8BD204600F027FB0028F9D1A078C106CA
:10D860004FF01100F4D5E17D0329F1D0FEF745FC1E
:10D870003070A07555B9FF208DF800006946002072
:10D88000FEF72AFC69460020FEF71BFC2046BDE897
:10D89000F840FEF793BB0022D2E70078C10801D020
:10D8A00012207047FA4988740020704710B504466A
:10D8B0000078C00704D1608810B1FEF7EEFB80B19C
:10D8C0002078618800F00102607800F037FB0028C2
:10D8D00006D1FEF7DAFB01466088884203D90720AB
:10D8E000BFE61220BDE66168FEF7F6FB0020B8E651
:10D8F00010B504460078C00704D1608810B1FEF767
:10D9000008FC70B12078618800F00102607800F0B6
:10D9100015FB002804D160886168FEF7D2FB002067
:10D920009FE612209DE67CB50446407842250128FA
:10D9300008D8A078FEF72EFA20B120781225012809
:10D9400002D090B128467CBDFEF7ECFB20B1A08848
:10D950000028F7D08028F5D8FEF7EBFB60B160789F
:10D960000028EFD02078012808D006F085F804467A
:10D9700006F0F5FC002878D00C207CBDFEF745FAB7
:10D9800010B9FEF7CDFB60B306F0CFFE0028F3D14F
:10D99000FEF7BFF9A0F57F41FF39EDD1FEF7B9FAE7
:10D9A000A68842F210704643A079FEF77DFBFEF791
:10D9B000A9FBC0B10022062101A801F085F80400EE
:10D9C00051D0B448002184602046FFF718F9204662
:10D9D000FEF7C7FCFEF7AFFBAD4D58B1288901211A
:10D9E0000CE012207CBD3146002006F0F1FC88B32B
:10D9F000FFDF44E0FEF7A1FB0146288906F0A0FD09
:10DA00000146A0620022204606F039F8FEF793FB9B
:10DA100038B9FEF792FB024621460120FFF7B3FA20
:10DA2000D0B19B4A21460E320120FFF7AEFAE878CA
:10DA30000090AB78EA88A988208801F02FF900B11E
:10DA4000FFDF208805F027FF3146204606F0C0FCA6
:10DA500000B1FFDF13E008E00621BDF8040001F08B
:10DA600073F800B1FFDF09207CBD44B1208805F0C8
:10DA700013FF2088062101F067F800B1FFDF0020C6
:10DA80007CBD00214FE770B50D46062101F04AF834
:10DA9000040003D094F8570110B10AE0022070BDD1
:10DAA00094F84D00142801D0152802D194F898015B
:10DAB00008B10C2070BD1022294604F5AC70FDF7AA
:10DAC000ACFC012084F85701002070BD10B5062180
:10DAD00001F028F818B190F8571111B107E00220B1
:10DAE000BFE590F84D10142903D0152901D00C2062
:10DAF000B7E5022180F857110020B2E52DE9FC417D
:10DB00000D464BF680321221954213D895B16946E5
:10DB100000F061F900280CD1019EB41C4036278822
:10DB20002A4639463046FFF72BF82088B842F6D10E
:10DB3000002009E6084607E61CB504460088694649
:10DB400000F049F9002808D10199A378084691F816
:10DB50002C2040319A4201D10C201CBD7F220A7238
:10DB60008A720022CA72E17880F82D10217980F83B
:10DB70002E10A17880F82C1010461CBD1CB50C4648
:10DB8000694600F028F9002806D1019890F85C0059
:10DB900000B10120207000201CBD7CB50D4614464C
:10DBA000694600F018F9002805D1019890F82C007A
:10DBB000012801D00C207CBD019890F848102970F4
:10DBC00090F84900207000207CBD70B50D461646C7
:10DBD000062100F0A7FF18B381880124C38842887A
:10DBE00004EB4104AC4217D842F210746343A41012
:10DBF0006243B3FBF2F2521E94B24FF4FA729442B3
:10DC000000D91446A54200D22C46491C641CB4FB22
:10DC1000F1F24A43521E91B290F884211AB901E000
:10DC2000022070BD01843180002070BD10B50C460B
:10DC3000062100F077FF18B1022C03D9122010E55D
:10DC400002200EE514F0010180F8C510C4F3400273
:10DC500080F8C42004D090F8C21009B106F087FC07
:10DC60000020FEE40178B9B14178A9B141881B29AF
:10DC700012D381881B290FD3C18802290CD30449F0
:10DC80000268283941F82A2F406848600020704710
:10DC90007C0500206C0000201220F8E710B506F08B
:10DCA0000CFC0020DDE410B506F00AFC0020D8E4EE
:10DCB00070B514460A46064600250121104606F0B6
:10DCC0003FFC002800D8284605460121304600F0D8
:10DCD00054F806460121002000F04FF831180122C7
:10DCE00096318D4206D901F19600691AB1FBF0F028
:10DCF000401C82B22280002070BD10B5044600F0A6
:10DD000056F808B10C20ACE4601C09F069FB2078DF
:10DD100000F00100FEF796F80020A2E410B50446DA
:10DD2000062000F09DFE08B10C209AE42078C00780
:10DD300010D00022607811460AF08EF808B1122047
:10DD40008FE4A06808F0ADFA6078616808F0B2FA74
:10DD5000002086E4002008F0A4FA00210846F5E738
:10DD600010B5006804F0E0FE00207AE418B1022843
:10DD700001D001208BE7002089E710B5012904D0EC
:10DD8000022905D0FFDF20466BE4C000503001E0DF
:10DD900080002C3084B2F6E710B506F0C6FC20B146
:10DDA000FEF72BF808B101205BE4002059E410B520
:10DDB00006F0BBFC002800D0012052E4416891F835
:10DDC000F40091F85C1021B918B1042801D00120A9
:10DDD0005DE700205BE710B50C46062100F0A2FECF
:10DDE000606018B10120207000203AE4022038E47D
:10DDF000416891F8C220002A05D0002281F8C22093
:10DE0000406806F0B4BB42E708B54FF6FF70ADF8C6
:10DE1000000006E00621BDF8000000F095FE00B10C
:10DE2000FFDF00216846FFF732FA0028F2D008BD74
:10DE300070B514460546012200F094F8002806D17A
:10DE400021462846BDE87040002200F08BB870BD26
:10DE50001FB55D49897CC90702D10178172902D015
:10DE6000002004B007E44088ADF8000002A9FFF7E5
:10DE7000B2FF00B1FFDF039810F8341F8DF80210D5
:10DE800040788DF803000020ADF8040001B9FFDFF1
:10DE90009DF8030000B9FFDF6846FFF7B9FA00B14B
:10DEA000FFDF0120DDE738B504460078EF2841D8D0
:10DEB0006088ADF80000009800F061F888B36188D0
:10DEC000080708D4D4E90120824233D8202A31D36C
:10DED000B0F5804F2ED8207B18B307282AD8607B56
:10DEE00028B1012803D0022801D0032822D14A07F3
:10DEF00003D4022801D0032805D1A07B08B1012852
:10DF000018D1480707D4607D28B1012803D0022822
:10DF100001D003280ED1C806E07D03D5012809D120
:10DF200004E007E0012801D0032803D1E07E18B106
:10DF3000012801D0122038BD002038BD70B50C4634
:10DF40000546FF2904D8FEF7F6F818B11F2C01D9B1
:10DF5000122070BD2846FDF71DFF08B1002070BDDE
:10DF6000422070BD0AB1012200E00222024202D129
:10DF7000880802D109B1002089E6112087E680B225
:10DF8000C1060BD401071CD481064FEAC07101D52C
:10DF9000B9B900E099B1800713D410E0410610D45C
:10DFA00081060ED4C1074FEA807104D0002902DB3C
:10DFB000400704D405E0010703D4400701D4012041
:10DFC00065E6002063E600007C05002030B505888A
:10DFD00025F4004421448CB24FF4004194420AD20B
:10DFE000121B92B21B339A4201D2A94307E005F4F7
:10DFF0000041214303E0A21A92B2A94311430180D8
:10E0000030BD0844083050434A31084480B270475C
:10E0100070B51D4616460B46044629463046049AFE
:10E02000FFF7EFFF0646B34200D2FFDF28220021B0
:10E030002046FDF71CFA4FF6FF70A082283EB0B2D2
:10E0400065776080B0F5004F00D9FFDF618805F18A
:10E050003C00814200D2FFDF60880835401B343825
:10E0600080B220801B2800D21B2020800020A077B7
:10E0700070BD8161886170472DE9F05F0D46C188F0
:10E08000044600F12809008921F4004620F40048E4
:10E0900000F063FB10B10020BDE8F09F4FF0000AD4
:10E0A0004FF0010BB0450CD9617FA8EB0600401A78
:10E0B0000838854219DC09EB060000210580418003
:10E0C0001AE06088617F801B471A083F0DD41B2F20
:10E0D00000DAFFDFBD4201DC294600E0B9B2681A70
:10E0E0000204120C04D0424502DD84F817A0D2E7E6
:10E0F00009EB06000180428084F817B0CCE770B5C8
:10E10000044600F12802C088E37D20F400402BB1D2
:10E1100010440288438813448B4201D2002070BD12
:10E1200000258A4202D30180458008E0891A09044B
:10E13000090C418003D0A01D00F01FFB08E0637FA5
:10E1400000880833184481B26288A01DFFF73EFFA3
:10E15000E575012070BD70B5034600F12804C5883F
:10E16000808820F400462644A84202D1002018826C
:10E1700070BD98893588A84206D3401B75882D1A32
:10E180002044ADB2C01E05E02C1AA5B25C7F20442D
:10E190003044401D0C88AC4200D90D809C8924B1CC
:10E1A000002414700988198270BD0124F9E770B544
:10E1B000044600F12801808820F400404518208A98
:10E1C000002825D0A189084480B2A08129886A88C6
:10E1D0001144814200D2FFDF288869880026084464
:10E1E000A189884212D1A069807F2871698819B1FC
:10E1F000201D00F0C2FA08E0637F28880833184425
:10E2000081B26288201DFFF7E1FEA68126820120EF
:10E2100070BD2DE9F041418987880026044600F150
:10E220002805B94219D004F10A0800BF21F40040C2
:10E230002844418819B1404600F09FFA08E0637F06
:10E2400000880833184481B262884046FFF7BEFE5A
:10E25000761C6189B6B2B942E8D13046BDE8F0819A
:10E260002DE9F04104460B4627892830A68827F47B
:10E270000041B4F80A8001440D46B74201D10020A4
:10E28000ECE70AB1481D106023B1627F691D184692
:10E29000FDF7C3F82E88698804F1080021B18A19B6
:10E2A00096B200F06AFA06E0637F62880833991933
:10E2B00089B2FFF78BFE474501D120896081304646
:10E2C000CCE78188C088814201D1012070470020BD
:10E2D000704701898088814201D101207047002068
:10E2E000704770B58588C38800F1280425F4004282
:10E2F00023F4004114449D421AD08389058A5E1993
:10E3000025886388EC18A64214D313B18B4211D32D
:10E310000EE0437F08325C192244408892B2801A92
:10E3200080B22333984201D211B103E08A4201D175
:10E33000002070BD012070BD2DE9F0478846C188DE
:10E340000446008921F4004604F1280720F4004522
:10E3500007EB060900F001FA002178BBB54204D9A9
:10E36000627FA81B801A002503E06088627F801B03
:10E37000801A083823D4E28962B1B9F80020B9F8CC
:10E3800002303BB1E81A2177404518DBE089384478
:10E39000801A09E0801A217740450ADB607FE18915
:10E3A0000830304439440844C01EA4F81280BDE847
:10E3B000F087454503DB01202077E7E7FFE761822F
:10E3C0000020F4E72DE9F74F044600F12805C08846
:10E3D000884620F4004A608A05EB0A0608B14045E9
:10E3E00002D20020BDE8FE8FE08978B13788B6F808
:10E3F000029007EB0901884200D0FFDF207F4FF039
:10E40000000B50EA090106D088B33BE00027A07F4B
:10E41000B9463071F2E7E18959B1607F294408308B
:10E4200050440844B4F81F1020F8031D94F821103C
:10E430008170E28907EB080002EB0801E18130807E
:10E44000A6F802B002985F4650B1637F3088083367
:10E45000184481B26288A01DFFF7B8FDE78121E072
:10E46000607FE18908305044294408442DE0FFE7EB
:10E47000E089B4F81F102844C01B20F8031D94F84D
:10E480002110817009EB0800E28981B202EB0800DB
:10E49000E081378071800298A0B1A01D00F06DF975
:10E4A000A4F80EB0A07F401CA077A07D08B1E08842
:10E4B000A08284F816B000BFA4F812B084F817B098
:10E4C00001208FE7E0892844C01B30F8031DA4F821
:10E4D0001F10807884F82100EEE710B5818800F1E4
:10E4E000280321F400442344848AC288A14212D024
:10E4F000914210D0818971B9826972B11046FFF7DB
:10E50000E8FE50B91089283220F4004010441979EF
:10E510000079884201D1002010BD184610BD00F1DD
:10E520002803407F08300844C01E1060088808B9DE
:10E53000DB1E136008884988084480B270472DE9C3
:10E54000F04100F12806407F1C46083090464318F1
:10E5500008884D88069ADB1EA0B1C01C80B290428C
:10E5600014D9801AA04200DB204687B298183A4698
:10E570004146FCF725FF002816D1E01B84B2B844C1
:10E58000002005E0ED1CADB2F61EE8E7101A80B2DF
:10E590000119A94206D8304422464146BDE8F0415F
:10E5A000FCF70EBF4FF0FF3058E62DE9F04100F1C7
:10E5B0002804407F1E4608309046431800250888EE
:10E5C0004F88069ADB1E90B1C01C80B2904212D9CF
:10E5D000801AB04200DB304685B299182A46404680
:10E5E000FCF71BFF701B86B2A844002005E0FF1C4F
:10E5F000BFB2E41EEAE7101A80B28119B94206D808
:10E60000211832464046FCF708FFA81985B2284673
:10E6100024E62DE9F04100F12804407F1E46083031
:10E6200090464318002508884F88069ADB1E90B153
:10E63000C01C80B2904212D9801AB04200DB304632
:10E6400085B298182A464146FCF7E7FE701B86B251
:10E65000A844002005E0FF1CBFB2E41EEAE7101A40
:10E6600080B28119B94206D8204432464146FCF7AF
:10E67000D4FEA81985B22846F0E5401D704710B5B4
:10E68000044600F12801C288808820F40043194420
:10E69000904206D0A28922B9228A12B9A28A904257
:10E6A00001D1002010BD0888498831B1201D00F03B
:10E6B00064F800202082012010BD637F6288083347
:10E6C000184481B2201DFFF781FCF2E70021C181CF
:10E6D00001774182C1758175704703881380C289B3
:10E6E00042B1C28822F4004300F128021A440A60B1
:10E6F000C08970470020704710B50446808AA0F595
:10E700007F41FF3900D0FFDFE088A082E08900B1BF
:10E710000120A07510BD4FF6FF7181820021817527
:10E72000704710B50446808AA0F57F41FF3900D1BB
:10E73000FFDFA07D28B9A088A18A884201D10020EE
:10E7400010BD012010BD8188828A914201D1807D57
:10E7500008B1002070470120704720F4004221F4E6
:10E7600000439A4207D100F4004001F4004188427E
:10E7700001D0012070470020704730B50446008862
:10E780000D4620F40040A84200D2FFDF21884FF45C
:10E79000004088432843208030BD70B50C000546FA
:10E7A00009D0082C00D2FFDF1DB1A1B2286800F00B
:10E7B00044F8201D70BD0DB100202860002070BD00
:10E7C0000021026803E093881268194489B2002A84
:10E7D000F9D100F032B870B500260D46044608297C
:10E7E00000D2FFDF206808B91EE004462068818857
:10E7F000A94202D001680029F7D181880646A942C2
:10E8000001D100680DE005F1080293B2002299429F
:10E8100009D32844491B026081802168096821606E
:10E820000160206000E00026304670BD00230B60D0
:10E830008A8002680A600160704700234360021DFD
:10E84000018102607047F0B50F4601884088154687
:10E850000C181E46AC4200D3641B3044A84200D9B9
:10E86000FFDFA019A84200D9FFDF3819F0BD2DE95C
:10E87000F041884606460188408815460C181F4618
:10E88000AC4200D3641B3844A84200D9FFDFE01932
:10E89000A84200D9FFDF70883844708008EB04007C
:10E8A000BDE8F0812DE9F041054600881E46174677
:10E8B000841B8846BC4200D33C442C80688830448A
:10E8C000B84200D9FFDFA019B84200D9FFDF68883D
:10E8D0003044688008EB0400E2E72DE9F041068847
:10E8E0001D460446701980B2174688462080B842FB
:10E8F00001D3C01B20806088A84200D2FFDF7019BE
:10E90000B84200D9FFDF6088401B608008EB06003A
:10E91000C6E700002DE9F041BF4D04469046A878B7
:10E920000E46A04200D8FFDF05EB8607786A50F854
:10E93000240000B1FFDFB868002816D0304600F090
:10E9400032F90146B868FFF746FF05000CD0786A37
:10E95000072E40F8245000D3FFDFB0484246294636
:10E9600050F82630204698472846BDE8F0812DE92A
:10E97000F84305000C46009524D00026E81C20F042
:10E980000300A84200D0FFDFDFF88C820027314669
:10E9900088F8007088F8014088F8024088F8034041
:10E9A00088F8044088F8054088F80640684600F07A
:10E9B00003F9002042460099C91C21F0030100918F
:10E9C00016B10FE00126D9E702EB8003596200215E
:10E9D00006E000BFD3F824C04CF82170491CC9B22E
:10E9E000A142F7D30099401C01EB8401C0B2009111
:10E9F0000728E0D3481BBDE8F88310B50446F2F7BA
:10EA000050FC08B1102010BD2078834A618802EBC9
:10EA1000800092780EE0436A53F8213043B14A1CDB
:10EA20006280A180406A50F82100A060002010BDE3
:10EA3000491C89B28A42EED86180052010BD70B5AC
:10EA400005460C460846F2F72CFC08B1102070BDB4
:10EA5000072D01D3072070BD25700020608070BD98
:10EA60000EB56946FFF7EBFF00B1FFDF6846FFF721
:10EA7000C4FF08B100200EBD01200EBD10B5044634
:10EA8000072800D3FFDF6448005D10BD3EB5054692
:10EA900000246946FFF7D3FF18B1FFDF01E0641CD3
:10EAA000E4B26846FFF7A9FF0028F8D02846FFF730
:10EAB000E5FF001BC0B23EBD57498978814201D9AC
:10EAC000C0B27047FF2070472DE9F04106291BD1E5
:10EAD000514C00273B464FF6FF7604EB810514F8B6
:10EAE00001C00AE0DC19D5F824E0A4B25EF824E005
:10EAF000BEF1000F04D05B1C9BB29C45F2D834469B
:10EB000004802046B44201D100202EE7BDE8F04148
:10EB100000E7A0F57F43FF3B01D0072901D3002088
:10EB20007047F7E6A0F57F42FF3A0BD0072909D2DC
:10EB3000394A9378834205D902EB8101496A51F839
:10EB400020007047002070472DE9F04104460D4633
:10EB5000A4F57F4143F20200FF3902D0072D01D313
:10EB6000072002E72C494FF000088A78A242F8D922
:10EB700001EB8506726A52F82470002FF1D0274805
:10EB800039461C3050F8252020469047716A2846A7
:10EB900041F8248000F007F802463946B068FFF7D4
:10EBA00045FE0020E1E61D49383131F810004FF6EE
:10EBB000FC71C01C084070472DE9F843164E88468A
:10EBC000054600242868C01C20F003002860204669
:10EBD000FFF7E9FF315D4843B8F1000F01D0002293
:10EBE00000E02A680146009232B100274FEA0D008A
:10EBF000FFF7D3FD1FB106E001270020F8E706EB81
:10EC00008401009A8A602968641C0844E4B2286080
:10EC1000072CD7D3EFE6000090050020E88C010018
:10EC200070B50E461D46114600F0D3F8044629463D
:10EC3000304600F0D7F82044001D70BD2DE9F041AA
:10EC400090460D4604004FF0000610D00027E01C4F
:10EC500020F00300A04200D0FFDFE5B141460020D4
:10EC6000FFF79BFD0C3000EB850617B113E0012781
:10EC7000EDE7614F04F10C00AA003C602572606072
:10EC800000EB8500206000216068FCF7F0FB414646
:10EC90003868FFF782FD3046BDE8F0812DE9FF4F6F
:10ECA000554C804681B020689A46934600B9FFDFF4
:10ECB0002068027A424503D9416851F8280020B102
:10ECC00043F2020005B0BDE8F08F5146029800F013
:10ECD00080F886B258460E9900F084F885B2701913
:10ECE000001D87B22068A14639460068FFF773FD12
:10ECF00004001FD0678025802946201D0E9D0746F1
:10ED00005A4601230095FFF783F92088314638449D
:10ED10000123029ACDF800A0FFF77AF92088C119E3
:10ED20003846FFF7A6F9D9F800004168002041F8FD
:10ED30002840C7E70420C5E770B52F4C054620687A
:10ED400000B9FFDF2068017AA9420DD9426852F864
:10ED5000251049B1002342F825304A880068FFF7A2
:10ED600065FD2168087A06E043F2020070BD4A683A
:10ED700052F820202AB9401EC0B2F8D20868FFF726
:10ED80001FFD002070BD70B51B4E05460024306885
:10ED900000B9FFDF3068017AA94204D9406850F811
:10EDA000250000B1041D204670BD70B5124E054609
:10EDB0000024306800B9FFDF3068017AA94206D923
:10EDC000406850F8251011B131F8040B4418204662
:10EDD00070BD10B50A460121FFF713F9C01C20F0E1
:10EDE000030010BD10B50A460121FFF70AF9C01C47
:10EDF00020F0030010BD00007800002070B504462C
:10EE0000C2F110052819FCF708FB15F0FF0109D025
:10EE1000491ECAB28020A0542046BDE8704000219F
:10EE2000FCF725BB70BD30B505E05B1EDBB2CC5CEA
:10EE3000D55C6C40C454002BF7D130BD10B5002414
:10EE400009E00B78521E44EA430300F8013B11F835
:10EE5000013BD2B2DC09002AF3D110BD2DE9F04309
:10EE600089B01E46DDE9107990460D00044622D097
:10EE700002460846F949FEF7CEFB102221463846E5
:10EE8000FFF7DCFFE07B000606D5F44A3946102385
:10EE900010320846FFF7C7FF102239464846FFF7F1
:10EEA000CDFFF87B000606D5EC4A49461023103208
:10EEB0000846FFF7B8FF102200212046FCF7D7FADA
:10EEC0000DE0103EB6B208EB06011023224668465C
:10EED000FFF7A9FF224628466946FEF79CFB102E45
:10EEE000EFD818D0F2B241466846FFF787FF1023EB
:10EEF0004A46694604A8FFF796FF1023224604A954
:10EF00006846FFF790FF224628466946FEF783FBD6
:10EF100009B0BDE8F08310233A464146EAE770B5F0
:10EF20009CB01E460546134620980C468DF80800F6
:10EF3000202219460DF10900FCF76FFA2022214624
:10EF40000DF12900FCF769FA17A913A8CDE9000112
:10EF5000412302AA31462846FFF780FF1CB070BD4E
:10EF60002DE9FF4F9FB014AEDDE92D5410AFBB4922
:10EF7000CDE90076202320311AA8FFF76FFF4FF06C
:10EF800000088DF808804FF001098DF8099054F8B9
:10EF9000010FCDF80A00A088ADF80E0014F8010C9E
:10EFA0001022C0F340008DF8100055F8010FCDF885
:10EFB0001100A888ADF8150015F8010C2C99C0F3C4
:10EFC00040008DF8170006A88246FCF726FA0AA82A
:10EFD000834610222299FCF720FAA04835230838EE
:10EFE00002AA40688DF83C80CDE900760E901AA9FF
:10EFF0001F98FFF733FF8DF808808DF8099020687F
:10F00000CDF80A00A088ADF80E0014F8010C10220B
:10F01000C0F340008DF810002868CDF81100A888D2
:10F02000ADF8150015F8010C2C99C0F340008DF8CF
:10F0300017005046FCF7F1F9584610222299FCF7C8
:10F04000ECF986483523083802AA40688DF83C90D0
:10F05000CDE900760E901AA92098FFF7FFFE23B0A5
:10F06000BDE8F08FF0B59BB00C460546DDE92210F7
:10F070001E461746DDE92032D0F801C0CDF808C0A1
:10F08000B0F805C0ADF80CC00078C0F340008DF8B2
:10F090000E00D1F80100CDF80F00B1F80500ADF871
:10F0A000130008781946C0F340008DF81500108849
:10F0B000ADF8160090788DF818000DF119001022A7
:10F0C000FCF7ABF90DF1290010223146FCF7A5F948
:10F0D0000DF1390010223946FCF79FF917A913A842
:10F0E000CDE90001412302AA21462846FFF7B6FEDA
:10F0F0001BB0F0BDF0B5A3B017460D4604461E4642
:10F10000102202A82899FCF788F906A8202239467F
:10F11000FCF783F90EA820222946FCF77EF91EA9E8
:10F120001AA8CDE90001502302AA314616A8FFF71C
:10F1300095FE1698206023B0F0BDF0B589B0044666
:10F14000DDE90E070D463978109EC1F340018DF8B8
:10F15000001031789446C1F340018DF80110196810
:10F16000CDF802109988ADF8061099798DF808103D
:10F170000168CDF809108188ADF80D1080798DF8FF
:10F180000F0010236A46614604A8FFF74CFE224692
:10F19000284604A9FEF73FFAD6F801000090B6F819
:10F1A0000500ADF80400D7F80100CDF80600B7F867
:10F1B0000500ADF80A000020039010236A4621469E
:10F1C00004A8FFF730FE2246284604A9FEF723FADA
:10F1D00009B0F0BD1FB51C6800945B68019313680B
:10F1E000029352680392024608466946FEF713FAF4
:10F1F0001FBD10B588B00446106804905068059093
:10F2000000200690079008466A4604A9FEF703FA14
:10F21000BDF80000208008B010BD1FB51288ADF801
:10F2200000201A88ADF80220002201920292039277
:10F23000024608466946FEF7EEF91FBD7FB5074B4B
:10F2400014460546083B9A1C6846FFF7E6FF22462F
:10F2500069462846FFF7CDFF7FBD0000368D0100CF
:10F2600070B5044600780E46012813D0052802D058
:10F27000092813D10EE0A06861690578042003F025
:10F2800083FA052D0AD0782300220420616903F057
:10F29000D1F903E00420616903F076FA3146204693
:10F2A000BDE8704001F08AB810B500F12D03C279B5
:10F2B0009C78411D144064F30102C271D2070DD045
:10F2C0004A795C7922404A710A791B791A400A719D
:10F2D0008278C9788A4200D9817010BD00224A71B3
:10F2E000F5E74178012900D00C21017070472DE924
:10F2F000F04F93B04FF0000B0C690D468DF820B025
:10F30000097801260C2017464FF00D084FF0110A1E
:10F310004FF008091B2975D2DFE811F01B00C40269
:10F3200007031F035E037103A303B803F9031A0461
:10F3300062049504A204EF042D0537055505600508
:10F34000F3053606390668068406FE062207EB0634
:10F35000F00614B120781D282AD0D5F808805FEA7D
:10F3600008004FD001208DF82000686A02220D901D
:10F370008DF824200A208DF82500A8690A90A88815
:10F380000028EED098F8001091B10F2910D27DD24C
:10F39000DFE801F07C1349DEFCFBFAF9F8F73808E6
:10F3A0009CF6F50002282DD124B120780C2801D03C
:10F3B0000026F0E38DF82020CBE10420696A03F0F9
:10F3C000E3F9A8880728EED1204600F0F2FF0228D2
:10F3D00009D0204600F0EDFF032807D9204600F0B1
:10F3E000E8FF072802D20120207004E0002CB8D0EA
:10F3F00020780128D7D198F80400C11F0A2902D328
:10F400000A2061E0C4E1A070D8F80010E162B8F809
:10F410000410218698F8060084F832000120287034
:10F420000320207044E00728BDD1002C99D020781B
:10F430000D28B8D198F8031094F82F20C1F3C0001C
:10F44000C2F3C002104201D0062000E00720890765
:10F4500007D198F805100142D2D198F80610014260
:10F46000CED194F8312098F8051020EA020211421A
:10F47000C6D194F8322098F8061090430142BFD1CB
:10F4800098F80400C11F0A29BAD200E008E2617DA1
:10F4900081427CD8D8F800106160B8F8041021814E
:10F4A00098F80600A072012028700E20207003201A
:10F4B0008DF82000686A0D9004F12D000990601D00
:10F4C0000A900F300B9022E12875FCE3412891D17E
:10F4D000204600F06EFF042802D1E078C00704D176
:10F4E000204600F066FF0F2884D1A88CD5F80C8048
:10F4F00080B24FF0400BE669FFF745FC32464146CB
:10F500005B464E46CDF80090FFF74FF80B208DF884
:10F510002000686A0D90E0690990002108A8FFF7B3
:10F520009FFE2078042806D0A07D58B1012809D07C
:10F5300003280AD04AE305202070032028708DF8A4
:10F540002060CEE184F800A032E712202070EAE1CA
:10F550001128BCD1204600F02CFF042802D1E0780D
:10F56000C00719D0204600F024FF062805D1E07816
:10F57000C00711D1A07D02280ED0204608E0CCE0C3
:10F5800084E072E151E124E103E1E9E019E0B0E156
:10F5900000F00FFF11289AD1102208F1010104F1A7
:10F5A0003C00FBF73AFF607801286ED012202070F3
:10F5B000E078C00760D0A07D0028C8D00128C6D060
:10F5C0005AE0112890D1204600F0F3FE082804D01C
:10F5D000204600F0EEFE132886D104F16C001022C4
:10F5E00008F101010646FBF718FF207808280DD026
:10F5F00014202070E178C8070DD0A07D02280AD021
:10F600006278022A04D00328A1D035E00920F0E76F
:10F6100008B1012837D1C80713D0A07D02281DD01A
:10F6200000200090D4E9062133460EA8FFF777FCAE
:10F6300010220EA904F13C00FBF7C2FEC8B1042061
:10F6400042E7D4E90912201D8DE8070004F12C03DC
:10F6500032460EA8616BFFF770FDE9E7606BC1F3FE
:10F660004401491E0068C84000F0010040F08000DD
:10F67000D7E72078092806D185F800908DF82090EA
:10F6800036E32870EFE30920FBE79EE1112899D1CA
:10F69000204600F08EFE0A2802D1E078C00704D18F
:10F6A000204600F086FE15288CD104F13C00102283
:10F6B00008F101010646FBF7B0FE20780A2816D0B3
:10F6C00016202070D4E90932606B611D8DE80F00AF
:10F6D00004F15C0304F16C0247310EA8FFF7C2FC91
:10F6E00010220EA93046FBF76BFE18B1F9E20B2091
:10F6F000207073E22046FFF7D7FDA078216AC0F1A1
:10F7000010020B1800211846FBF7B1FE26E339461C
:10F7100008A8FFF7A5FD06463CE20228B7D120461F
:10F7200000F047FE042804D3204600F042FE0828DB
:10F7300009D3204600F03DFE0E2829D3204600F0D4
:10F7400038FE122824D2A07D0228A0D10E208DF8E8
:10F750002000686A0D9098F801008DF82400F5E308
:10F76000022894D1204600F024FE002810D0204624
:10F7700000F01FFE0128F9D0204600F01AFE0C28E8
:10F78000F4D004208DF8240098F801008DF82500AD
:10F7900060E21128FCD1002CFAD020781728F7D18C
:10F7A0006178606A022912D05FF0000101EB41012B
:10F7B000182606EBC1011022405808F10101FBF7A1
:10F7C0002CFE0420696A00F0E7FD2670F0E50121B7
:10F7D000ECE70B28DCD1002CDAD020781828D7D120
:10F7E0006078616A02281CD05FF0000000EB4002E4
:10F7F000102000EBC2000958B8F8010008806078BA
:10F80000616A02280FD0002000EB4002142000EBB8
:10F81000C2000958404650F8032F0A60406848600B
:10F8200039E00120E2E70120EEE71128B0D1002CF9
:10F83000AED020781928ABD16178606A022912D045
:10F840005FF0000101EB41011C2202EBC10110221B
:10F85000405808F10101FBF7E0FD0420696A00F05F
:10F860009BFD1A20B6E00121ECE7082890D1002C7E
:10F870008ED020781A288BD1606A98F80120017800
:10F8800062F347010170616AD8F8022041F8012F44
:10F89000B8F8060088800420696A00F07DFD90E2D7
:10F8A000072011E63878012894D1182204F11400B9
:10F8B0007968FBF7B2FDE079C10894F82F0001EAFE
:10F8C000D001E07861F30000E070217D002974D15F
:10F8D0002178032909D0C00725D0032028708DF88E
:10F8E0002090686A0D90412008E3607DA1788842ED
:10F8F00001D90620E8E502262671E179204621F0AB
:10F90000E001E171617A21F0F0016172A17A21F0E8
:10F91000F001A172FFF7C8FC2E708DF82090686A84
:10F920000D900720EAE20420ABE6387805289DD147
:10F930008DF82000686A0D90B8680A900720ADF82D
:10F9400024000A988DF830B06168016021898180B7
:10F95000A17A817104202070F8E23978052985D1D7
:10F960008DF82010696A0D91391D09AE0EC986E81F
:10F970000E004121ADF824108DF830B01070A88C25
:10F98000D7F80C8080B24026A769FFF70EFA4146EF
:10F990003A463346C846CDF80090FEF73AFE0021BD
:10F9A00008A8FFF75DFCE07820F03E00801CE070C6
:10F9B0002078052802D00F200CE04AE1A07D20B17C
:10F9C000012802D0032802D002E10720BEE584F816
:10F9D0000080EDE42070EBE4102104F15C0002F003
:10F9E000F4FB606BB0BBA07D18B1012801D00520ED
:10F9F000FDE006202870F8486063A063C2E2387812
:10FA0000022894D1387908B12875B7E3A07D02287F
:10FA100002D0032805D022E0B8680028F5D0606342
:10FA20001CE06078012806D0A07994F82E100128F7
:10FA300005D0E94806E0A17994F82E00F7E7B86808
:10FA40000028E2D06063E078C00701D0012902D02D
:10FA5000E14803E003E0F8680028D6D0A063062060
:10FA60000FE68DF82090696A0D91E1784846C90744
:10FA700009D06178022903D1A17D29B1012903D0E0
:10FA8000A17D032900D00720287033E138780528AC
:10FA9000BBD1207807281ED084F800A005208DF85F
:10FAA0002000686A0D90B8680A90ADF824A08DF81F
:10FAB00030B003210170E178CA070FD0A27D022A7D
:10FAC0001AD000210091D4E9061204F15C03401C15
:10FAD000FFF725FA6BE384F80090DFE7D4E9092308
:10FAE000211D8DE80E0004F12C0304F15C02401C82
:10FAF000616BFFF722FB5AE3626BC1F34401491EBD
:10FB00001268CA4002F0010141F08001DAE738785A
:10FB10000528BDD18DF82000686A0D90B8680A905C
:10FB2000ADF824A08DF830B0042100F8011B10229C
:10FB300004F15C01FBF771FC002108A8FFF790FBC2
:10FB40002078092801D0132044E70A2020709AE584
:10FB5000E078C10742D0A17D012902D0022927D037
:10FB600038E0617808A8012916D004F16C010091F1
:10FB7000D4E9061204F15C03001DFFF7BBFA0A206A
:10FB8000287003268DF82080686A0D90002108A84F
:10FB9000FFF766FBE1E2C7E204F15C010091D4E902
:10FBA000062104F16C03001DFFF7A4FA0026E9E723
:10FBB000C0F3440114290DD24FF0006101EBB010E5
:10FBC0004FEAB060E0706078012801D01020BDE4F9
:10FBD0000620FFE6607801283FF4B6AC0A2050E525
:10FBE000E178C90708D0A17D012903D10B20287035
:10FBF000042030E028702EE00E2028706078616BC1
:10FC0000012818D004F15C0304F16C020EA8FFF780
:10FC1000E1FA2046FFF748FBA0780EAEC0F11002D3
:10FC200030440021FBF723FC06208DF82000686A91
:10FC300009960D909BE004F16C0304F15C020EA8A0
:10FC4000FFF7C8FAE8E73978022903D139790029A2
:10FC5000D0D0297592E28DF82000686A0D9056E5A3
:10FC600038780728F6D1D4E909216078012808D02E
:10FC700004F16C00CDE90002029105D104F16C039E
:10FC800004E004F15C00F5E704F15C0304F14C00CE
:10FC90007A680646216AFFF763F96078012822D165
:10FCA000A078216AC0F110020B1800211846FBF75A
:10FCB000DEFBD4E90923606B04F12D018DE80F0010
:10FCC00004F15C0300E05BE204F16C0231460EA833
:10FCD000FFF7C8F910220EA904F13C00FBF770FBF6
:10FCE00008B10B20ACE485F8008000BF8DF82090AF
:10FCF000686A0D908DF824A009E538780528A9D107
:10FD00008DF82000686A0D90B8680A90ADF824A0BC
:10FD10008DF830B080F80080617801291AD0D4E9DC
:10FD2000092104F12D03A66B03910096CDE9013260
:10FD300004F16C0304F15C0204F14C01401CFFF778
:10FD400091F9002108A8FFF78BFA6078012805D007
:10FD500015203FE6D4E90912631DE4E70E20287060
:10FD600006208DF82000686ACDF824B00D90A078A8
:10FD70008DF82800CBE438780328C0D1E079C0079B
:10FD800070D00F202870072065E7387804286BD1E1
:10FD90001422391D04F11400FBF73FFB616A208C2B
:10FDA000A1F80900616AA078C871E179626A01F07E
:10FDB00003011172616A627A0A73616AA07A81F83A
:10FDC000240016205DE485F800A08DF82090696A73
:10FDD00050460D9192E00000368D010038780528DC
:10FDE00042D1B868A8616178606A022901D0012116
:10FDF00000E0002101EB4101142606EBC10140584F
:10FE0000082102F0E2F96178606A022901D001213B
:10FE100000E0002101EB410106EBC101425802A8BC
:10FE2000E169FFF70BFA6078626A022801D00120CD
:10FE300000E0002000EB4001102000EBC100022395
:10FE4000105802A90932FEF7EEFF626AFD4B0EA8B8
:10FE50000932A169FFF7E1F96178606A022904D0EB
:10FE6000012103E044E18DE0BFE0002101EB41010D
:10FE7000182606EBC101A27840580EA9FBF7CDFA6F
:10FE80006178606A022901D0012100E0002101EBC4
:10FE9000410106EBC1014158A0780B18C0F11002D6
:10FEA00000211846FBF7E3FA05208DF82000686A68
:10FEB0000D90A8690A90ADF824A08DF830B0062105
:10FEC00001706278616A022A01D0012200E00022FA
:10FED00002EB420206EBC202401C89581022FBF7DB
:10FEE0009CFA002108A8FFF7BBF91220C5F818B04A
:10FEF00028708DF82090686A0D900B208DF82400F2
:10FF000005E43878052870D18DF82000686A0D90D6
:10FF1000B8680A900B20ADF824000A9807210170F8
:10FF20006178626A022901D0012100E0002101EB21
:10FF30004103102101EBC30151580988A0F80110B9
:10FF40006178626A022902D0012101E02FE10021DB
:10FF500001EB4103142101EBC30151580A6840F839
:10FF6000032F4968416059E01920287001208DF85D
:10FF7000300074E6162028708DF830B0002108A8F3
:10FF8000FFF76EF9032617E114202870AEE63878E3
:10FF900005282AD18DF82000686A0D90B8680A906B
:10FFA000ADF824A08DF830B080F800906278616AD6
:10FFB0004E46022A01D0012200E0002202EB42025A
:10FFC0001C2303EBC202401C89581022FBF725FAC0
:10FFD000002108A8FFF744F9152028708DF820604B
:10FFE000686A0D908DF8246039E680E0387805283D
:10FFF0007DD18DF82000686A0D90B8680A90ADF840
:020000040001F9
:10000000249009210170616909784908417061698A
:1000100051F8012FC0F802208988C18020781C285F
:10002000A8D1A1E7E078C00702D04FF0060C01E0AC
:100030004FF0070C607802280AD000BF4FF0000094
:1000400000EB040101F1090105D04FF0010004E0CB
:100050004FF00100F4E74FF000000B78204413EA62
:100060000C030B7010F8092F02EA0C02027004D185
:100070004FF01B0C84F800C0D2B394F801C0BCF15F
:10008000010F00D09BB990F800C0E0465FEACC7C3D
:1000900004D028F001060670102606E05FEA887C8E
:1000A00005D528F00206067013262E70032694F854
:1000B00001C0BCF1020F00D092B991F800C05FEA14
:1000C000CC7804D02CF001060E70172106E05FEA10
:1000D0008C7805D52CF002060E70192121700026AF
:1000E0000078D0BBCAB3C3BB1C20207035E012E03F
:1000F00002E03878062841D11A2015E4207801283A
:100100003CD00C283AD02046FFF7EBF809208DF8B8
:100110002000686A0D9031E03878052805D0062067
:10012000387003261820287046E005208DF820003E
:10013000696A0D91B9680A910221ADF82410012174
:100140008DF830100A990870287D4870394608A843
:10015000FFF786F8064618202870012E0ED02BE0F7
:1001600001208DF82000686A0D9003208DF824008E
:10017000287D8DF8250085F814B012E0287D80B127
:100180001D202070172028708DF82090686A0D902F
:1001900002208DF82400394608A8FFF761F80646CA
:1001A0000AE00CB1FE2020709DF8200020B1002153
:1001B00008A8FFF755F80CE413B03046BDE8F08FFF
:1001C0002DE9F04387B00C464E6900218DF80410EC
:1001D00001202578034602274FF007094FF0050C50
:1001E00085B1012D53D0022D39D1FE2030708DF80C
:1001F0000030606A059003208DF80400207E8DF8A1
:10020000050063E02179012925D002292DD0032999
:1002100028D0042923D1B17D022920D131780D1FA6
:10022000042D04D30A3D032D01D31D2917D12189A3
:10023000022914D38DF80470237020899DF80410CE
:10024000884201E02E8D010018D208208DF80000B0
:10025000606A059057E070780128EBD0052007B060
:10026000BDE8F0831D203070E4E771780229F5D1F4
:1002700031780C29F3D18DF80490DDE7083402F8C9
:1002800004CB94E80B0082E80B000320E7E7157825
:10029000052DE4D18DF800C0656A05959568029535
:1002A0008DF8101094F80480B8F1010F13D0B8F154
:1002B000020F2DD0B8F1030F1CD0B8F1040FCED12E
:1002C000ADF804700E202870207E6870002168460A
:1002D000FEF7C6FF0CE0ADF804700B202870207EFE
:1002E000002100F01F0068706846FEF7B9FF377004
:1002F0000020B4E7ADF804708DF8103085F800C028
:10030000207E6870277011466846FEF7A9FFA6E7B1
:10031000ADF804902B70207F6870607F00F00100C2
:10032000A870A07F00F01F00E870E27F2A71C0076C
:100330001CD094F8200000F00700687194F82100A8
:1003400000F00700A87100216846FEF789FF2868C1
:10035000F062A8883086A87986F83200A0694078D3
:1003600070752879B0700D203070C1E7A97169717E
:10037000E9E700B587B004280CD101208DF8000012
:100380008DF80400002005918DF8050001466846AF
:10039000FEF766FF07B000BD70B50C46054602F0DB
:1003A000F3F921462846BDE870407823002202F088
:1003B00041B908B1007870470C20704770B50C0047
:1003C00005784FF000010CD021702146F2F725FF8F
:1003D00069482178405D884201D1032070BD022028
:1003E00070BDF2F71AFF002070BD0279012A05D016
:1003F00000220A704B78012B02D003E004207047E2
:100400000A758A6102799300521C0271C15003205F
:100410007047F0B587B00F4605460124287905EBF3
:10042000800050F8046C7078411E02290AD25249AB
:100430003A46083901EB8000314650F8043C284622
:10044000984704460CB1012C11D12879401E10F0B8
:10045000FF00287101D00324E0E70A208DF8000096
:10046000706A0590002101966846FFF7A7FF032CEC
:10047000D4D007B02046F0BD70B515460A460446F4
:1004800029461046FFF7C5FF064674B12078FE28BE
:100490000BD1207C30B100202870294604F10C00DB
:1004A000FFF7B7FF2046FEF71CFF304670BD7047D0
:1004B00070B50E4604467C220021FAF7D8FF0225CB
:1004C000012E03D0022E04D0052070BD01206070E3
:1004D00000E065702046FEF704FFA575002070BDA2
:1004E00028B1027C1AB10A4600F10C01C4E70120D0
:1004F000704710B5044686B0042002F045F9207814
:10050000FE2806D000208DF8000069462046FFF73F
:10051000E7FF06B010BD7CB50E4600218DF8041033
:100520004178012903D0022903D0002405E00469A1
:1005300000E044690CB1217C89B16D460146284632
:10054000FFF753FF032809D1324629462046FFF71B
:1005500093FF9DF80410002900D004207CBD04F115
:100560000C05EBE730B40C460146034A204630BC8C
:10057000024B0C3AFEF751BE748D01002E8D010026
:1005800070B50D46040011D085B122010021284626
:10059000FAF76DFF102250492846FAF73EFF4F4800
:1005A0000121017044704560002070BD012070BDC4
:1005B00070B505460024494E11E07068AA7B00EB37
:1005C0000410817B914208D1C17BEA7B914204D126
:1005D0000C222946FAF7F4FE30B1641CE4B23078FC
:1005E0008442EAD3002070BD641CE0B270BD70B5D7
:1005F0000546FFF7DDFF002805D1384C20786178EB
:10060000884201D3002070BD6168102201EB001008
:100610002946FAF702FF2078401CC0B2207070BD56
:100620002E48007870472D490878012802D0401ED6
:1006300008700020704770B50D4600219170144677
:100640001180022802D0102815D105E0288890B129
:100650000121A17010800CE0284613B1FFF7C7FFFD
:1006600001E0FFF7A5FFA07010F0FF0F03D0A889ED
:100670002080002070BD012070BD0023DBE770B535
:10068000054614460E0009D000203070A8780128D5
:1006900006D003D911490A7890420AD9012070BDC9
:1006A00024B1287820702888000A50700220087031
:1006B0000FE064B14968102201EB001120461039A7
:1006C000FAF7ABFE287820732888000A60731020A0
:1006D0003070002070BD0000838D01007C00002080
:1006E0002DE9F04190460C4607460025C2EB481123
:1006F000FE48072F00EB410607D2DFE807F00707A7
:10070000070704040400012500E0FFDF06F8147069
:10071000002D13D0F5487C3000EB880191F82700BC
:100720001F2803D006EB4000447001E081F826400A
:1007300006EB44021F20507081F82740BDE8F0818D
:10074000F0B51F4614460E4605461F2A00D1FFDFAE
:10075000E648C7EB471100EB410CE4490CEB4400C1
:100760007C3101EB87021F2E07D00CEB460140784D
:100770004B78487018461F210AE092F825304078DF
:1007800082F82500F6E701460CEB41000570407841
:10079000A142F8D192F827401F2C03D00CEB44045F
:1007A000637001E082F826300CEB41041F23637074
:1007B00082F82710F0BD30B50D46CD4B441900220C
:1007C000181A72EB020100D2FFDFCA48854200DD31
:1007D000FFDFC8484042854200DAFFDFC448401CC2
:1007E000844207DA002C01DB204630BDC048401CA3
:1007F000201830BDBE48C043FAE710B50446016872
:10080000407ABD4A52F82020114450B102200844D9
:1008100020F07F40F8F7CFF994F90810BDE81040B8
:10082000C9E70420F3E72DE9F047B04E7C3696F88F
:100830002D50DFF8B89206EB850090F8264036E0A0
:10084000C5EB451109EB41074FF0070817F81400F5
:10085000012806D004282ED005282ED0062800D046
:10086000FFDF01F04FF9014607EB4400427806EB49
:10087000850080F8262090F82720A24202D11F226E
:1008800080F82720084601F048F92A462146012031
:10089000FFF726FF9948414600EB04100268204606
:1008A000904796F82D5006EB850090F826401F2CB7
:1008B000C6D1BDE8F087022000E003208046D0E7E3
:1008C00010B58A4C1F217C3484F8251084F826103A
:1008D00084F82710002084F8280084F82D0084F87C
:1008E0002E10411EA16044F8100B20746074207318
:1008F0006073A0738249E07720750870487000210A
:100900007A4A103C02F81100491CC9B21F29F9D3D8
:100910000120F8F744F80020F8F741F8012084F8A6
:100920002200F2F7CDFA7748F2F7DFFA744CA41EF2
:1009300020707548F2F7D9FA6070BDE81040F7F7FB
:10094000BBBF10B5F7F7DDFF6D4CA41E2078F2F7A2
:10095000E5FA6078F2F7E2FABDE8104001F00AB972
:100960001F2070470020F7F7F3BF70B5054601243C
:100970000E46AC405AB1FFF7F5FF0146634800EB65
:10098000C500C0F81015C0F81465614801E0604862
:10099000001D046070BD2DE9F34F544D00247C35DB
:1009A00005EB810A89B09AF825001F2823D0611E23
:1009B00002915249009401EB0017391D03AB07C99E
:1009C00083E8070005F11400A0460189ADF81C106A
:1009D000807A8DF81E009DF81500C8B102264649A0
:1009E00051F820400399A219114421F07F4101914F
:1009F00084B102210FE00120F7F7D1FF0020F7F7C3
:100A0000CEFFF7F79CFF01F0B5F885F82F40A9E07D
:100A10000426E4E700218DF81810022801D00128EF
:100A200020D1039801190998081A801C9DF81C1000
:100A300020F07F4001B10221353181420BD20320E9
:100A40008DF815000398C4F13201401A20F07F4060
:100A5000322403900CE095F8240018B901F06DFAE7
:100A6000002863D0322C03D214B101F077F801E0F2
:100A700001F080F8224A107818B393465278039B0D
:100A8000121B00219DF81840994601281AD003280E
:100A900018D000208DF81E00002A04DD981A03905B
:100AA00001208DF818009DF81C0000B10221039868
:100AB000184A20F07F40039003AB099801F066F8D4
:100AC00010B110E00120E5E79DF81D0018B99BF872
:100AD0000000032829D08DF81C80CDF80C908DF8EB
:100AE00018408DF81E809DF8180015E0C007002002
:100AF000FF7F841E0020A107948D0100D0050020F7
:100B000086000020E32401002708010000F00140D6
:100B100004F50140FFFF3F0058B1039801238119FC
:100B200000221846F7F78EFF06E000200BB0BDE864
:100B3000F08F0120F7F733FF97F90C2001230020F5
:100B40000199F7F77FFFF87BC00701D0F8F75FF84E
:100B5000012085F82F008AF8288020226946FE4867
:100B6000FAF75BFC0120E1E72DE9F05FDFF8E883AD
:100B7000064608EB860090F825501F2D21D0A8F1DD
:100B80007C01C6EB46102C4601EB4007A1F5F87935
:100B9000DFF8C8B305E0A24607EB4A0044781F2CF3
:100BA0000AD0F7F79AFF09EB04135A4601211B1DDF
:100BB00000F0ECFF0028EED0AC4202D033465246A3
:100BC0001EE0E74808B1AFF30080F7F786FF98F81A
:100BD0002F206AB1D8F80C20411C891A0902CA17C3
:100BE00001EB12610912002902DD0020BDE8F09F2F
:100BF0003146FFF7D0FE08B10120F7E733462A4619
:100C00001F210420FFF79CFDEFE72DE9F041D24CB6
:100C10002569F7F762FF401B0002C11700EB116066
:100C2000001200D4FFDF94F8220000B1FFDF01279B
:100C300084F8227094F82E001F2800D1FFDF94F86A
:100C40002E601F2084F82E00002584F82F5084F891
:100C5000205084F82150C34825600078022835D000
:100C6000032833D000202077A068401C05D04FF027
:100C7000FF30A0600120F7F792FE0020F7F78FFE0B
:100C8000F7F786FFF7F77EFFF7F759FE07F080F9D1
:100C9000B548056005604FF0E0214FF40040B846CC
:100CA000C1F88002F2F794F894F82D703846FFF7F7
:100CB0005BFF0028FAD0A849C7EB47107C3901EB4D
:100CC000400010F81600022802D006E00120CAE712
:100CD0003A4631460620FFF703FD84F8238004EBF3
:100CE000870090F826001F2804D09E48801E407878
:100CF000F2F71AF9207F002803D0F7F739FF25779C
:100D000065771BE5944910B591F82D20924B00248E
:100D1000C2EB42117C3B03EB410100BF11F81430E0
:100D20002BB1641CE4B21F2CF8D31F2010BD8F49D7
:100D300001EB041108600020C87321460120FFF771
:100D4000CFFC204610BD10B5012801D0032800D1EA
:100D500081B3814A92F82D307F4C0022C3EB4313BC
:100D60007C3C04EB430300BF13F812400CB1082095
:100D700010BD521CD2B21F2AF6D37A4A48B10228BB
:100D800007D0072917D2DFE801F01606080A0C0E73
:100D9000100000210AE01B2108E03A2106E058215A
:100DA00004E0772102E0962100E0B5215170107037
:100DB000002010BDFFE70720FBE76A4810B5407828
:100DC000F7F7F9FE80B2F4E710B51F2815D2624993
:100DD00091F82D20C2EB4213A1F17C0202EB4304F7
:100DE00014F810304BB191F82D30C3EB431302EBE4
:100DF000430212F81020012A01D00020D9E791F80F
:100E00002D2001460020FFF76BFC0120D1E710B533
:100E1000F7F763FEBDE81040F7F7CDBE2DE9F041CE
:100E20000E464D4F01781F257C3FC3EB43130C4604
:100E300007EB430303E0254603EB45046478944243
:100E400002D01F2CF7D108E01F2C06D0A14206D1FA
:100E500003EB41014978017007E000206EE403EBE9
:100E6000440003EB450140784870414F7EB127B103
:100E7000002140F22D40AFF300803078A04206D12F
:100E800027B100214FF48660AFF30080357027B1A1
:100E9000002140F23540AFF3008001204EE410B550
:100EA00042680B689A1A1202D41702EB14621212EB
:100EB00016D4497A91B1427A82B92E4A006852F822
:100EC0002110126819441044001D891C081A0002E0
:100ED000C11700EB11600012322801DB012068E726
:100EE000002066E72DE9F0478146204EC1EB411016
:100EF00006F5F8719846144601EB400713E000BF71
:100F000006EB0415291D4846FFF7C9FF68B988F8A4
:100F10000040A97B99F80A00814201D80020C8E46A
:100F200007EB440044781F2CEAD10120C1E42DE9ED
:100F3000F047824608480E4600EB8600DFF82C801A
:100F400090F825401F201070C1EB461099461546B9
:100F500008F5F87110E000003C080020FFFF3F009A
:100F6000000000008600002000F50040D0050020B1
:100F700000000000948D010001EB40070BE000BF72
:100F800008EB04105146001DFFF789FF28B107EB5D
:100F900044002C7044781F2CF2D1297889F8001075
:100FA0004B46224631465046BDE8F0479AE72DE9C8
:100FB000FC410F4604460025FE4E0FE09DF8000060
:100FC000256806EB00108168204600F0F3FD2068DC
:100FD000A84202D10020BDE8FC8101256B4601AA90
:100FE00039462046FFF7A3FF0028E7D02846F2E75E
:100FF00070B50446C0EB44110125EF48A54300EB52
:101000004101C5EB451200EB42003E22FAF705FA1A
:10101000EA4E26B1002140F29D40AFF30080E64841
:101020007C3000EB850100EB8400D0F82500C1F88E
:10103000250026B1002140F2A140AFF300802846F0
:1010400070BD8A4203D003460520FFF779BB1F29F4
:1010500008D0D94AC0EB401002EB400000EB410041
:1010600040787047D4497C3101EB800090F825002E
:101070007047D04901EB0010001DFFF7BEBB7CB5E7
:101080001D46134604460E4600F108022146184646
:10109000F7F79EFD94F908000F2804DD1F38207231
:1010A0002068401C206096B10220C54951F82610E6
:1010B000461820686946801B20F07F40206094F924
:1010C00008002844C01C1F2803DA012009E004207E
:1010D000EBE701AAF7F77CFD9DF8040010B100983A
:1010E000401C00900099206831440844C01C20F046
:1010F0007F4060607CBDFEB50C460646097860798D
:10110000907220791F461546507279B121790022DC
:101110002846A368FFF7B3FFA74928467C3191F81A
:101120002E201F2A0AD00969491D0DE0D4E90223A7
:10113000217903B02846BDE8F040A0E7A1494978ED
:10114000052900D20521314421F07F4100F032FD14
:1011500039462846FFF72BFFD4E902322179684649
:10116000FFF78DFF2B4600213046019A00F00EFD5F
:10117000002806D103B031462846BDE8F04000F013
:1011800019BDFEBD2DE9F14F84B000F0CFFCF0B1E8
:1011900000270498007800284FF000006DD1864D9C
:1011A000864C824683467C3524B1002140F20450AF
:1011B000AFF3008095F82D8085F823B0002624B188
:1011C000002140F20950AFF3008017B105E001277C
:1011D000DFE74046FFF70CFF804624B1002140F2D4
:1011E0001150AFF30080F7F778FC814643466A461A
:1011F0000499FFF780FF24B1002140F21750AFF3AC
:10120000008095F82E001F280CD029690098401AFC
:101210000002C21700EB1260001203D5684600F00E
:10122000C9FC01264CB1002140F22150AFF30080EF
:10123000002140F22650AFF300806B46624A002145
:10124000484600F0A3FC98B127B941466846FFF72D
:10125000AEFE064326B16846FFF7CFFA04998860D0
:101260004FF0010A24B1002140F23A50AFF3008060
:1012700095F82300002897D1504605B057E42DE992
:10128000F04F89B08B46824600F050FC4A4C7C34CB
:1012900030B39BF80000002710B1012800D0FFDF19
:1012A000464D25B1002140F2F950AFF3008041498D
:1012B000012001EB0A18A946CDF81C005FEA0906D7
:1012C00004D0002140F20160AFF30080079800F0E5
:1012D00024FC94F82D50002084F8230067B119E015
:1012E00094F82E0001271F2800D1FFDF9BF8000093
:1012F0000028D5D0FFDFD3E72846FFF779FE054663
:1013000026B1002140F20B60AFF3008094F8230077
:101310000028D3D126B1002140F21560AFF3008040
:10132000F7F7DBFB2B4602AA59460790FFF7E3FECF
:1013300098F80F005FEA060900F001008DF813002D
:1013400004D0002140F21F60AFF300803B462A46E4
:1013500002A9CDF800A0079800F037FC064604EB80
:10136000850090F828000090B9F1000F04D000210A
:1013700040F22660AFF3008000F0C4FB0790B9F1A3
:10138000000F04D0002140F22C60AFF3008094F8ED
:101390002300002892D1B9F1000F04D0002140F2BF
:1013A0003460AFF300800DF1080C9CE80E00C8E932
:1013B00001120BE0D0050020C00700200000000053
:1013C000948D010086000020FFFF3F00C8F80C301C
:1013D0004EB35FEA090604D0002140F24160AFF34A
:1013E00000800098B84312D094F82E001F280ED128
:1013F00026B1002140F24660AFF300802846FFF797
:10140000B3FB20B99BF80000D8B3012849D0B9F14B
:10141000000F04D0002140F26360AFF30080284643
:1014200000F069FB01265FEA090504D0002140F2C3
:101430006C60AFF30080079800F06FFB25B10021CE
:101440004FF4CE60AFF300808EB194F82D0004EB22
:10145000800090F826001F2809D025B1002140F215
:101460007760AFF30080FA484078F1F75DFD25B171
:10147000002140F27C60AFF3008009B03046BDE847
:10148000F08FFFE7B9F1000F04D0002140F24E6069
:10149000AFF3008094F82D2051460420FFF720F987
:1014A000C0E7002E3FF40AAF002140F25960AFF3CD
:1014B000008003E72DE9F84FE64D814695F82D00B1
:1014C0004FF00008E44C4FF0010B474624B10021D7
:1014D00040F28A60AFF30080584600F01EFB85F8AA
:1014E000237024B1002140F28F60AFF3008095F8A3
:1014F0002D00FFF77DFD064695F8230028B1002C4E
:10150000E4D0002140F295604DE024B1002140F28A
:101510009960AFF30080CF49C6EB46107C3901EBF0
:10152000400111F81900032856D1334605EB830A10
:101530004A469AF82500904201D1012000E000209F
:1015400000900AF125000021FFF768FC0146009891
:10155000014203D001228AF82820AF77E1B324B1F9
:10156000002140F29E60AFF30080324649460120E0
:10157000FFF7B6F89AF828A024B1002140F2A9603C
:10158000AFF3008000F0BEFA834624B1002140F2A0
:10159000AE60AFF3008095F8230038B1002C95D0F1
:1015A000002140F2B260AFF300808FE7BAF1000F84
:1015B00007D095F82E001F2803D13046FFF7D4FA44
:1015C000E0B124B1002140F2C660AFF300803046A4
:1015D00000F091FA4FF0010824B1002140F2CF60F1
:1015E000AFF30080584600F098FA24B1002140F291
:1015F000D360AFF300804046BDE8F88F002CF1D0F7
:10160000002140F2C160AFF30080E6E70120F7F768
:101610009FB98F48007870472DE9F0418D4C94F8C0
:101620002E001F2821D194F82D6004EB860797F82F
:1016300025501F2D00D1FFDF8649C6EB46107C39AF
:1016400001EB400000EB4500407807F8250F012032
:10165000F87084F82300294684F82E503246022080
:101660002234FFF73DF80020207017E42DE9F04107
:101670007A4E784C012538B1012821D0022879D042
:1016800003287DD0FFDF09E400F068FAFFF7C4FF0C
:10169000207E00B1FFDF84F821500020F7F77FF9AA
:1016A000A168481C04D0012300221846F7F7CAF9A4
:1016B00014F82E0F217806EB01110A68012154E07D
:1016C000FFF7AAFF0120F7F76AF994F8210050B15B
:1016D000A068401C07D014F82E0F217806EB0111EA
:1016E0000A68062141E0207EDFF86481002708F1C6
:1016F0000208012803D002281ED0FFDFB5E7A77734
:10170000F7F736FA98F80000032801D165772577B6
:10171000607D534951F8200094F8201051B948B128
:1017200061680123091A00221846F7F78BF9022095
:1017300020769AE7277698E784F8205000F00EFA92
:10174000A07F50B198F8010061680123091A0022B6
:101750001846F7F777F9257600E0277614F82E0F6C
:10176000217806EB01110A680021BDE8F04110471D
:1017700000E005E036480078BDE8F041F1F7D4BB61
:10178000FFF74AFF14F82E0F217806EB01110A68C3
:101790000521EAE710B52F4C94F82E001F2800D140
:1017A000FFDF14F82E0F21782C4A02EB01110A6892
:1017B000BDE81040042110477CB5264C054694F83E
:1017C0002E001F2800D1FFDFA068401C00D0FFDFE3
:1017D00094F82E00214901AA01EB0010694690F906
:1017E0000C002844F7F7F4F99DF904000F2801DDF7
:1017F000012000E00020009908446168084420F0BE
:101800007F41A16094F82100002807D002B0012395
:10181000BDE8704000221846F7F714B97CBD30B51A
:10182000104A0B1A541CB3EB940F1FD3451AB5EB97
:10183000940F1BD3934203D9101A43185B1C15E075
:10184000954211D9511A0844401C43420EE0000051
:10185000840000203C08002000000000D00500208B
:10186000948D0100FF7F841EFFDF0023184630BDEA
:101870000123002201460220F7F7E4B80220F7F71F
:101880008EB8F7F72AB92DE9FE4FF34C05468A4684
:1018900094F82E001F2800D1FFDFEF4E94F82E1091
:1018A000A0462046A6F51B7202EB01141F218DF8FD
:1018B000001090F82D10376900EB8101D8F8000076
:1018C00091F82590284402AA01A90C36F7F780F96F
:1018D0009DF90800002802DD0198401C0190A068D5
:1018E0000199642D084454D3DC4B00225B1B72EB3E
:1018F00002014ED36168411A21F07F41B1F5800F9A
:1019000047D220F07F40706086F80AA098F82D102A
:1019100044466B464A463046FFF7E4FAC0B3A06837
:10192000401C10D0F7F7D9F8A168081A0002C117B7
:1019300000EB1160001202282DDD0120F7F72FF8CF
:101940004FF0FF30A06094F82D009DF800201F217B
:101950000F34FFF776FBA17FBF4AC1EB41117C3A00
:1019600002EB4101E27F01EB4201487054F80F0C99
:10197000284444F80F0C012020759DF800001F2812
:1019800003D0B7484078F1F7CFFA0120BDE8FE8FC9
:1019900001E00020FAE77760FBE72DE9F047AE4C65
:1019A000074694F82D00A4F17C06C0EB401006EB2E
:1019B000400010F8170000B9FFDF94F82D50A04642
:1019C000A84C24B1002140F6EA00AFF30080C5EB3B
:1019D000451040F6F60940F6FF0A06EB400600BF48
:1019E00016F81700012819D0042811D005280FD0A7
:1019F00006280DD01CB100214846AFF3008006F048
:101A000061FF002CECD000215046AFF30080E7E7E7
:101A10002A4639460120FEF763FEF2E74FF0010A3D
:101A20004FF00009454624B1002140F60610AFF3FF
:101A30000080504600F071F885F8239024B1002111
:101A400040F60B10AFF3008095F82D00FFF7D0FAA9
:101A5000064695F8230028B1002CE4D0002140F67A
:101A600011101FE024B1002140F61510AFF30080E3
:101A700005EB860000F1270133463A462630FFF792
:101A8000CDF924B1002140F61910AFF3008000F029
:101A900039F8824695F8230038B1002CC3D00021D4
:101AA00040F61F10AFF30080BDE785F82D600120E0
:101AB00085F82300504600F030F8002C04D00021B7
:101AC00040F62C10AFF30080BDE8F08730B5044637
:101AD00061480D4690F82D005F49C0EB40107C39FD
:101AE00001EB400010F8140000B9FFDF5E4800EB86
:101AF0000410C57330BD584981F82D00012081F8CC
:101B00002300704710B5594808B1AFF30080EFF3D8
:101B1000108000F0010072B610BD10B5002804D18D
:101B2000534808B1AFF3008062B610BD5148006859
:101B3000C005C00D10D0103840B2002804DB00F101
:101B4000E02090F8000405E000F00F0000F1E02034
:101B500090F8140D400970470820704710B53E4CAE
:101B600094F82400002804D1F7F7A6F8012084F89F
:101B7000240010BD10B5384C94F82400002804D07F
:101B8000F7F7C3F8002084F8240010BD10B51C68D6
:101B90005B68241A181A24F07F4420F07F40A14289
:101BA00006D8B4F5800F03D2904201D8012010BDB1
:101BB000002010BDD0E90032D21A21F07F43114439
:101BC00021F07F41C0E9003170472DE9FC41844696
:101BD000214815460F46C2EB45117C38089C00EBA6
:101BE000410616F81400012804D0022802D0002073
:101BF000BDE8FC813B46204A01216046FFF7C6FF55
:101C0000F0B101AB6A4629463846FFF790F9B8B102
:101C10009DF804209DF800102846FFF712FA06EB05
:101C2000440148709DF800001F280DD006EB4000CD
:101C300044702A4621460320FEF752FD0120D7E7D3
:101C40002A4621460420F7E70348012100EB8500DE
:101C500000F8254FC170ECE73C080020FF1FA107EA
:101C60008400002000000000D005002000000000DB
:101C70000000000004ED00E0FFFF3F002DE9F0410F
:101C8000044680074FF000054FF001060CD56B4865
:101C90000560066000F0E8F920B16948016841F488
:101CA0008061016024F00204E0044FF0FF3705D5A5
:101CB00064484660C0F8087324F48054600003D57B
:101CC0006148056024F08044E0050FD55F48C0F806
:101CD0000052C0F808735E490D60091D0D605C4A32
:101CE00004210C321160066124F48074A00409D52B
:101CF00058484660C0F80052C0F80873564805605E
:101D000024F40054C4F38030C4F3C031884200D0BE
:101D1000FFDF14F4404F14D050484660C0F80873F9
:101D20004F488660C0F80052C0F808734D490D60F6
:101D30000A1D16608660C0F808730D60166024F4F2
:101D4000404420050AD5484846608660C0F80873BC
:101D5000C0F848734548056024F4006406F0F2F8C2
:101D60004348044200D0FFDFBDE8F081F0B5002217
:101D7000202501234FEA020420FA02F1C9072DD0E1
:101D800051B2002910DB00BF4FEA51174FEA870715
:101D900001F01F0607F1E02703FA06F6C7F8806195
:101DA000BFF34F8FBFF36F8F0CDB00BF4FEA5117AC
:101DB0004FEA870701F01F0607F1E02703FA06F64E
:101DC000C7F8806204DB01F1E02181F8004405E0FE
:101DD00001F00F0101F1E02181F8144D02F101023F
:101DE000AA42C9D3F0BD10B5224C20600846F7F7CF
:101DF0007CF82068FFF742FF2068FFF7B7FF05F087
:101E0000D9FC00F092F906F09DF805F0DCFFF1F73F
:101E100057F8BDE8104005F081BD10B5154C20689D
:101E2000FFF72CFF2068FFF7A1FF06F08BF8F7F70C
:101E30004DF90020206010BD0A207047FC1F0040B3
:101E40003C17004000C0004004E501400080004015
:101E50000485004000D0004004D5004000E0004070
:101E600000F0004000F5004000B0004008B5004020
:101E7000FEFF0FFD8800002070B526490A680AB3EE
:101E80000022154601244B685B1C4B600C2B00D3D1
:101E90004D600E7904FA06F30E681E420FD0EFF380
:101EA000108212F0010272B600D001220C689C432D
:101EB0000C6002B962B649680160002070BD521C16
:101EC0000C2AE0D3052070BD4FF0E0214FF48000D4
:101ED000C1F800027047EFF3108111F0010F72B6E4
:101EE0004FF0010202FA00F20A48036842EA0302D4
:101EF000026000D162B6E7E7064800210160416058
:101F000070470121814003480068084000D001204B
:101F1000704700008C000020012081070860704796
:101F20000121880741600021C0F8001118480170A4
:101F3000704717490120087070474FF08040D0F873
:101F40000001012803D012480078002800D00120A9
:101F5000704710480068C00700D0012070470D4846
:101F60000C300068C00700D00120704709481430C9
:101F700000687047074910310A68D20306D509681E
:101F800001F00301814201D1012070470020704718
:101F900094000020080400404FF08050D0F8300139
:101FA0000A2801D0002070470120704700B5FFF7D4
:101FB000F3FF20B14FF08050D0F8340108B1002079
:101FC00000BD012000BD4FF08050D0F830010E2838
:101FD00001D000207047012070474FF08050D0F8AA
:101FE0003001062803D0401C01D00020704701209A
:101FF00070474FF08050D0F830010D2801D00020FC
:102000007047012070474FF08050D0F83001082809
:1020100001D000207047012070474FF08050D0F869
:102020003001102801D0002070470120704700B512
:10203000FFF7F3FF30B9FFF7DCFF18B9FFF7E3FF55
:10204000002800D0012000BD00B5FFF7C6FF38B161
:102050004FF08050D0F83401062803D3401C01D043
:10206000002000BD012000BD00B5FFF7B6FF48B15C
:102070004FF08050D0F83401062803D3401C01D023
:10208000012000BD002000BD0021017008467047FE
:102090000146002008707047EFF3108101F0010144
:1020A00072B60278012A01D0012200E00022012349
:1020B000037001B962B60AB1002070474FF40050B6
:1020C0007047E9E7EFF3108111F0010F72B64FF09E
:1020D0000002027000D162B600207047F2E70000F3
:1020E0002DE9F04115460E460446002700F0EBF8B6
:1020F000A84215D3002341200FE000BF94F84220EE
